:020000040800F2
:10000000E83D00209D010008D10C000839060008D9
:1000100000000000000000000000000000000000E0
:10002000000000000000000000000000D50C0008E7
:100030000000000000000000D30C0008F50D0008CF
:10004000AF010008AF010008AF010008AF010008D0
:10005000AF010008AF010008AF010008AF010008C0
:10006000AF010008AF010008AF0100083106000829
:10007000AF010008AF010008AF010008AF010008A0
:10008000AF010008AF010008AF010008AF01000890
:10009000AF010008AF010008AF010008AF01000880
:1000A000AF010008AF010008AF010008AF01000870
:1000B000AF010008AF010008AF010008AF01000860
:1000C00000F002F800F03EF80CA030C80838241800
:1000D0002D18A246671EAB4654465D46AC4201D180
:1000E00000F030F87E460F3E0FCCB6460126334274
:1000F00000D0FB1AA246AB4633431847085601000E
:1001000028560100103A02D378C878C1FAD85207AD
:1001100001D330C830C101D504680C6070470000BD
:100120000023002400250026103A01D378C1FBD813
:10013000520700D330C100D50B6070471FB51FBDFB
:1001400010B510BD00F03DFA1146FFF7F7FF10F0B3
:1001500043F800F055FA03B4FFF7F2FF03BC00F0D8
:1001600055FA000070B505460C46164602E00FCC65
:100170000FC5103E102EFAD2082E02D303CC03C5B1
:10018000083E042E07D301CC01C5361F03E02178B9
:100190002970641C6D1C761EF9D270BD074880471B
:1001A00007480047FEE7FEE7FEE7FEE7FEE7FEE75B
:1001B00004480549054A064B70470000690E0008CF
:1001C000C1000008E8300020E83D0020E8390020A8
:1001D000E8390020034670B502460B439B070FD158
:1001E0000E4CE60100E008C208C91D1B9D433542C4
:1001F000F9D0D9B21170521C00290DD01B0AF8E7B2
:100200000B78491C1370521C002B05D00B78491C2D
:100210001370521C002BF3D170BD000001010101CD
:1002200030B5441C03E00178401C00290DD0810743
:10023000F9D10B4BDD0104C8D11A91432940FAD002
:10024000001B0A0603D0C01E30BD001B30BD0A04CF
:1002500001D0801E30BD0902FCD0401E30BD000020
:1002600001010101F8B5042A2CD3830712D00B78C1
:10027000491C0370401C521E83070BD00B78491C8D
:100280000370401C521E830704D00B78491C037076
:10029000401C521E8B079B0F05D0C91ADF0020237C
:1002A000DE1B08C90AE0FFF75DFFF8BD1D4608C95F
:1002B000FD401C46B4402C4310C0121F042AF5D246
:1002C000F308C91A521EF0D40B78491C0370401C65
:1002D000521EEAD40B78491C0370401C012AE4D456
:1002E00009780170F8BD01E004C0091F0429FBD2A0
:1002F0008B0701D50280801CC90700D002707047AF
:1003000000290BD0C30702D00270401C491E0229ED
:1003100004D3830702D50280801C891EE3E70022F4
:10032000EEE70022DFE7000082078B079A4237D111
:1003300070B5920F0AD0032402780B78401C491C38
:10034000002A2BD09A4229D12042F5D11D4EF4012A
:1003500004C808C9951B9543254010D19A4207D17E
:1003600004C808C9951B9543254008D19A42EFD08F
:1003700012BA1BBA01209A4200D2404270BD12BA92
:100380001BBA2DBA18241000E0401900E140401AB1
:1003900005D12E00E64002D1083CF4D1D01A70BD40
:1003A00002780B78401C491C002A09D09A4207D1D8
:1003B00002780B78401C491C002A01D09A42EFD0E9
:1003C000D01A704701010101002203098B4273D347
:1003D000030A8B4258D3030B8B423CD3030C8B4252
:1003E00021D312E003460B437FD4002243088B4203
:1003F00074D303098B425FD3030A8B4244D3030BAC
:100400008B4228D3030C8B420DD3FF22090212BA70
:10041000030C8B4202D31212090265D0030B8B42EC
:1004200019D300E0090AC30B8B4201D3CB03C01AD6
:100430005241830B8B4201D38B03C01A5241430BB1
:100440008B4201D34B03C01A5241030B8B4201D3A1
:100450000B03C01A5241C30A8B4201D3CB02C01A0C
:100460005241830A8B4201D38B02C01A5241430A84
:100470008B4201D34B02C01A5241030A8B4201D373
:100480000B02C01A5241CDD2C3098B4201D3CB011A
:10049000C01A524183098B4201D38B01C01A5241C9
:1004A00043098B4201D34B01C01A524103098B42CD
:1004B00001D30B01C01A5241C3088B4201D3CB00B8
:1004C000C01A524183088B4201D38B00C01A52419B
:1004D00043088B4201D34B00C01A5241411A00D24B
:1004E00001465241104670475DE0CA0F00D04942B4
:1004F000031000D34042534000229C4603098B4224
:100500002DD3030A8B4212D3FC22890112BA030AAB
:100510008B420CD3890192118B4208D3890192112D
:100520008B4204D389013AD0921100E08909C309B2
:100530008B4201D3CB01C01A524183098B4201D3B4
:100540008B01C01A524143098B4201D34B01C01A9F
:10055000524103098B4201D30B01C01A5241C30817
:100560008B4201D3CB00C01A524183088B4201D386
:100570008B00C01A5241D9D243088B4201D34B00A1
:10058000C01A5241411A00D20146634652415B10E3
:10059000104601D34042002B00D5494270476346C4
:1005A0005B1000D3404201B50020C046C04602BDEA
:1005B0007047704770470000004870478430002043
:1005C00070477546FFF7F8FFAE460500694653468B
:1005D000C008C000854618B020B5FFF7E9FD60BC33
:1005E00000274908B6460026C0C5C0C5C0C5C0C55D
:1005F000C0C5C0C5C0C5C0C5403D49008D46704797
:100600000446C046C0462046FFF7A5FD0149182014
:10061000ABBEFEE72600020001200349000448604B
:10062000024901204860704700000240E0000020BD
:1006300010B5FFF7F1FF10BDFEE7000010B5034A4B
:100640008021916200F0C8FB10BD0000000400484A
:1006500070B50D460646064980208861002404E0F6
:10066000305D00F0B9FB641CA4B2AC42F8D370BD9D
:100670000004004870B50C4605461049802088618A
:100680000F4E0F210902304600F0A2F90022304639
:100690000DE05100695A83689B07DB0FFBD0C160F6
:1006A000C16881680906C90FFBD1521C92B2A242EF
:1006B000EFD30721090200F08BF970BD0004004858
:1006C0000038004010B51120FFF7B8FF962000F069
:1006D0008DF92920FFF7B2FF962000F087F910BDB1
:1006E000F8B50646104D402017460C46A862CB8848
:1006F0008A884988208800F05FF8A088218862886D
:10070000401AE188401C891A491C48438021A9618C
:1007100081B2384600F0E0FA4020A861304607F088
:1007200037FA4020A861F8BD0004004870B500F019
:1007300071F900F0D9F90521134800F093F8134836
:10074000016840263143016000F026F8FFF7BAFF48
:10075000104D0F4CAE622078641C411ECEB20028B2
:100760000CD02078641CFFF769FF31462046FFF764
:100770006FFFA4190A2000F039F9ECE74020A861C6
:10078000282000F035F870BD00000240003800401D
:100790008B5601080004004810B5064C0820A062E2
:1007A0000A2000F023F90820A061322000F01EF991
:1007B00010BD000000040048F8B507461C46154669
:1007C0000E462A20FFF73AFF68460780458002213F
:1007D000FFF750FF2B20FFF731FF6846068044806B
:1007E0000221FFF747FF2C20FFF728FFF8BD00008C
:1007F00031B568460378FF2141310C48F022282B9F
:1008000010D0E82B0ED042800180094C4020A0621D
:100810003620FFF713FF01216846FFF719FF40203C
:10082000A06138BD41800280EFE70000E0000020B9
:100830000004004808B504494A6902434A6149690D
:100840000140009108BD00000010024008B50449B5
:10085000CA690243CA61C9690140009108BD00002C
:1008600000100240044A51182039C97F42585208EA
:10087000520042507047000084560108F0B4002333
:100880000A68002A51D001240A689C402240002AAC
:1008900047D04C68012C01D0022C10D18D68144631
:1008A000866864436700E719BE436C43264386604D
:1008B000CD680C684668A6436C43264346600F69C2
:1008C0001446C668644365006519AC46AE432546C8
:1008D0007D432E43C6604D68022D1BD1FF2A0CD8E4
:1008E0004F691646056A2246724372431601B61ACC
:1008F000B5437A43154305620CE04E69150A2A4652
:100900006A436A436A431501476AAD1AAF437243AB
:10091000174347624A6805686646B5435443254312
:1009200005605B1C0A68DA40ADD1F0BC002070475E
:1009300010B57D21C900FFF747FD0449401E4861FD
:10094000002088610520086110BD000000E000E083
:1009500030B4012203685B06DB0FD402002B2DD1DB
:100960004B680A680D691A43CB682B431A434B69DD
:100970001A438B691A43CB691A430B6A1A430368FB
:10098000114D2B401A4302604268104B1A404B69CC
:100990001B0C1A438B681A4342608A68A24204D235
:1009A000630042689A431A43426001230A6A5B0368
:1009B0009A4202D1898C89B201610022C169A143A6
:1009C000C16130BC104670474000FFFFFBF0FFFFE5
:1009D00042680F231B029A430A434260704700009B
:1009E0000149086070470000E800002081B0084914
:1009F0000A690092421C00D0401C002805D00A69F8
:100A0000D20300D5401E0028F9D101B07047000084
:100A100000E000E008B50948012142690A4342614B
:100A2000406908400090064801680902090A01600F
:100A300001200449C002086008BD00000010024007
:100A400008E400E000E100E0F0B587B01821684656
:100A5000FFF767FC0120C004FFF7ECFE01208005D2
:100A6000FFF7E8FE01208004FFF7E4FE01204004C8
:100A7000FFF7E0FE01201B4D8002A8620821A96259
:100A80002021A9624021A9628021A96201240326B4
:100A900000276946D1C1694628460494FFF7EEFE57
:100AA00008206946D1C1694628460494FFF7E6FE4E
:100AB00020206946D1C1694628460494FFF7DEFE2E
:100AC00040206946D1C1694628460494FFF7D6FE06
:100AD00080206946D1C1694628460494FFF7CEFEBE
:100AE00007B0F0BD0004004870B592B028216846F8
:100AF000FFF717FC18210AA8FFF713FC2D48012166
:100B0000C26989030A43C261C06900240840109089
:100B1000072040030A9002200B9003200C900AA9A2
:100B20000D942548FFF7AAFE254924480D79102287
:100B30004359244E3340134343510A7983580325C4
:100B40002D03AB4383500B79C2582025AA43C250D2
:100B50000B79C2584025AA43C2500D7942598023CF
:100B60009A431A4342510B798515C258032636021F
:100B7000B2432A43C2500A7903158158B500A943EC
:100B80001943815028010090FF2005300190072073
:100B900000020290581005900494072003940990D5
:100BA00006940794089469460748FFF7D1FE12B0EF
:100BB00070BD000000100240000400480000024028
:100BC00084560108EFBFFFFF00380040F0B591B038
:100BD000282106A8FFF7A5FB18216846FFF7A1FB0F
:100BE0000127BF033846FFF731FE3801FFF722FE29
:100BF0000024781002250326039404946A46059481
:100C000061C269462D48FFF739FE009703940494AA
:100C100069462A48029601950594FFF72FFEA8031E
:100C2000039404946A46059461C269462348FFF719
:100C300025FE244922480B791025C258224E324005
:100C40002A43C2500A79835803252D03AB438350AE
:100C50000B79C2582025AA43C2500B79C2584025AF
:100C6000AA43C2500D79425980239A431A434251F4
:100C70000B798515C25803263602B2432A43C25067
:100C8000097903154258B500AA431A434250280176
:100C90000690FF20053007900720000208905810AA
:100CA0000B900A94072009940F900C940D940E94C5
:100CB00006A90648FFF74CFE11B0F0BD000400483D
:100CC00000000240FC560108EFBFFFFF0038004063
:100CD000FEE7704770470000F3B50F46394C0F210F
:100CE00081B009022046FFF773FE2168402081434E
:100CF0002160354D05212846FFF7B4FD6015686079
:100D00008000686060680226304360602F4C207964
:100D10002958314329502079295808221143295054
:100D2000052128461B3CFFF79DFDE17F281D0A5841
:100D3000120C12043A430A50E37F2248EA58019900
:100D40000C30234F3A40204F0C37102A34D03A1F32
:100D50009950E17FC851E07F295801221143295061
:100D6000184F38684021084338601A484168002904
:100D7000FCD00021416005212846FFF773FD3A6849
:100D8000384640218A433A60CA006A604A016A6074
:100D90007A68B2437A60E27FAB58B343AB50E27FEC
:100DA000AB580824A343AB5002680A4302600721F2
:100DB0000902FFF70DFEFEBDD9510349E27F08315C
:100DC0005050C8E700380040000002408456010837
:100DD00010400000E000002005498A689207D20F09
:100DE000FBD00873C86888680006C00FFBD1704745
:100DF000003800407047000010B5184801684908E5
:100E0000490001600168C907C90FFBD11448016896
:100E100001221143016001688907C90FFBD00168F5
:100E2000F82291438022114301604168F0229143EE
:100E3000416041680722120291434160416889087C
:100E4000890041600C2241681142FCD1054C2046CA
:100E5000FFF76EFD2046FFF7C3FD10BD00200240E6
:100E60000010024000127A0070472021020C01D0CD
:100E700010211046020A01D010460839020901D09B
:100E80001046091F820801D01046891E420801D071
:100E9000881E7047081A704730B47446641E25785F
:100EA000641CAB4200D21D46635D5B00E31830BC9E
:100EB000184700008307FF22DB0E9A408907090EBE
:100EC0009940002808DB830809489B001B18186814
:100ED00090430843186070470007000F08388308E4
:100EE00004489B001B18D86990430843D861704799
:100EF00000E400E000ED00E010B54421074800F0F8
:100F000093FC00221E2106480EF056FD054CA06001
:100F100001F0ECF80020207010BD00001C11002032
:100F2000A9210008B8000020F7B50D4684B0164688
:100F30001146284600F007F9002809D00022314662
:100F4000284600F0B0F8002805D0002007B0F0BD1A
:100F50000020C043FAE700240422AA5E295F501A49
:100F600000B203900220EB88285E1B1A1FB2738820
:100F70001B1A1BB2002B0BDD6C4621806080A28007
:100F8000C018E0800124082269460498FFF76AF936
:100F90000620305E6988411A791A09B2002913DDEA
:100FA0000622AA5E90420FDA2B886A461380508090
:100FB0004018AB889380D080E1000498082208187C
:100FC0006946641CFFF74EF902200227305EEF5F8E
:100FD000B84200DD074606210620715E285E814288
:100FE00000DA0846C01B00B2029000223088AA5ED8
:100FF000801A01B2002913DD0298002810DD68462E
:10100000028047805118818002980822391868466A
:10101000C180E1000498641C08186946FFF722F9B2
:101020000420305E2988421A0399891A0AB2002ADC
:101030000FDD694608804F8080188880029808225A
:101040003818C880E1000498641C08186946FFF746
:1010500009F920467AE770B5002400230C5FD35EBF
:101060009C4200DD23460380022502244D5F145F6D
:10107000A54200DD2C464480042604258E5F555F82
:10108000AE4200DA3546858006268E5F0621515E27
:101090008E4200DB0E46C6800120AB4201DCB4422A
:1010A00000DD002070BDF8B50D460446002000218B
:1010B000205E695E1646884243DB02210222615EA1
:1010C000AA5E91423DDB04210422615EAA5E914248
:1010D00037DC06210622615EAA5E914231DC002ED9
:1010E0002DD069460880608848803246284600F046
:1010F00096F8002824D0A188684601806188418044
:1011000032466946284600F08AF8002818D021881F
:1011100068460180E188418032466946284600F0F1
:101120007EF800280CD0A18868460180E1884180C3
:1011300032466946284600F072F8002800D00120A7
:10114000F8BD0020F8BD00220423825ECB5E9A42E7
:1011500013DC04220023825ECB5E9A420DDB022266
:101160000623825ECB5E9A4207DC0622825E022064
:10117000085E824201DB0120704700207047F8B50D
:101180000D46044604200021205E695E1646884212
:1011900043DB06200221205E695E88423DDB0020A1
:1011A0000421205E695E884237DC02210622615EEE
:1011B000AA5E914231DC002E2DD0694608806088FD
:1011C00048803246284600F02AF8002823D1A1881A
:1011D000684601806188418032466946284600F0B1
:1011E0001EF8002817D1218868460180E1884180D7
:1011F00032466946284600F012F800280BD1A18833
:1012000068460180E188418032466946284600F000
:1012100006F8002801D00020F8BD0120F8BDFEB579
:1012200014460E4600210022715E825E0546914200
:1012300039DB0420285E814235DC02210227715E01
:10124000EF5FB9422FDB0623EB5E99422BDC002CCB
:1012500070DD801A401C00B2C10F08184110D81B65
:10126000401C00B2C30F18184010814200DA084633
:10127000844200DD04466846028028880022011965
:101280006846818069884180688801196846C18004
:101290003146FFF7C4FF002807D06846808801194F
:1012A000684681803DE00020FEBDE8886946001B5D
:1012B0004880E888C880002231466846FFF7AFFFC3
:1012C000002805D06846808801196846818011E0B1
:1012D000A8886946001B0880A888888000223146BB
:1012E0006846FFF79CFF002809D068460088011B6C
:1012F000684601804088011B6846418015E0688887
:1013000069464880688800220019C88031466846CE
:10131000FFF785FF00280DD068460088011B68464E
:101320000180C08801196846C18031460EF018F866
:10133000FEBDFFE70120FBE710B5002400230C5F92
:10134000D35E9C4200DA23460380022402230C5F12
:10135000D35E9C4200DA23464380042404230C5FBE
:10136000D35E9C4200DD234683800623CB5E0621AC
:10137000515E8B4200DC0B46C38010BDF8B50546BC
:101380000EF006FB00263D4C07460096002D06D0C9
:10139000E868606028460EF0DDFB606802E006F059
:1013A000FDFB606000690DF00BFF6068406900287C
:1013B00001D00DF005FF6068C0690DF001FF6068A5
:1013C000006A0DF0FDFE60680169002915D00EF07D
:1013D00037F80FF08FFD0FF0DFFBFF216068513110
:1013E000095A002942D00068017CC90722D0C06890
:1013F000406800281ED0002516E0FF3041300682EC
:10140000F8BD4119FF312131097C00290AD1FF3093
:10141000593000F062FA6268E90089180822303118
:10142000FEF720FF6D1CADB2FF2160685131095AF3
:10143000A942E6D86068FF21013130300AF0E3FEAE
:1014400060682021FF3031300AF0DDFE6068FF3037
:101450004130068238460EF094FA009060680068C9
:10146000436A002B02D02268009998470AF066FD73
:1014700000F032F800F004F8F8BD00002C00002065
:1014800070B50A4D002420461C2148430646A85941
:10149000002801D00AF0C2FD70191C210AF0B3FE29
:1014A000641CE4B2042CEED370BD0000781500205B
:1014B00008490122496809E04B68834202D00B6861
:1014C000834202D10B7E13430B7649690029F3D185
:1014D00070470000000000207047000010B5042194
:1014E000014800F0A1F910BD1011002010B5202115
:1014F000014800F099F910BD28110020F0B585B021
:10150000044600200B9F0A9E1D46002B02D1F31FAC
:10151000F93B29D000900190029003906B4699808E
:101520005A819981DA813B463246294668460DF058
:1015300075FE3B463246294601A80DF06FFE3B463C
:101540003246294602A80DF069FE3B46324629463E
:1015500003A80DF063FE6B4600200421185E595E5F
:10156000884209DA054608E02080491E6080A18093
:10157000521EE28005B0F0BD0D461E4608230C2227
:10158000F35EB25E934201DA1E4600E01646B542B3
:1015900003DA884206DA014604E0934201DA19468A
:1015A00000E01146891E2180684600210423415E27
:1015B000C35E994201DD0D4600E01D460646082047
:1015C0000C22305EB25E904201DD064600E0164617
:1015D000B54203DD994206DC194604E0904201DD84
:1015E000014600E01146891CA180684602230622BC
:1015F000C35E825E934201DA1D4600E01546064650
:101600000A200E21305E715E884201DA064600E053
:101610000E46B54205DA934201DA194604E0114656
:1016200002E0884200DA0146891E61806846022392
:101630000622C35E825E934201DD1D4600E0154630
:101640000A210646415E0E20305E814201DD0E46D3
:1016500000E00646B54205DD934201DD184604E090
:10166000104602E0814200DD0846801CE08081E7F0
:10167000F8B515460E460746124C0EF089F9009053
:101680002B4632463946204609F040FE002805D058
:101690000020A062E069002809D010E02C2120463B
:1016A0000AF0B1FD0120C007A0620020F8BD00983B
:1016B0000EF067F9E061002801D10120E0612046C9
:1016C000F8BD00004C11002010B51421084800F0AE
:1016D000ABF809F0E1FD002808D006490160064991
:1016E0004160064981600649C16010BDFEE7000007
:1016F0003411002059AC0008E1AF0008B5B1000872
:1017000023AC0008F0B585B00D46040003D106F007
:1017100045FA040030D006F0B3FA00282CD0282077
:10172000005D400728D40026002D22D068460680A0
:101730004680204606F04CFA411E684681802046CD
:1017400006F088FA411E6846C1806A46294602A80A
:10175000FFF781FC00280FD02068017C89070DD598
:1017600001990098616320630121FF2051300153EA
:101770002DE0FF344134268205B0F0BD8269002A95
:1017800001D002A9904725460027FF3541350AE0E0
:10179000F8000119002202A83031FFF784FC00286C
:1017A000EAD17F1CBFB2288AB842F1D880B2202883
:1017B00004D2C000001902A9303003E020462E8276
:1017C0003030694605F0CCFE288A401C28826068CB
:1017D0000028D1D00EF0CAF9CEE770B5054600F06A
:1017E00012F804460CE02146284600F010F80646A0
:1017F0002146284600F09DF820460AF00FFC3446AA
:10180000002CF0D170BD002800D0406870470068FF
:10181000091D40180068704700684018006870474C
:10182000002800D0806870470022C91C42608908E7
:10183000890082600160704770B504460068083016
:101840000AF064FB050015D00146002220460FF087
:101850002CF82946204662680FF020F861680029BC
:1018600003D02A4620460FF020F86560A0680028C3
:1018700000D1A560284670BDF8B50C4606000BD017
:10188000002C09D0FFF7BFFFA04207D13046FFF779
:10189000D3FF050001D01EE00020F8BD30680830FD
:1018A0000AF034FB0500F8D030682A4600190768B2
:1018B000304639460EF0F2FF3A46294630460EF0E1
:1018C000F4FF2A46214630460EF0EFFF2246294615
:1018D00030460EF0E3FF2846F8BD70B504460068B8
:1018E00008300AF013FB050015D0014600222046FF
:1018F0000EF0D4FF29462046A2680EF0D6FFA1685C
:10190000002903D02A4620460EF0C8FFA560606873
:10191000002800D16560284670BD002807D04168C6
:10192000002902D18068002801D0002070470120E2
:10193000704770B504000DD0FFF765FF00228842A4
:10194000204608D1FFF763FF6060010001D000224C
:101950001FE0A26070BDFFF763FF884220680BD1D3
:1019600040180168A160002904D0002220460EF032
:1019700095FF70BD626070BD401805682046FFF796
:1019800046FF06460246294620460EF087FF2A46B5
:10199000314620460EF089FF70BD8168002902D0D3
:1019A0001620085E7047002070478068002801D02C
:1019B000807E8009704770B50546164608460C467D
:1019C00030431AD028460AF07DFCA8680123018A1A
:1019D000324609190182A868418A89194182214643
:1019E00028460CF0CAFB00220B21284608F092FC86
:1019F000012803D128460CF040FB012070BD77B5CB
:101A000081B00E46050017D062220CF000F80400E9
:101A100012D0206800280FD02846314663220BF0F0
:101A2000F6FF0206120E07D0236820460399984756
:101A30000090684601888181039804B070BD000061
:101A4000FFB50646408C99B008210843229D70845A
:101A50001B9830842A8930461A990BF0D8FF044627
:101A600011901C9830842A8930461A990BF0CFFFC8
:101A70001290728C08218A4307467284844204D1F2
:101A800010A88188008981426AD01B9830842A89F5
:101A900030461A990BF0BBFF044611901C98308415
:101AA00030461A9905F04EF92989006822460DF052
:101AB000C7FE28890B2825D12B48844201D08742B4
:101AC00020D130460CF00CF9C10F081844103046F4
:101AD0000BF038FAC10F0818234A119940109142AF
:101AE00006D1611C431C994200DA00E019461191AD
:101AF000974207D1611C421C914201DA601C00E050
:101B0000401C12901948FFF797FE04002AD0119844
:101B1000E0601298266020612889A0801A98A06051
:101B2000684605F06FFC1248019012480290124876
:101B3000039000210094FF20089109910A902888C1
:101B40000B90688810A940420C90E868079088784C
:101B500040084000887028690690684605F0A8FC97
:101B60001DB0F0BDFEE70000FF7F00004011002027
:101B7000BD180108A51A0108091A010810B5142199
:101B80000148FFF751FE10BD40110020F7B50025B8
:101B900082B006462C46FCE0E100F268081D1058B1
:101BA00083017DD480B2039B07469F430FD000235F
:101BB000049FB8430DD00020834271D057586A4625
:101BC000102138460DF0A0FC00287ED103E001234F
:101BD000EEE70120F0E76A46112138460DF094FC4B
:101BE000002872D16A46122138460DF08DFC00287B
:101BF0006BD16A46132138460DF086FC002864D16B
:101C00006A46152138460DF07FFC00285DD16A46F2
:101C1000142138460DF078FC002856D16A460A2176
:101C200038460DF071FC00284FD16A466B213846CA
:101C30000DF06AFC002848D16A466C2138460DF048
:101C400063FC002841D16A46012138460DF05CFC56
:101C500000283AD16A46042138460DF055FC002888
:101C600033D16A46022138460DF04EFC00282CD1B3
:101C70006A46032138460DF047FC002825D16A4604
:101C8000052138460DF040FC00281ED16A46062189
:101C900038460DF039FC002817D16A46322101E0A0
:101CA00076E012E038460DF02FFC00280DD16A4690
:101CB0006E2138460DF028FC002806D16A466D21B9
:101CC00038460DF021FC002802D0032005B0F0BDFD
:101CD0006A46692138460DF017FC002853D16A4640
:101CE0006A2138460DF010FC00284CD16A466E215E
:101CF00038460DF009FC002845D16A466D2138466A
:101D00000DF002FC00283ED16A46372138460DF01E
:101D1000FBFB002837D16A46382138460DF0F4FB2A
:101D2000002830D16A46352138460DF0EDFB0028F9
:101D300029D16A46402138460DF0E6FB002822D121
:101D40006A46452138460DF0DFFB00281BD16A4664
:101D5000412138460DF0D8FB002814D16A464221B3
:101D600038460DF0D1FB00280DD16A464321384694
:101D70000DF0CAFB002806D16A46492138460DF00D
:101D8000C3FB002801D0022502E0002D00D101256F
:101D9000641C708C8005800EA04200D9FCE62846A9
:101DA00094E7000001484068704700002C000020C4
:101DB0007047C005C00E072800D9072070470000F3
:101DC0000C49884201D11F2070470028FCD071289F
:101DD00001D2094909E009497138096880B200292E
:101DE00005D0074A5268904201D2085C7047002033
:101DF00070470000FFFF0000901F0108AC000020AA
:101E0000B000002010B518210348FFF70DFD03496D
:101E10000120087010BD0000EC1000206C000020B4
:101E2000FFB50A4D0E466A6881B01C460746194642
:101E300090473060002804D020686A68C0190021EB
:101E400090470399086005B0F0BD000080000020B5
:101E5000FFB587B00446109D00201F46002D00D01E
:101E60002880002C0CD02178002909D0089900295D
:101E700006D0119900264907890F14D0002003E0ED
:101E800000200BB0F0BD401C215C0A2904D00D29B4
:101E900002D00029F7D100E0401C002DF1D0002134
:101EA000C9432980EDE71199890700D5274F002004
:101EB00069460875049028E00020069060460028D6
:101EC00031D00021119805AA06AB0090019302922F
:101ED0000391604620183B46099A08990DF086FF49
:101EE00006997A1A711817B20EB2002813D0049905
:101EF0000918049120780A280DD00D280BD0605CB9
:101F00000A2812D00D2810D008468446205C0028EC
:101F100001D0002FD0DC0498002809D0002D00D07B
:101F20002E800498ADE70121CCE7481C0490F2E72D
:101F3000074A04A95268204690470146002DF0D078
:101F40000022089808F0D1FA06B2E9E7FF1F000066
:101F50008000002000230278232902D0012A0ED01D
:101F600010E0002A05D00021012A04D0022A04D062
:101F700008E0012101E0017004E0017001E0202986
:101F800002D00123184670470221F6E7FFB581B061
:101F900014460E4613E004986508684387190A9AA8
:101FA000394601989047002806DDE007C0172C1A33
:101FB00004983E18641E02E0002805DA2C46002C26
:101FC000E9D1002005B0F0BD3846FBE7024610B568
:101FD0000020002A0DD04B1E194200D0FEE75118F8
:101FE000491E012299431203914202D20C2901D9C0
:101FF000084610BD0C2010BD40184A1E401E9043DC
:10200000114200D0FEE77047F7B582B002980F4644
:10201000407A4007400F022817D01046019097429F
:1020200000DD3A465000C01C85082C492C4B8C68BA
:102030001868AD001646201A103549682A188A42D9
:1020400005D260684000400825E00846E6E7234CDA
:102050008D4211D916E00020C0430090002269464D
:10206000204804F0E0FE002269461F4804F0DBFE31
:102070001B48A1680068081A616840198842EAD8BC
:10208000A468DEE7284609F041FF04001AD00121C8
:102090006068C907084360603A460199029800F0F9
:1020A00054FF206060680121800F80078907401C71
:1020B00088436060A6810199E18104D520461030F3
:1020C000A06007E0FEE70549886802461032401923
:1020D000A2608860204605B0F0BD0000C40000206A
:1020E000A800002075680008856E000810B5074C30
:1020F000012020700648FFF786FB0028A06802D068
:102100000DF034FD10BD0DF025FD10BDB800002010
:102110001C11002070B5044640308178A36B8A07FB
:1021200007D40288002A07D01D4DAA421CD0521E97
:1021300002800288002A17D1002B01D08A0713D50C
:1021400021461848FFF7F5FBFFF7D0FFE1680029AB
:1021500001D0204688472169002901D020468847C0
:10216000204609F05BFF70BDE26B52422263002BF8
:10217000F9D08A0702D4626B524222638A07D217CF
:102180005200921C9207FD25920F29400A4382704B
:10219000A16A206A2162A062E06AE362A06370BD66
:1021A000FFFF00001C110020F8B5324D68680DF0EB
:1021B000E8FB074668780121484068704BE0002042
:1021C000264628704036B0784107CA0F69788A429F
:1021D00045D0FB22104089000843B070216BCA191A
:1021E000030719D4002917DC002A15DBC0070AD120
:1021F0006169002907D020468847216A09182162B1
:10220000A16A0818A062A168002901D02046884769
:10221000B07808210843B070206BC019206317D430
:10222000E16A884200DD2163E16920468847626AED
:1022300001468A4205D061626268002A01D02068A6
:102240009047216BE06A814202DB2046FFF762FF84
:102250002878002803D00848FFF7D5FA03E0214684
:102260000548FFF7D4FA0400A9D10DF091FB68608E
:10227000F8BD0000B80000201C11002070B5044615
:1022800040680D46002801D0FFF7F8FF2268002AB9
:1022900002D029462046904770BDFFB599B02399DA
:1022A0002298149000200A90299816461391042829
:1022B00012D0052812D0062813D014287DD101276A
:1022C00002251C980024704340000E901A98401E6E
:1022D0000590701E0D9055E10027F1E701270325B9
:1022E000EFE701270225FFF75DFD0068806B0A908C
:1022F000E7E724986043011214980A182598604370
:102300000112139809180B1210129C46002807DBC3
:102310001A9B984204DA6346002B01DBB44503DBC9
:102320002898002101552BE1D2B2CBB2802A06DADF
:102330000021C94307917F21891A490004E0012146
:1023400007915100FF3901390891802B06DA0021ED
:10235000C94302917F21C91A490004E00121029179
:102360005900FF3901390B911C9B61465943069175
:10237000199A0918694389188E460799411873D428
:10238000059A914270DC029A62440F92002A6BDB3C
:102390000D9B9A42F6DC079A1C9B6A437244169284
:1023A000029A5A436A43724473461192002F6ED0C8
:1023B000299A052A06D0142A00E0E7E00AD0062A66
:1023C00053D061E011989A78807884461698807886
:1023D000009010E0199B0E9AD3181818069A84469C
:1023E000125C0698C318585C00901C9B0F996046BD
:1023F0005943085C8446604694450BD001460B98CF
:1024000041430346FF200130C31A5343C818000458
:10241000000E84460098904209D00899FF23484353
:102420000133591A514340180004000E00900099DE
:102430006046401828994008085543D070460178F6
:1024400040780002091868460182119801784078A6
:1024500000020918684681811698017840780002C8
:1024600009186846818020E047E068461988008D99
:10247000814207D011990988814203D016990988B1
:10248000814201D1002079E0FF208446CEE71988FF
:1024900068460182169801886846818011980188F3
:1024A000684681812899FF2008556946088A8989EC
:1024B000884208D169468988884204D127996200F8
:1024C000511808805CE00B980499C2B2039805F09B
:1024D0003FFA039008980499C2B2019805F038FABF
:1024E0007F220190039905F033FA0090279861004C
:1024F000081869460988018042E0724671465278A0
:10250000097812028918279A89B26300D152299A50
:10251000052A04D0062A05D0142A09D10AE07146FA
:1025200089780DE06A46128D914201D1002107E0C1
:10253000FF2105E0199A06998A180E990918515C2D
:10254000002802D1079A002A05DB059A904204D19F
:102550000798002801DD08980CE06046002802D1A9
:102560000298002805DB0D9A94458BD1029800282B
:1025700088DD0B98FF22101A48430012289908554D
:10258000641C24B22698844200DAB2E61DB0F0BD85
:1025900010B50446406882080AD049688908890055
:1025A000091D08186060204600F045F8204610BD5F
:1025B000FEE74068103180088000884201D3012086
:1025C000704700207047F0B50546486885B00C4656
:1025D0008008800001AA69460EF024F9009F019846
:1025E0000290F80141190298800008180390C06A0F
:1025F00000280DD0002C0CD0E560A06026460836DF
:10260000C46030460421FFF7F7FC864202D0FEE7A3
:10261000FEE7FEE70398C462012002462969BA403A
:1026200011432961B9004919029B4A699840024344
:102630004A6105B0F0BD10B5044600F08AF80460A8
:1026400010BDF0B50646002085B00D460090074647
:102650000190002945D06846039001A80C460290DD
:10266000802907D308460FF020F9411F0120884038
:10267000401E24182046029A03990EF0D3F8009CBD
:10268000062C2EDAA00000218019019AC943406966
:102690000B46934018400DD1641C3069A14008409E
:1026A0001FD00FF0F8F804468100009088194069A7
:1026B000002810D00FF0EFF80346E20101909119C5
:1026C00080000818C76A002F0BD078688008800047
:1026D000A84201D2FEE7FEE739463046009A0EF0E6
:1026E000B6FC384605B0F0BD10B50446FFF7A3FFB1
:1026F0004168022211434160606801210843606023
:1027000010BD10B5044600F024F841680222914340
:102710004160606840084000606010BD70B50646CA
:102720000D46084600F015F8040010D02079C007C7
:102730000BD0686880080BD02146304600F03EF888
:1027400021462846FFF724FF0546284670BDFEE7D0
:10275000FEE701464268083190088000001F081813
:10276000910800D1FEE7704770B5064600200C4680
:10277000002920D0002A1FD020791546C0071CD080
:1027800011462046FFF715FF00280FD029462046A6
:1027900000F025F805462046FFF74DFF6868022146
:1027A0000843686029463046FFF70DFF2046FFF7D3
:1027B000A8FF2046083070BDFEE7FEE77CB5054661
:1027C00048680C468008800001AA69460EF02AF885
:1027D00021462846019B009A0EF039FC7CBDF8B5D5
:1027E0000D46014604460831281F0E18606837461A
:1027F00080088000401B001F0837009038460421E5
:10280000FFF7FAFB874200D0FEE760688108009876
:1028100089004019001D814200D0FEE730790099FF
:102820008007800F08437060800880000C2800D269
:10283000FEE720798007800F284360603046FFF76D
:1028400053FF3046F8BD0000F1B584B000221146B8
:1028500004980CF067FB002104980BF03EF8044646
:10286000002104980BF0C7F8001901B20291002171
:1028700004980BF09CF8001900B2019004980AF03B
:10288000D1FF0299294C41180198081805B2049803
:102890000AF0B6FA074600262EE00498B1008068D8
:1028A00000684058224900900BF027FA002822D1F6
:1028B00000980BF037FC00282BD1002100980AF07B
:1028C000D5FF002825D0012823D0022821D00328B5
:1028D0001FD0002100980BF04AF900280BD1009876
:1028E000418BC08A081A401C029900B24018A042CD
:1028F00000DB044624B2761CBE42CED30B48844291
:1029000004D00198201800B2A84200DC284605B087
:10291000F0BD00981A21415E04981622825E881A42
:10292000411CA142E6DB0C46E4E7000001E0FFFFAA
:1029300001000400F1B584B00022114604980CF0A7
:10294000DDFA002104980AF0C8FF0446002104982B
:102950000BF045F8001900B20190002104980BF02B
:1029600032F8001901B2009104980AF069FF009949
:10297000524C41180198081805B204980AF040FA20
:102980000746002104980AF07CFF012801D00026A8
:1029900078E0002631E00498B10080680068405873
:1029A000474902900BF0A9F9002825D102980BF0B5
:1029B000B9FB002828D1002102980AF057FF00280F
:1029C00022D0032820D006281ED008281CD00021A1
:1029D00002980BF0C6F800280ED10298143002902D
:1029E00004F0FFFD01994018A04204DB029804F0B6
:1029F000F8FD0199441824B2761CBE42CBD32F486F
:102A000084424CD0009843E004981821415E02981B
:102A10001422825E881A411CA142ECDB0C46EAE7D4
:102A20000498B100806800684058254902900BF076
:102A300064F9002825D102980BF074FB002831D1ED
:102A4000002102980AF012FF00282BD0012829D07B
:102A5000042827D0072825D0002102980BF087F8FA
:102A600000280ED102981430029004F0BAFD0099AB
:102A70004018A04204DB029804F0B3FD009944180A
:102A800024B2761CBE42CBD30C48844207D00198B6
:102A90000A49201800B2884201D0A84200DC28462A
:102AA00005B0F0BD02981821415E04981422825EA0
:102AB000881A411CA142E3DB0C46E1E701E0FFFF7D
:102AC000010004001CB50B8804891C196B461C808E
:102AD0004B8844891C196B465C808B8804891C19BF
:102AE0006B469C80C9884389C9186B46D980436965
:102AF000694698471CBD0000F3B593B0054614988D
:102B000000283ED028832868002801D009F086FAE2
:102B1000149806214843801D09F0F8F92860002820
:102B200025D06860149901224900891C4118E96088
:102B300014998C00211D4118A9601499012917D0FE
:102B4000C800083009F010FA064600200F9020B2A5
:102B50006A4600219081D1810122131A6A46A71981
:102B6000138380100C463F1D07910B90B9E0FEE7E0
:102B7000B4210170E86800210180E8684280A868FB
:102B8000018015B0F0BD0020059068461821415E17
:102B9000002906DCC0894000C01C09186846018372
:102BA00009E0C38980891A1A5200521D51186A46D9
:102BB0001183401E90816946C889401CC88103A8C2
:102BC00000F000F9002810D068460C21415E0598FD
:102BD0008A1080000BAB1A508907890F07AA115081
:102BE0000598401C05900428CFDB059804287DD16A
:102BF0000B990E98814212D1600031520F993952CF
:102C00000899079842180A99099840186968101895
:102C10000855696800010855641C24B25EE0084646
:102C20000C9988421FD00146600031520F9A3A52E7
:102C3000696807980855696800010855641C0B9B72
:102C400021B248005B1E33523A52099A0898821802
:102C50000A98001D10186A6850546A6800015054A0
:102C6000491C0CB23AE00D998842014618D0600028
:102C700031520F993952089A079880186A6810558E
:102C80006A6800011055641C0B9B20B242005B1E59
:102C9000B352B9520A9A0999891808316A6817E03B
:102CA000600031520F993952089A07988018099A92
:102CB00080186A6810556A6800011055641C0B9AE8
:102CC00020B24300521EF252F9520A996A680C313E
:102CD00011546A6809011154401C04B20F98401C39
:102CE0000F9003A800F06EF8002800E001E000D08B
:102CF00049E7334914983E23484361008A19403A12
:102D00008446D35E8012834205D1CA19403A3E23DD
:102D1000D35E83421BD0820263469A1A01235B0270
:102D20009A4203DC52435200121407E001239B0233
:102D30009A1A5243520012140F239A1A7052785260
:102D400068681101025568680155641C24B2A01E10
:102D50000BE04300FA5A61007252F25A7A526A68E2
:102D6000115C1155641C24B2401E0028F1DA0020C9
:102D7000EA68844610801DE062465200E968964683
:102D800088524100AB68715A995209E0AB687246AB
:102D90009A5A715E8A4200DA114672469952401C74
:102DA00041007B5E6246634501D1A042EEDB511CCF
:102DB00009B28C46A042DFDB304609F01DF9E0E69F
:102DC000D302000002210022415E825E914201DCBA
:102DD000012070470020704717B581B0022A68466D
:102DE00002D8008904B010BD01898088CB0AC40ACA
:102DF00040051B19400D1F2B00D31F23DB061B0CA6
:102E000018436B4698804B0544059B0EA40E1B1976
:102E10003F246401A0433F2B00D33F239B065B0D5F
:102E200018436B469880C306C906C90EDB0E4009DD
:102E3000C91840011F2900D31F21C906C90E084324
:102E400069468880FF2A07D00299019804F062FD44
:102E5000009068460088C5E78888C3E717B581B049
:102E6000022A03D86846008904B010BD69468888E4
:102E70000B89C40AD90A4C4361094005C902400DB7
:102E80000143C806DC06C00EE40E60434909400950
:102E90004901084341055B05890E9B0E5943890989
:102EA0004B013F2149018843034369468B80FF2A38
:102EB00007D00299019804F02DFD00906846008823
:102EC000D2E78888D0E717B581B0022A684602D8D1
:102ED000008904B010BD01898088CB0AC40A40056E
:102EE0001B1B400D002B00DC0023DB061B0C1843D2
:102EF0006B4698804B0544059B0EA40E1B1B3F247C
:102F00006401A043002B00DC00239B065B0D1843EB
:102F10006B469880C306C906C90EDB0E4009C91A64
:102F20004001002900DC0021C906C90E084369469A
:102F30008880FF2A07D00299019804F0EBFC0090EA
:102F400068460088C5E78888C3E752104A40504069
:102F50007047FFB589B004460A98129E0090700031
:102F60001499169F159D00B20290042923D00629BA
:102F700021D0052968D0142964D10220205E0021C7
:102F80000246615E724352185300009A9A180092EA
:102F9000029A0492E288101A401C00B20390A088A2
:102FA000401A401C00B2019000200290019840009D
:102FB000069002988CE0204604F005FB0146049040
:102FC000384609F04AF90220205E00210246615E7F
:102FD000724352185300009A06469A180092A2882B
:102FE0000395511A491C09B24900069101910299B1
:102FF00005910EE0019A0099039809F04BF80599A4
:10300000009840180090039906984018761C36B234
:1030100003900620205EB042ECDA1498062811D105
:1030200000213F22520168460280019282880846B0
:1030300005E04300EB5A934200D13954401C049BF5
:103040009842F6D30DB0F0BD0221615E0022084621
:10305000A25E704380184300C31800981818A38814
:103060009A1A521C12B2B31A5E009B191BB201933A
:10307000E388591A491C09B28C46002351008E4638
:1030800014E000210AE084787C5446780478360203
:10309000A4194E00491CAC5309B2C01C9142F2DB8A
:1030A0000199BF1840185B1C75441BB26345E8DBEF
:1030B000C8E72846069A009908F0ECFF069804999C
:1030C00045190098401800900298401C00B20290E8
:1030D00003998842EDDB0B990C9A490051430A98F9
:1030E000002208180221615EA25E714389180D1842
:1030F000002409E029463846019A08F0CBFF0198E0
:10310000AD193F18641C24B203988442F2DB99E79E
:10311000F0B50746C87A8DB015460E46022802D88B
:1031200001200DB0F0BD18463269B168FEF7A0FA73
:10313000040008D0207DC006C00E07F06AFD0028FC
:1031400003D0062015E00020EBE7207DC006C00E6E
:103150000E2807D014280CD007F04AFD002807D00D
:10316000052006E00E2005903088002807D102E0F7
:103170000420059007E07188C81FF93803D00520A6
:1031800005900020A061226A002A04D02946384612
:103190000EF05BFBB7E0A069002849D0294602A8E1
:1031A00004F0E7F90020305E8446002803D17188DE
:1031B000C81FF93826D0A88829886A88401A401C78
:1031C00001B2E888331D801A401C02B27088019356
:1031D0000090634602A8FEF791F9684600892988A5
:1031E00041186846018140896988411868464181D3
:1031F00080892988411868468181C0896988411879
:103200006846C18102AA06A8B968FDF724FF002814
:1032100079D0B868019006A8B860059800902A4651
:1032200031463846A36904F063FD0198B8606AE04E
:103230002A4606A8B968FDF70EFF002863D0694644
:10324000888B098B401A401C00B241000290401844
:1032500008F08AFE0890B868099006A903A804F04F
:1032600088F9012103A804F0EFF969461820085EE7
:103270000021695E401A0A9069461A20085E022100
:10328000695E0546411A019133E003AA0BA809992A
:10329000FDF7E1FE00282BD0089800900198029BD2
:1032A00002B20A9801B2204608F094F801280BD027
:1032B000204607F0DEFF089808F09EFE204607F043
:1032C000D8FF0998B8603EE70BA8B8600598009051
:1032D00003AA31463846089B04F00AFD6846C189B6
:1032E000491CC181418A491C41820198401C0190BE
:1032F0006D1C69461E20085EA842C6DA0998B860AF
:10330000089808F079FE204607F0B3FF08E7F7B504
:10331000C878A0B00C4602287DD91146684604F052
:1033200043F92020205E012823DD214620318878C2
:10333000FD281ED3208800281BD0CA7868461307B2
:103340000088DB0FC3186846038040885207D20FFD
:10335000821868464280CA788088D206D20F821AC4
:1033600068468280C288C8788007C00F111A6846F4
:10337000C1802098694682680BA8FDF76CFE002882
:1033800049D0E07B4607760F19D0E08869468886E9
:103390006846808E6189884200D10026684605F023
:1033A000FFF907461C2102A8FCF7BBFFA17808A87B
:1033B00041706846818E0182002F03D007E060686B
:1033C0000D90E5E72088002801D1002E54D0E07848
:1033D000FD2800D3FF201190684681880088081AD4
:1033E000401C01B268461591C1884088081A401CEB
:1033F00000B215991290814200DA08460025655FF7
:103400004010854200DB05466846018E808D081A13
:10341000401C00B200E038E010900020C04318903B
:1034200000200D90002D01DC002F0ED0109808F028
:103430009BFD0D9000232A4669461AA805F03EFC24
:1034400000211AA804F0CCFF18906846818D818471
:10345000018E01850D98059009A802900790FF2123
:1034600008A80170A01D129A159907F06BFA0400C4
:1034700019D0022E0BD016E068460290E07808A919
:10348000087002A9209805F0D7FE23B0F0BD684669
:103490002C21415EA2684800111868460022825E15
:1034A0005000081A0390002F7DD068462E25455FF6
:1034B00028E02FB2CF844F85109A11990D9808F00B
:1034C00074FE68462C21415E3A46109B0D9805F02B
:1034D0002FF9014668460176012902D1022069468A
:1034E0000876012E09D168460222825EA168A81AD8
:1034F0004000081801886846018202A9209805F05A
:103500009BFE6D1C69463220085EA842D1DABFE0FE
:1035100040882E21C01900B217906846C088C01B91
:1035200000B216906846415E1798814205DD6846F4
:103530003221415E1698814248DB109A11990D980C
:1035400008F033FE6A462421515E109B179A0D98AD
:1035500005F0EEF86A461076012801D102201076B7
:103560002E21515E1798814213DCD08417981146A2
:103570005085012E09D102228A5E1799A068891A06
:103580004900401800886946088202A9209805F081
:1035900053FE68463221415E1698814216DB694629
:1035A000C884169800E012E04885012E0AD16846CA
:1035B0000222825E1698A168801A400008180188CD
:1035C0006846018202A9209805F036FE7F1CAF42B2
:1035D00068469DDB018810A881816846818810A813
:1035E000018268464088411910A8C1816846C08898
:1035F000411B10A8418213A805F0D2F81690304361
:103600000CD008A8119901700121684601760621A5
:10361000415E4F1B0221415E4D1937E068464088EC
:1036200041196846C184C088411B6846418508A885
:10363000119901700020059002A9209805F0FCFD69
:1036400026E0169800280ED0109A11990D9808F0CF
:10365000ACFD6A462C21515E2AB2109B0D9805F0F4
:1036600067F86A4610766846C5844585012E08D1FC
:1036700002460220105EA168281A4000081800883F
:10368000108202A9209805F0D7FD6D1CBD42D8DD3F
:103690000D98002801D008F0AFFC1898401C05D008
:1036A000189805F0AFFB1AA805F060F8002C00D1BF
:1036B000EBE6204607F03EF9E7E60000F0B50646E7
:1036C000086991B015460C4600287AD0A07E0228E1
:1036D00077D929460FA8B268FDF7BDFC002870D045
:1036E000B0680E900FA8B060206907F084FE022831
:1036F00006D006A9206907F0DDFD012848D0C3E007
:10370000002763480190009702973B460BA8626927
:1037100021690CF00BFC284603F06FFF01466A4656
:103720002C20105ECB0F2A88591849105118C20F4F
:1037300012185210891A6A4608181186401E90867F
:10374000284603F03AFF01466A462E20105ECB0F52
:103750006A88591849105118C20F12185210891A44
:103760006A4608185186401ED08603A804F088FDDA
:1037700060690390208B6A461083A07E08AA90712E
:1037800000970CAA03A93046236904F0D3FA7BE022
:10379000684604F0B5FAA17868460173218B01816F
:1037A000E17E8172A17EC172207F00280AD06988E3
:1037B0006846C1830698400D401E0918684641843A
:1037C0005BE063E0284603F018FFC20F2988101859
:1037D000401008180699C902890D411A684681836C
:1037E000284603F0EAFEC20F698810184010081836
:1037F00006998A0D821A6846C283838BC802400DDF
:10380000401E1B1868460384480D401E1118684668
:10381000418407AA69463046236904F041FA33E03F
:103820002888694688830699C902490D491E4018AF
:103830006946088411E007AA69463046236904F006
:103840002FFA06996846808BC902490D42186846CE
:103850008283008C41186846018469461C20085EFA
:103860000421695E8842E6DD6A460698D18B400DE8
:103870000918D183518C0818508469461E20085EAF
:103880000621695E8842CBDD0E98B06011B0F0BDB4
:10389000FF1F0000F7B50E462036B07886B01746F9
:1038A0000C46022863D9208C002860D0F07881066D
:1038B000C90E5CD0C0075AD1B88839887A88401AB6
:1038C000401C01B2F8880025801A401C00B2655FD8
:1038D000814200DA08464110A94200DA4510394613
:1038E00004A803F061FE68461022825EF078410869
:1038F00048072048205E01D44019404210186A460B
:103900001082142308071B48D35E205E01D440199F
:103910004042181A9082F07812214008800715481A
:10392000515E205E01D44019404208185082F07860
:1039300016214008C0070F48515E205E01D1401992
:103940004042081AD082208C281A00B2002800DADF
:103950000020A278B17803920291E18B6A469180AF
:1039600000902B4604AA3946069800F005F809B0E5
:10397000F0BD000020000000FFB5A9B0349F1D4637
:1039800016460C46FF2F00D3FF27084604F008FF19
:1039900014903299284308437DD0299821468268A3
:1039A0000AA8FDF758FB00287CD06846818D008D61
:1039B000081A401C00B200901C2103A808F023FC48
:1039C000009808F0D1FA06900020C0431190002D15
:1039D0000ADD00232A4621461CA805F06FF90021C4
:1039E0001CA804F0FDFC11900123314622A8329A54
:1039F00005F064F9002122A804F0F2FC129001A85D
:103A00000390089030A881896846818208A80771D0
:103A1000359941710020205E1A900021715E401995
:103A20008E46704500DC084600B2694608860F9055
:103A30000420205E17900421715E401B884200DB49
:103A4000084600B26A4690860E900220205E1690CC
:103A500042190220305E824200DC024617B26A46FA
:103A600057860622A25E19920623F35E521B9C46DD
:103A7000624500DB1A4612B26B46DA860D920F9B46
:103A80000E9AD21A521C13B2169A82420CDC0120F2
:103A90000BE000E006E0009732462146339B299870
:103AA00000F0ADF92DB0F0BD0020109019986045E0
:103AB00001DB012000E0002016901498002840D07F
:103AC0006846018D8180818D01812A24045F20E078
:103AD0001098002801D1A7421ADC1698002802D1BC
:103AE0000D98A0421ADB25B2CD804D810099069831
:103AF00008F0B3FB6B462821595E2A46009B0698C6
:103B000004F016FE6B46187703A9299805F094FB7C
:103B1000641C69462E20085EA042D9DA22A804F06F
:103B200025FE129805F06EF91198401C05D01CA8CE
:103B300004F01CFE119805F065F9069808F05CFA8F
:103B4000B0E71A98704501DC012000E000201490D5
:103B50001798884201DB012100E000210120159027
:103B6000149813910840109908401699084203D000
:103B7000322B01DA0020159001206946087715994B
:103B8000109808420DD069460F9888800E980881D9
:103B90006088C8807088401E488103A9299805F074
:103BA0004BFB1599169808420DD068460F998180F5
:103BB0000E990181F188491CC180E188418103A9E6
:103BC000299805F039FB149800280CD02188684604
:103BD00081803188491E0181C7800D99418103A9E7
:103BE000299805F029FB139800280CD0B188684665
:103BF000491C8180A1880181C7800D99418103A959
:103C0000299805F019FB1598002819D06A46282133
:103C1000515E91802C20105E0F9A521E904201DB63
:103C20000F98401E6A461081401A401C06B2002EB2
:103C30007EDD10991498084364D02A24145F5FE055
:103C40006846018D8180818D018102200221305ED4
:103C5000615E401AA84200DB054628B2002510909C
:103C600033E060886946401906B2E088401B07B21D
:103C70002A20085EB04203DD2E20085EB84223DB16
:103C80000099069808F0E9FA68460421415E324638
:103C9000009B069804F04CFD0146684601772A21F6
:103CA000415EB14205DCC680468103A9299805F032
:103CB000C3FA69462E20085EB84205DBCF804F81EB
:103CC00003A9299805F0B8FA6D1C10988542C8DB45
:103CD0008EE025B26B46DD805D813146069808F0A6
:103CE000BCFA6B460421595E33462A46069804F016
:103CF0001FFD6B46187703A9299805F09DFA641CEF
:103D0000A742E6DC1699149808431ED00D9C16E0D5
:103D100025B2CD804D813146069808F09EFA6A465C
:103D20000421515E33462A46069804F001FD00E066
:103D30000BE06A46107703A9299805F07DFA6946D9
:103D40002E20085E641CA042E2DA69462820085E44
:103D50000E99491C884201DC0E98401C6A469080EE
:103D6000918D1181081A401C05B2002D40DD10997B
:103D7000139808431BD02A24145F16E026B26B4622
:103D8000DE805E812946069808F067FA6B460421BA
:103D9000595E2B463246069804F0CAFC6B461877EB
:103DA00003A9299805F048FA641CA742E6DC169995
:103DB000139808431CD00D9C14E026B2CE804E818F
:103DC0002946069808F049FA6B460421595E2B46AD
:103DD0003246069804F0ACFC6B46187703A9299884
:103DE00005F02AFA69462E20085E641CA042E4DA37
:103DF00022A804F0BBFC129805F004F897E6FFB582
:103E00008FB00C4615461C216846189E08F0FBF939
:103E100007A8009010A80189684601810676022053
:103E20000221205E695E884201DC012700E0002754
:103E300006200621205E695E884201DB012600E043
:103E4000002600200021205E695E884201DC0121FD
:103E500000E000210C9104210422615EAA5E9142DF
:103E600001DB012100E000210B9169468883A088D5
:103E700008846088C8836888401E4884002F02D068
:103E80000F9805F0D9F9E8886946401CC883E08896
:103E90004884002E02D00F9805F0CEF9208869469C
:103EA00088832888401E0884002F02D00220285EC4
:103EB00001E00220205EC883002E02D00620285E8A
:103EC00001E00620205E48840C98002802D00F985C
:103ED00005F0B2F9A8886946401C8883A088088448
:103EE0000B98002802D00F9805F0A6F913B0F0BD8A
:103EF000F8B5324D0746686803F066FE0446386838
:103F0000C66B716B002901D0304688476868002174
:103F100000680222415E825EE0685143814201D125
:103F2000012000E00020216800290ED061680029EE
:103F30000BD0002806D008E068680068816A002974
:103F400000D0884720690028F6D1012020616968E7
:103F50000968C9688A69D20702D08969890700D4CB
:103F6000002060616069002801D0012500E0002583
:103F70003868416900290ED001698A06920F06D07F
:103F8000490704D53168706800F01AF803E0326818
:103F90007168FEF797FD206800280BD06168002942
:103FA00008D03A68127CAA43D20703D1A2688242A1
:103FB00001D1A160F8BDA060F8BD00002C00002078
:103FC000F3B504468C4893B04068056829698A07B0
:103FD00001D54A073BD48906890F02292DD0012932
:103FE00001D0032933D100210E9103F0EDFD0F9094
:103FF0000027A088E75F0226C01B401C00B200908B
:10400000E088A65F801B401C01B20391052080025E
:104010000099FCF7D9F90399884200DB0846059618
:104020000C90287C8006800F012812D067800098B1
:10403000401E3818E0800020D2E021462846149A1D
:1040400000F0E6F821462846149AFEF73BFD15B02D
:10405000F0BD6888C01B401EE0800099401A401CDB
:104060006080E8E708460299401A0C99884200DD12
:10407000084600B201900F990120086102980028BB
:1040800020D10099039888421CDB0191287C80068E
:10409000800F03280FD00020149A00F0EDF8287C40
:1040A0008006800F012808D029880598081A401E2C
:1040B000A080009957E00120EEE705982080009944
:1040C00005986AE00E98002804D10520C00207F088
:1040D0004BFF0E90287C8006800F03281DD0002007
:1040E0001190009809901498019986460E981290A4
:1040F00009984843401E0B900998401E48430D9074
:1041000000208446884221DA0D9A1018119A002A5C
:1041100001D00B9A101A002611E00120E0E7129B53
:104120004700FF187246931C9E4613883B80119BE4
:10413000002B01D0401800E0401A761C36B2099AD4
:104140009642ECDB6046401C00B2DAE7287C800631
:10415000800F01281CD029880598091A0298081A8E
:10416000401EA0800199401A401C208002990198AD
:104170000E180398864214DB0F988069C00710D090
:104180000F98806980070CD50F99012048610BE0DA
:10419000059902980818208001994018401EA080B7
:1041A000E4E70F98002141610E98002805D00246EF
:1041B00021462846FEF786FC06E0149AF8E7A96A2D
:1041C000002901D0284688470F9800690028F6D1B9
:1041D000019900984843410014980818149030B28F
:1041E00003990290884200DA3CE70E98002800D13B
:1041F0002DE707F001FF2AE72C00002030B50488E6
:104200000D88058010880880188810801C8030BDBB
:10421000F8B58B880C884D881B1BCC885B1C641BF5
:10422000641C1BB224B2634300245B1E0DE05D00DE
:10423000AD182F886E4637806600B618BC463788A2
:104240002F8067465B1E3780641CA342EFD84288EC
:104250004C88CB88121B521ECA804288D21A521E2A
:104260004A8002880C888B88121B521E8A80008824
:10427000C01A401E0880F8BDF7B50C46C80F0026CE
:10428000001982B040101746019039E0601CC10F40
:1042900000250818401000902DE0A01B401E01B220
:1042A000601B401E029A00B2002A0BD02A466243CD
:1042B0005218614309185200D3194900CA196043C2
:1042C00080190CE00246624392195200D3190A4643
:1042D000624310184000C21928466043401840004D
:1042E000C1193046604340194000C019FFF786FFEE
:1042F0006D1C00982DB2A842CFDC761C019836B216
:10430000B042C3DC05B0F0BDFFB5987B9FB0040799
:104310002098240F827E032C18D0012C1DD0022C53
:1043200021D0042C13D0082C7ED1FF209D4D411CA0
:104330001490FD2A2AD29C480078904203D19A48D2
:104340004068A0421ED00020984F19E00424954DEB
:10435000F020103D10211490EBE7924D8020163D87
:1043600002211490E5E78F4DC020143D04211490E4
:10437000DFE72E5CFF2E1AD05643360A3E54401C0F
:104380008842F6D38848894D02704460D8880C90E2
:1043900018891290219900228A5E1F990C988968C9
:1043A0000023CB5E60439A4203DB002302E0164603
:1043B000E4E79B1A0E930C9BD6180423CB5E9E4217
:1043C00001DC0C9A01E09A1A521C1092219B0222E5
:1043D0009A5E0223CB5E9A4201DB002300E09B1A27
:1043E0001593129BD6180623CB5E9E4201DC1299D0
:1043F00001E0991A491C1191159941430E986043A7
:104400000818C20828994707511828917F0F1C21C6
:1044100001A807F0F8FE20988189684681812098DC
:10442000817E6846017700E0BAE02098807F8006B0
:10443000410F68464177FDF7B5FC03F0C9FB129ABE
:104440000C995143814200DC0846169007F08CFD20
:10445000129004902198002601880E980B18684647
:104460000384219801881098401E0A1868468284A7
:10447000219841881598091868464184C184D01A4A
:10448000401C00B2139068460385418582851198CF
:1044900009186846C1850AA804F082F91D9008A889
:1044A000019006900820001B18900E990C98411856
:1044B0001098081A6043199015985CE01498B44657
:1044C000F8400E991AE0289A189B1278DB1B0240DC
:1044D000DA4003D0AB5C129A935502E0129B0022A3
:1044E0009A55189A974202D23F19E04004E0289A60
:1044F0000027521C14982892491C761C109A91424D
:10450000E1DB1D98002812D06B462622202112984C
:104510009A5E595E60441A90139B04F009F96B4649
:104520001875002803D113991A9807F06CFE0E999C
:104530001098401A81191698814204D26946C88C95
:10454000401CC8840CE002206946087501A91F9828
:1045500004F072FE6946C88C401C4884C88400265A
:104560001998289A3818C1084707891815987F0F95
:10457000401C28911590119988429FDB6A462221A0
:104580002620515E105E814207D0401ED08402205A
:10459000107501A91F9804F04FFE129807F02CFD2A
:1045A00023B0F0BD17200108D000002068160020BD
:1045B000FFB50220085E0C46401E4110C007C00F28
:1045C000451800260020965F185E8DB0864200DAFE
:1045D00030466E46B08300200026105E9E5FB042DB
:1045E00000DC30466B46401E18845088401BD88340
:1045F0005088401858840D9807A982680846FCF72F
:104600002AFD002822D0E088002804D0A0880028B5
:1046100001D0012700E00027012507A804F0C0F819
:10462000002801D1002F00D000251C21684607F08A
:10463000EAFD07AE0096218868460181217A01765D
:10464000002D05D001460D9804F0F6FD11B0F0BD27
:104650001C22018C825E881A401C05B26846222109
:10466000415E0B91C18B418400200A90002F08D03D
:1046700006200421205E615E41181046FBF7B2FE61
:104680000A91284607F070FC099005960390684649
:104690001E26865F3DE02946099807F0DEFD6A4642
:1046A0001C21515E2B4632B2099804F041F86A464B
:1046B0001074002F21D000281FD000210A9817E085
:1046C0000422A25E824205DB121A8918801809B200
:1046D00000B209E00623E35E9A18824201DC002062
:1046E00002E0099B00225A54491C401C09B200B246
:1046F000A942E5DB02206946087469460D9804F07A
:104700009BFD6846C18B491CC183418C491C418477
:10471000761C0B988642BEDD099807F06DFC95E784
:10472000FFB502200224105E1C5FC5B0A04269469E
:1047300005DA4886CC8510880886188804E04C86FF
:10474000C885188808861088888508462C21415E0F
:1047500030241291045F32250E1B2E21415E1491EC
:10476000455F4F1B002E01DD304600E07042002FF8
:1047700001DD394600E07942884201DD012000E098
:104780000020139046980221415E13980091002862
:104790000AD0002E01DD314600E07142002F01DD1C
:1047A00038460BE0784209E0002F01DD394600E091
:1047B0007942002E01DD304600E070424001FBF7F7
:1047C00011FEAC49085C009948433F30C0114110CC
:1047D000C207D20F10915118119112998C4200DA30
:1047E0002146091A6A46118112998C4200DD214640
:1047F0000918918114998D4200DA2946091A5181CC
:1048000014998D4200DD29460818D081459802A9E7
:1048100082680846FCF71FFC00287DD01398002111
:1048200000287AD01498002E179016DD109A019166
:10483000801A00B20090A81A129B02B2214618A852
:10484000159304F04FF8119A17980121801800B2BF
:1048500001910090A818159B15E0119A01918018FC
:1048600000B20090A818129B02B2214618A8159316
:1048700004F038F8109A17980121801A00B20191BB
:104880000090159BA81A02B2214623A804F02AF82A
:10489000002118A803F0A4FD1290002123A803F022
:1048A0009FFD11900020C043139010904698407ACD
:1048B000C00625D4A81900B200900321E01B019185
:1048C00003B22A4621462EA804F00CF868462E2290
:1048D000825E0221901900B20191009068462C215D
:1048E000415EC81B03B239A803F0FCFF00212EA8CB
:1048F00003F076FD1390002139A803F071FD1090AC
:10490000684681890089081A401C04B2FDF74AFAFA
:1049100003F05EF9054601E0A9E008E002A802F014
:1049200052FEA8421ED202A802F04DFE1BE01498CF
:10493000169001910090129811991790401803B2A7
:10494000601801B22A4618A803F0CCFF012116987E
:1049500001910090109917982A46401A03B2601AE4
:1049600001B292E728460D9007F0FEFA00906846E3
:104970000E27C75F4189C18100250D99009807F076
:104980006CFC1C2104A807F03EFC02A94698049187
:1049900002886846028346980A26027A08A80272AC
:1049A0000098079009916846865F2DE06A460821C5
:1049B0000098515E4019234632B20F9003F0B8FEC2
:1049C00008AA1070002803D121460F9807F01BFC9D
:1049D0002D190D982919814204D26946C889401CB5
:1049E000C88110E0022008A9087004A9459804F0C5
:1049F00023FC6946C8890025401C4881C8810D995F
:104A0000009807F02AFC761CBE42CFDD69460A22D8
:104A10000E208A5E085E824208D0401EC8810220B5
:104A200008A9087004A9459804F006FC009807F04E
:104A3000E3FA18A803F09AFE23A803F097FE139850
:104A4000401C02D02EA803F091FE1098401C02D00A
:104A500039A803F08BFE129804F0D4F9119804F0F1
:104A6000D1F9139804F0CEF9109804F0CBF949B0BD
:104A7000F0BD000017210108FFB50220085E0C46BA
:104A8000401E4110C007C00F1588401891B0281A69
:104A90006D46A88310884018288402210220515EA8
:104AA000185E814200DA0846E88302200221105E87
:104AB000595E884200DC0846401E6884119807A9A8
:104AC00082680846FCF7C7FA002822D0E088002850
:104AD00004D0A088002801D0012600E0002601278C
:104AE00007A803F05DFE002801D1002E00D00027AA
:104AF0001C21684607F087FB07AD009521886846B2
:104B00000181217A0176002F05D00146119804F029
:104B100093FB15B0F0BD018C808B2227081A401C36
:104B200000B20A906846C75FC18B41840A9807F0BB
:104B30001BFA0021099005950390002E09D006204C
:104B40000421205E615E6A4641181E20105EFBF75C
:104B500049FC68461E250F91455F32E00A99099885
:104B600007F07BFB6A461C21515E2AB20A9B09981A
:104B700003F0DEFD6A461074002E16D0002810D017
:104B80000421615E0F98814201DA00201074062032
:104B90000421205E615E41180F98814201DC0020F3
:104BA0000F900F98401C00B20F901146119804F01E
:104BB00043FB6846C18B491CC183418C491C41841D
:104BC0006D1CBD42CADD099807F016FAA1E7000086
:104BD000F0B593B0054605F09AFB0446284605F06B
:104BE0005EFB07460BA9204608F00FF92546403525
:104BF000287A0026C10600D50126800601D50220AC
:104C000006430021204608F0A6FF8849884204D1C7
:104C1000608C000501D40420064303A803F030FB98
:104C2000A98868464184E988818408A8467203AA55
:104C30000021204609F066F808A8007A002802D171
:104C4000012008A90872E06B0490206C0590784858
:104C5000049981421CD00599814219D00121204636
:104C600055228904009408F0D2FE024601218904ED
:104C70000098FCF7C4FE009068460188418320221A
:104C80002046510308F0C3FE0090684601888183E6
:104C9000287A4007400F022801D0032821D108A814
:104CA000007A022801D003281BD168461E22825EAA
:104CB00060490092029601912023C35E039A0DA8D9
:104CC000616A0BF033F96846018E808D3422081A30
:104CD000401C01B26846825E914202DA012008A9B6
:104CE0000872204630301090287A4007400F032881
:104CF00009D06846418EC08D081A401C012100B2BF
:104D00008902884201DA002010900BA90EA8BA6827
:104D1000FCF7A1F900287DD0287A40070BD1204666
:104D200008F046FA404202B200210BA802F078FCDB
:104D3000618B68464186287A4007400F022813D0CD
:104D4000032811D0109800900BAA03A93846636A73
:104D500002F0F0FFB86811900EA8B860287A4007FA
:104D6000400F03280FD05DE0B86801900EA8B8602E
:104D7000109800900BAA03A93846636A02F0DAFF84
:104D80000198B860E7E768461E22825E29490092D2
:104D9000029601912023C35E039A0DA8616A0BF06D
:104DA000C5F86846018E808D081A401C02B268461C
:104DB0003421415E8A4217DA20221146039805F019
:104DC00094FB410041186846AA88808E1018091883
:104DD00068464184E9888184109800900BAA03A951
:104DE0003846636A02F0A6FF6946488EC98D401AAC
:104DF000401C02B269463620085E824212DAAA8856
:104E00004A840399EA880989101808186946888431
:104E1000109800E008E000900BAA03A93846636AE6
:104E200002F088FF1198B86013B0F0BDD1270000E0
:104E3000FFFF0000FF1F000070B50D46064620353D
:104E4000A87A88B00C46022855D9E08C002852D0A8
:104E5000114604A802F0A8FB208D6946098A401E6D
:104E60000A1A69460A82498A0A1A69464A82898A5E
:104E70000A1869468A82C98A08186946C88204A93C
:104E800006A802F091FB6946098BE08C0A1A694674
:104E90000A83898B081869468883488BE18C401AFD
:104EA00069464883C88BE18C40186946C883888A64
:104EB000098A401A6946CA8A498A401C511A491C03
:104EC0000AB2002100B2615E904200DB104642103F
:104ED0008A4200DA4110E08CA278401803B2A87A26
:104EE00003920290A8886A469080009104AA06A9BD
:104EF0003046FEF741FD08B070BD7CB504468069C0
:104F000061898668A0896D4600290CD0002865D08B
:104F1000814203D12289E3889A427ED302297DD03F
:104F200003297CD0A9E0002822D1E0882189884289
:104F30001ED20620205E0AF033FF04210E22615E9D
:104F4000A25E891A48432168C013498841186846FF
:104F50004180E0885A3000B20AF022FF0421615EED
:104F600048432168C01309884118684681803FE0A2
:104F70002068018829802068A18840884118E9803C
:104F80000620205E0AF00CFF04210E22615EA25E64
:104F9000891A48432168C0134988411868464180EE
:104FA000E0885A3000B20AF0FBFE0421615E32460E
:104FB00048432168C013098841186846818001462A
:104FC000FCF749F8002806D0A0698560626921696C
:104FD000A06903F025FFA08900284ED12068A18890
:104FE0000088411868468180206841886846418071
:104FF0000820205E0AF0D4FE0421615E4843216847
:10500000C013498841186846C18020895A3000B2CF
:105010000AF0C6FE0421615E02E010E00DE00AE045
:105020000E22A25E891A48432168C01309884118DC
:105030006846018014E0022801D001281DD12068B3
:10504000018829802068418869802068A1880088BB
:105050004118A9802068A188408841182846E98025
:1050600032460146FBF7F7FF002806D0A0698560AD
:1050700062692169A06903F0D3FEA06986607CBDE6
:105080007CB50446806961898668A0896D460129DE
:105090000CD0012865D0814203D12289E3889A424D
:1050A0007ED300297DD003297CD0AEE0012822D117
:1050B000E088218988421ED20620205E0AF070FE18
:1050C0000421615E48432168C0134988411868463D
:1050D000C180E0885A3000B20AF062FE04210E223C
:1050E000615EA25E891A48432168C013098841188D
:1050F0006846818040E02068A1880088411A2980A4
:105100002068418869800620205E0AF049FE04215B
:10511000615E48432168C013498841186846C180D0
:10512000E0885A3000B20AF03BFE04210E22615E94
:10513000A25E891A48432168C01309883246411883
:10514000684681800146FBF786FF002806D0A069EB
:10515000856062692169A06903F062FEA089012867
:1051600053D1206801886846491E81802068A18843
:10517000408841186846C1800820205E0AF010FE71
:1051800004210E22615EA25E891A48432168C01381
:10519000498841186846418020895A3000B202E0AF
:1051A00014E00CE010E00AF0FBFD0421615E4843CE
:1051B0002168C013098841186846018018E0022858
:1051C00004D0032802D020E002281ED12068A18844
:1051D0000088411A298020684188698020680188F8
:1051E000491EA9802068A188408841182846E98086
:1051F00032460146FBF72FFF002806D0A0698560E4
:1052000062692169A06903F00BFEA06986607CBD1C
:105210007CB50446806961898668A0896D4602294B
:105220000CD002287ED0814203D12289E3889A42A1
:1052300079D3002978D0012977D0CEE002283FD158
:10524000E088218988423BD25A3000B20AF0A8FD9A
:105250000421615E48432168C013098841186846EB
:1052600001800620205E0AF09BFD04210E22615E73
:10527000A25E891A48432168C013498841186846CC
:10528000C1800820205E0AF08BFD0421615E484346
:105290002168C013498841186846418020895A30E6
:1052A00000B20AF07DFD04210E22615EA25E891A21
:1052B00048432168C01309884118684681807FE00F
:1052C00020680188491EA9802068A1884088411A69
:1052D0006980E0885A3000B20AF062FD0421615E04
:1052E00048432168C0130988411868460180062098
:1052F000205E0AF055FD04210E22615EA25E891A2D
:1053000048432168C0134988324641186846C18025
:105310000146FBF7A0FE00280BD0A06985606269FA
:10532000216903E008E038E030E032E0A06903F0F2
:1053300077FDA089022850D12068A1880088411AF1
:1053400068460180206841886846491EC1802089DE
:105350005A3000B20AF024FD04210E22615EA25EE2
:10536000891A48432168C01309884118684681801A
:105370000820205E0AF014FD0421615E4843216884
:10538000C013498841186846418019E0032804D0B9
:1053900023E0032801D000281FD12068A1880088BD
:1053A000411A29802068A1884088411A69802068B4
:1053B0000188491EA980206841882846491EE98045
:1053C00032460146FBF747FE002806D0A0698560FB
:1053D00062692169A06903F023FDA06986607CBD34
:1053E0007CB50446806961898668A0896D46032979
:1053F0000ED0032865D0814203D12289E3889A42E6
:105400007ED302297DD001297CD002297BD0ABE05C
:1054100003281FD1E088218988421BD25A3000B26C
:105420000AF0BEFC04210E22615EA25E891A484386
:105430002168C01309884118684601800620205E53
:105440000AF0AEFC0421615E48432168C01349881C
:1054500041183EE02068A18800884118A980206892
:105460004188491EE980E0885A3000B20AF098FC71
:1054700004210E22615EA25E891A48432168C0138E
:1054800009884118684601800620205E0AF088FCE1
:105490000421615E324648432168C013498841189F
:1054A000684641800146FBF7D6FD002806D0A0697A
:1054B000856062692169A06903F0B2FCA0890328B4
:1054C00052D120680188684601802068A188408800
:1054D000411A6846418020895A3000B20AF060FCC7
:1054E0000421615E48432168C01309884118684659
:1054F00081800820205E0AF053FC0421615E03E0F5
:1055000013E00BE00FE00BE00E22A25E891A484385
:105510002168C01349884118684617E0002804D064
:10552000012802D020E000281ED1206801882980AF
:105530002068A1884088411A69802068A188008875
:105540004118A980206841882846491EC1803246FA
:105550000146FBF780FD002806D0A06985606269DE
:105560002169A06903F05CFCA06986607CBD000035
:1055700070B5A4B00C46054620AA22A907F02DFE5E
:1055800022A802F020F8002804D120A802F01BF87D
:1055900000283FD012A928460BF066FF012839D118
:1055A0002146684607F074FA1B48019002200290D9
:1055B00012A80490012000040D9022A802F003F824
:1055C000002810D022A803906A461A21284604F029
:1055D000A1FE22AA12A9204603F022FC6A461B2142
:1055E000284604F097FE20A801F0EDFF002811D016
:1055F00020AE6A461A212846039604F08BFE20AAA4
:1056000012A92046039603F00BFC6A461B2128468C
:1056100004F080FE24B070BD181D0108F7B50C46DB
:105620002E21615EAAB01546002971D02046203097
:105630001A90807D02286BD9012909D13420205E7F
:10564000002805DC208E002802D1608E0028ECD0D6
:105650002888228EA38E8018C01A10A90883A988D2
:105660008918CE1810A98E836988628E8918A28E37
:105670008B1A10A94B83E988628E8918A28E8A182A
:1056800010A9CA832E21615ECF0F79184F10C01B5D
:105690006946401E88857F1CF01908862E20205EF2
:1056A000C10F08184010181A6946401EC8852E20E0
:1056B000205EC10F08184010401C1018694648862B
:1056C0001A98807D1C90FD2801D9FF201C902A98F3
:1056D0000BA9826828A8FBF7BEFC0028A5D02946A4
:1056E00020A801F061FF0021C9430A4620A801F06B
:1056F0008AFF0026A65F20A801F07FFF054620A8AC
:1057000001F05BFF854220A803DA01F076FF02E09A
:10571000FEE301F052FF4110B14200DA46100027CB
:10572000E75F16A801F069FF054616A801F045FFDE
:10573000854216A802DA01F060FF01E001F03DFFAA
:105740004110B94200DA47102E20205EC5192846C4
:105750006843400006F008FC15902E220146A25E28
:105760003B4616A80BF0A8FF0BA803F019F8012779
:10577000002805D1E078FF2802D3A07800280BD0BC
:1057800000270123324620A922A803F097FA00211E
:1057900022A802F025FE01E00020C0431E900BA8C5
:1057A00001F02BFF06F0E0FB0D901C2104A806F091
:1057B0002AFD6846049009900D980790A18D6846CF
:1057C00001831A98817D08A80172A1784172684608
:1057D000018E828D881A401C00B2C30F1818401029
:1057E000101800B218906846438EC28D981A401C5B
:1057F00000B2C30F18184010101804B26846818018
:10580000481B401C01B2684601804280681E199006
:10581000101802B26846C2801898814200DC014626
:1058200068460180A24200DB2246C2802A9869466F
:10583000826802A8FBF70FFC00285AD0324620A944
:1058400002A8FBF730FC002853D16A460820105EFE
:1058500091898446081A401C00B21B900A21515EAF
:1058600068462E22825E159B881A6946302268435C
:105870008A5EC3186046511B401AC018401E109023
:10588000002F09D0324620A902A8FBF778FC002897
:1058900002D00120149000E014971B98002828DD06
:1058A0000D980790684601890180818981800221D5
:1058B00008A8017068460A22825E0F9213E06946CA
:1058C00048800F98C880149800283BD01098079003
:1058D00004A92A9803F0B0FC1098401910900F9872
:1058E000401C00B20F9068460E21415E0F98814225
:1058F000E5DA6946088E8880401B401C02B20A80A7
:105900004B8E581B401C00B24880CB8018998A42AD
:1059100000DC0A4669460A80611C1B91884200DC53
:10592000601C694648802A98826802A8FBF793FBAE
:1059300000286FD0324620A902A8FBF7B4FB00284C
:1059400014D067E02A4610990D9806F0A3FB6A462A
:105950000821515E1B9B0F9A0D9802F0E9FE08AAE0
:1059600010700128B4D102201070B1E76A460820F7
:10597000105E91898446081A401C00B21D900621D1
:10598000515E68460E22825E159B881A6946302257
:1059900068438A5EC3186046511B401AC018401EF7
:1059A0001090002F09D0324620A902A8FBF7E7FB90
:1059B000002802D00120149000E014971D980028C0
:1059C00028DD0D98079068460189018081898180D2
:1059D000022108A8017068460E22825E0F9213E031
:1059E000694648800F98C8801498002836D01098CF
:1059F000079004A92A9803F01FFC109840191090F2
:105A00000F98401E00B20F9068460A21415E0F9821
:105A10008142E5DD6846808D411968460180008E2F
:105A2000411B68468180C18D41801998081801B2D8
:105A30006846C180A14200DB2146C1802A986946A0
:105A4000826802A8FBF707FB002806D0324620A98F
:105A500002A8FBF728FB002814D07CE02A46109906
:105A60000D9806F017FB6A460821515E1D9B0F9AA0
:105A70000D9802F05DFE08AA10700128B9D102202D
:105A80001070B6E76846818900890222081A401C16
:105A900000B21D9068460A21415E825E159B881AFD
:105AA0006843C0181090002F09D0324620A902A8E0
:105AB000FBF765FB002802D00120149000E014974A
:105AC0001D98002847DD149800280AD00020079070
:105AD000684601890180818981800A21415E0F9198
:105AE00033E00D98F3E7694648800F98C880149812
:105AF00000280BD01C98FF281098007803D01A9922
:105B0000897D4843000A08A9087213E010981D9A7D
:105B100001780D9806F049FB6A460821515E1D9BED
:105B20000F9A0D9802F004FE08AA1070012801D106
:105B30000220107004A92A9803F07EFB10984019E7
:105B400010900F98401C00B20F9068460E21415EE5
:105B50000F988142C7DA1A9808A9807D08726946B1
:105B6000888D40190880088E401B88804A8E501B03
:105B7000401C00B24880CA801B99884200DC601C2F
:105B8000694648802A98826802A8FBF764FA0028D0
:105B90006AD0324620A902A8FBF785FA002863D113
:105BA0006846818900890E22081A401C00B21490B0
:105BB00068460621415E825E159B881A6843C018BC
:105BC0001090149800284FDD002F06D0324620A9EF
:105BD00002A8FBF7D4FA002000E00D980790684671
:105BE00001890180818981800E21415E0F9135E01C
:105BF000694648800F98C880002F10D0324620A9EF
:105C000002A8FBF7BCFA1C98FF281098007803D074
:105C10001A99897D4843000A08A9087213E0109870
:105C2000149A01780D9806F0C0FA6A460821515E70
:105C3000149B0F9A0D9802F07BFD08AA10700128A2
:105C400001D10220107004A92A9803F0F5FA1098E7
:105C5000401910900F98401E00B20F9068460A211C
:105C6000415E0F988142C3DD1A9808A9807D0872B1
:105C70006946088E411B491C0BB269460B8088801F
:105C8000C88D401900B24880498E491B0AB2694646
:105C9000CA801B99884200DB601C69464880A2428A
:105CA00000DC2246CA801898834200DC03460B8041
:105CB0002A98826802A8FBF7CEF9002864D0324601
:105CC00020A902A8FBF7EFF900285DD1694608205A
:105CD0008A89085E111A491C09B21A91199A1599F4
:105CE0006A435318694630228A5E511B401AC01815
:105CF000401E1090002F1CD0324620A902A8FBF7AE
:105D00003EFA002802D00120149000E01497109869
:105D100007901A98002837DD68460189018081893B
:105D20008180022108A8017068460A22825E0F92D3
:105D300024E014970D98EBE7694648800F98C880D7
:105D40001498002812D11A9A10990D9806F0A2F909
:105D50006A460821515E1A9B0F9A0D9802F0E8FCE2
:105D600008AA1070012801D10220107004A92A98F5
:105D700003F062FA0F98401C00B20F9068460E21A3
:105D8000415E0F988142D7DA002115981AE0411937
:105D90001F91491E1091EA0F00215219521094468A
:105DA0000AE0109B02781B780370109B401C1A704D
:105DB000109A521E491C10928C45F2DC0F991F98C4
:105DC000491C09B20F91A942E1DB6A46908D10800F
:105DD0001999401801B29180D08D401900B25080BD
:105DE000528E521B13B26A46D3801B9A904200DB3C
:105DF000601C6A465080A34200DC2346D38018987A
:105E0000401E1C90814201DB1899491E91802A98FE
:105E10006946826802A8FBF71EF9002862D0324664
:105E200020A902A8FBF73FF900285BD169460820AA
:105E30008A89085E111A491C09B21A91199A159992
:105E40006A435318694600228A5E801AC01810906F
:105E5000002F1CD0324620A902A8FBF790F9002899
:105E600002D00120149000E01497109807901A981F
:105E7000002837DD684601890180818981800221FF
:105E800008A8017068460A22825E0F9224E01497E7
:105E90000D98EBE7694648800F98C8801498002851
:105EA00012D11A9A10990D9806F0F4F86A46082152
:105EB000515E1A9B0F9A0D9802F03AFC08AA1070D6
:105EC000012801D10220107004A92A9803F0B4F926
:105ED0000F98401C00B20F9068460E21415E0F984B
:105EE0008142D7DA6946888D08801999401800B236
:105EF00069468880CA8D4A80199951180AB2694644
:105F0000CA801C99884201DB1898401E694600E04F
:105F100062E18880A24200DB2246CA802A98826819
:105F200002A8FBF798F8002859D0324620A902A809
:105F3000FBF7B9F8002852D16A460820105E918913
:105F40008446081A401C00B21A900A21515E684625
:105F50000222825E159B881A684369460022C31894
:105F60008A5E6046801AC0181090002F09D0324611
:105F700020A902A8FBF703F9002802D00120149001
:105F800000E014970D9807901A98002827DD6846BE
:105F90000189018081898180022108A801706846F9
:105FA0000A22825E0F9214E00846694648800F98E4
:105FB000C880149800283BD01098079004A92A980C
:105FC00003F03AF91098401910900F98401C00B255
:105FD0000F9069460E20085E0F998842E4DA6A46FF
:105FE000908D10801999401801B29180538E581BE2
:105FF000401C00B25080D3801B9A904200DC601C91
:106000006A4650801C98814201DB1899491E918094
:106010002A986946826802A8FBF71DF800286BD011
:10602000324620A902A8FBF73EF8002814D063E00E
:106030002A4610990D9806F02DF86A460821515EFF
:106040001A9B0F9A0D9802F073FB08AA1070012892
:10605000B4D102201070B1E7684608248189045F3A
:106060000622081B401C00B2139068460E23825E75
:10607000C35E1599D01A6843411868460022825EB3
:10608000A01A40181090002F09D0324620A902A86B
:10609000FBF775F8002802D00120149000E0149757
:1060A0000D9807901398002826DD68460189018025
:1060B00081898180022408A8047068460E21415E0F
:1060C0000F9113E0694648800F98C8801498002803
:1060D00035D01098079004A92A9803F0ADF81098CD
:1060E000401910900F98401E00B20F9068460A2188
:1060F000415E0F988142E5DD6846808D4119684612
:106100000180008E411B68468180C08D4119684620
:106110004180408E411B6846C1800D9807902A98A7
:106120006946826802A8FAF796FF002846D03246F0
:1061300020A902A8FAF7B7FF002813D03EE02A46AC
:1061400010990D9805F0A6FF6A460821515E139B31
:106150000F9A0D9802F0ECFA08AA10700128BAD133
:106160001470B8E768460C220821825E415E501A1E
:10617000401C05B2002D21DD6846018082800A2482
:10618000045F16E04C80CC8029460D9806F065F837
:1061900069460820085E2B46014622460D9802F00B
:1061A000C7FA08A9087004A92A9803F045F8641CE6
:1061B00024B269460E20085EA042E3DA002F05D122
:1061C00022A802F0D3FA1E9802F01CFE159805F0E2
:1061D00013FF0D9805F010FF2DB0F0BD70B504460B
:1061E00005F01CF900280AD000688268002A01D056
:1061F000217A9047207E810745D4C0077DD10021B8
:10620000606806F08BFE002518E0017ACA0910D0FC
:10621000802904D04906227A490E914209D1416869
:10622000E160016820468847207E81072BD4C007A3
:1062300069D16D1C2946606806F070FE002803D005
:1062400001680029F5D0E0E72146002006F0C0FDF6
:1062500005005AD00021606806F060FE00261BE0B1
:106260000168002913D0017A0A0610D4002902D04F
:10627000227A91420BD14168E1600168204688474B
:10628000207E810701D5012070BDC0073BD1761C5F
:106290003146606806F042FE002802D0012DDFD0B2
:1062A00033E0012D31D16068416800292DD0217E75
:1062B00049072AD4217A23291AD0242918D0A903DE
:1062C00007F014FD002820D0207A11380300FAF7D7
:1062D000E3FD1C1C1C1C1C1C1C1C1C1C1C1C0F0F70
:1062E0001C0F0F1C1C1C1C0F0F0F0F1C1C0F1C0F56
:1062F000606840686060204600E004E0FFF76EFFE1
:106300000546012801D0002070BD284670BD000060
:10631000FFB58B880D888BB05B1B5B1C1FB2CB88D5
:1063200049880446591A491C179809B20591012851
:1063300014D0022814D0032843D1454E510015989B
:10634000089100280ED00020069020886946888099
:1063500015980078FD2836D3149A37E03D4EEDE7C6
:106360003D4EEBE72088694688800881149A02999F
:106370000E98B047049000201FE0002517E0684603
:10638000818868000690205A81420AD006986946A2
:106390000019008888808884149A09990E98B0475B
:1063A0000490069869460019098A01806D1CBD4257
:1063B000E5DB089804190298401C05990290884270
:1063C000DBDB0FB0F0BD14994843020A01990E9827
:1063D000B0470A90002036E000252AE01598405D7D
:1063E000002825D00699884205D169466A00898827
:1063F000A25A914217D0FD2801D3149A02E01499B1
:106400004843020A68000990001900886946088319
:1064100006990E98B0470A9015986946405D069017
:106420000998205A8880680069460019098D018002
:106430006D1CBD42D2DB08981699041915984018B6
:1064400015900298401C059902908842C4DBB8E779
:106450005D2E0008D92D0008C72E0008FFB50446A0
:1064600088880A888DB0801A401C05B2C88849887F
:10647000179E401A401C00B205900F9840000890EB
:10648000002E0CD010A8008807900104401802903C
:106490001698FD287ED3281F019000202CE1169825
:1064A000FD280ED3002607E02A462046109901F069
:1064B0008FF908980419761C05988642F4DB11B010
:1064C000F0BD684600883F214009400149018843EA
:1064D0004105490D6846018088B2009068460088F1
:1064E00001900146169A109801F014FA029016983D
:1064F000001DC008C006010E1098039068468289EE
:10650000D30A4B4303835005830ED2064B436846A0
:10651000D20E43834A438283FF20401A86460022DC
:106520004DE0002046E0694643008988E65AB142C2
:106530003BD0191909886F46B98039813E8B8C464A
:10654000CF0A71464F43F119934F79436F463F8EFF
:10655000C90E7F05C9027F0D39430C916F46614614
:106560007E8B49058F0E71464F43F1198B4F3F26A5
:106570007943890E4F010C997601B1430F4361466F
:10658000CE060C976F46F60E7146BF8B4E43BE1972
:10659000814900E0B8E04E430C9FF10E7E09760180
:1065A00031436F46398689B2029119196B461B89AE
:1065B0000B80401CA842B6DB08980419521C0598B1
:1065C0008242AEDB7BE7002710E03278FF2A12D050
:1065D0002188684601830699109801F09BF906907E
:1065E0006846008B2080A41C761C7F1CAF425BDABF
:1065F000B007EAD158E00798F4E73168481C42D068
:1066000000294ED03278FF2A52D021886846018373
:106610000699109801F07EF906906846008B20805C
:106620007278A41C761CFF2A44D021886846018316
:106630000699109801F06EF906906846008B20804C
:106640007278A41C761CFF2A36D021886846018304
:106650000699109801F05EF906906846008B20803C
:106660007278A41C761CFF2A28D0218868460183F2
:106670000699109801F04EF906906846008B20802C
:10668000A41C761C0FE0A00707D007982080A01C50
:10669000029901600798E08003E002982060029868
:1066A00060600834361D3F1D01988742A5DD18E063
:1066B0000798B4E70798C2E70798D0E70798DEE79E
:1066C0003278FF2A1ED021886846018306991098E7
:1066D00001F020F906906846008B2080A41C761CEF
:1066E0007F1CAF42ECDB0F98401B40000419189848
:1066F000401B86190398401C05990390884200DAD4
:1067000061E7DCE60798E8E720886A469080002188
:1067100090840846029137E000272CE0307800286A
:1067200027D0884205D0169AFF2801D04243120A8A
:106730000292884205D168467A008088A25A904227
:1067400012D00298FF2824D07800001900886946EA
:106750000883029A0699109801F0DCF809907800F5
:106760003178205A6A46908078006A460019928CE7
:106770000280761C7F1CAF42D0DB08980419189861
:10678000401B86190398401C059A03909042C3DB76
:1067900095E61098E2E700001008080008040400DD
:1067A000FFB58DB00C46FBF7FDFA0A9010A81799BB
:1067B0000088099000290DD0A0882188401A401C2B
:1067C00000B20590E0886188401A401C00B20026A3
:1067D000079043E00226A65F18E00025655F30B20F
:1067E00007900EE0169802906946099888800798ED
:1067F00000900A982BB200680F9AC7690D99B847A4
:106800006D1C0420205EA842ECDA761C0620205E77
:10681000B042E2DA11B0F0BD002517E0405D00287B
:1068200013D016994843000A029069460998888057
:1068300060880D99801900B2009020880F9A401945
:1068400003B20A980068C769B8476D1C059885426D
:106850001798E3DB18994018761C17900798864222
:10686000DADBD7E700680968884201D10120704768
:106870000020704740680A6880008008904200D27B
:10688000086000207047F7B5054684B000200090EE
:10689000287FC00766D100260120EC680190029095
:1068A000002C0FD1287F0007C00F401E304259D165
:1068B0000298002856D005992846884704460020AB
:1068C00001900290002E01D126004BD001980028A3
:1068D00006D0069A2146284690470446B04241D049
:1068E00001200190002CDDD0206806F0B7FF0006E3
:1068F000D6D4276823E00121384607F0F7F90028AD
:1069000019D0002F05D00121384607F0EFF90028F3
:10691000C6D1E868A04225D0002817D0284600F04C
:10692000B7F8E96802460B680F21184603F0F2FC3D
:10693000012817D106E0384606F00AFB0746002F6B
:10694000D9D1E6E7E868006807F097FB2846EC60D5
:1069500000F09EF80246E8680E21006803F0DAFCB9
:10696000012802D0009807B0F0BDE868006807F081
:1069700084FB2969002901D0284688470120F2E7D5
:106980000C21415E4800C01C800880001030704718
:10699000FEB50F0021D005696969002904D0086897
:1069A000B84201D14868FEBD688A0024C605F60DCC
:1069B0000BE022461420AB6842439858121D9A5AA5
:1069C000381A82420BD2641CA4B2A642F1D8002924
:1069D00003D00F606969002048600020FEBD1422CA
:1069E0005443224612329A5C00261946022A07D0E6
:1069F000002A08D0254B032A0CD0012A21D03CE0E4
:106A0000A41D195B38E022460C328A58A41D195B7C
:106A1000105C31E06A4690802046009310300A5A9C
:106A2000083802900958022301A8FBF7AFFA0028A2
:106A300023D0A968029A8A58801A4010A41D095BC5
:106A40001AE06A4690802046009310300A5A0838AF
:106A500002900958022301A8FBF798FA00280CD0ED
:106A6000A968029A8A58801A22460C32A41D401046
:106A70008A584000095B105A0E186869002802D035
:106A80000760686946603046FEBD0000111D0108C0
:106A9000F8B500260746354630460EE004F0EDFC1A
:106AA000616DB94208D1022802D0042802D002E068
:106AB0002046F8BD26462546204604F0B5FC0400D5
:106AC000ECD1002E01D03046F8BD002D01D0284673
:106AD000F8BD002004F0A8FCF8BD00007CB50369F7
:106AE00000695B8AC4680025A0689B042CD4830FCE
:106AF00003D0800F012813D034E0120251186A46E7
:106B0000266891801849820000919208022331463C
:106B100001A8FBF73BFA002824D0801B401011E0AD
:106B2000100440182668019010480090A0680423C3
:106B300082009208314601A8FBF728FA002811D0FC
:106B4000801B801061680CE06368805C595C0029E0
:106B500008D0002806D0627B491E23684A43991852
:106B6000401E0D5628467CBD6F6E00085B6E000807
:106B7000FEB500681546C068C068F9F725FC0446F4
:106B8000A84200DD2C46154F78680068806900280F
:106B900021D00020694608808880488025B2681E80
:106BA00006B26846C6807868694600688269904780
:106BB0006846C1884088081A401C00B2A04202DD25
:106BC000351EECDC01E0002D01DC0020FEBD684636
:106BD0000624045F641C2046FEBD00002C0000203B
:106BE000FFB585B005461F460798FBF7E2F801217F
:106BF0008140C8B20490288C0290C04380B20390B8
:106C0000688C00260007C00FF643002400901EE0A9
:106C1000EA68E100501843689B0141D5009B002BB6
:106C200014D1091D51580902090E0A0406998A4215
:106C30000CD10068049A8179114207D001AA079902
:106C400008F062FC012832D0022833D0641C688C22
:106C50008005800EA042DBD822E0E968E0000A58F7
:106C6000049B944692791A4219D0001D08580102DB
:106C700080B20090090E0698090481420FD1039951
:106C8000009808420BD10098B04208DD604601AA86
:106C9000079908F039FC01280ED002280AD0641C9C
:106CA000688C8005800EA042D7D8002E0EDB01989C
:106CB0003860012009B0F0BD029900988842F6D0F2
:106CC0008642ECDA064601983860E8E70020F1E7F2
:106CD000FFB5D00781B0C6170F4601985A21081A90
:106CE0001D46540800B2761C09F05AF8391B484377
:106CF000C7110091019809F053F800994843C01159
:106D0000002F06DD7F3F39120A1B92192A800919CC
:106D100005E07F3739120A1B09192A80891BA980CF
:106D2000002806DD7F380012011B891969800019CF
:106D300005E07F300012011B00196980801BE8808C
:106D400005B0F0BDF8B50446638C0D4600209905EA
:106D5000890EE26809E0C600361D9659B70103D5D1
:106D60003602360AAE4202D0401C8142F3D881423C
:106D700002D0C0001018F8BD0A20C34101208006CF
:106D800018181621C84160848005800EC100104685
:106D900005F068F9E060608C8005800E06E0E2682E
:106DA000C10053180839521806CA06C3401EF6D14E
:106DB0000821E06805F027FA082005F0A7F8E16847
:106DC000086008F049FCE168012248685206104357
:106DD0004860000E00062A02120AE168104348606B
:106DE000E068F8BD024600B50021303A092A01D812
:106DF000D1B216E0612801D32038C0B24138030077
:106E0000FAF74AF8060406080A0C0E0F0A2108E0F1
:106E10000B2106E00C2104E00D2102E00E2100E030
:106E20000F21084600BDF8B5064615460F4600205E
:106E300005E039462046B047012809D0204609F030
:106E400015FD040002D060688000F2D10020F8BD7A
:106E5000002D00D02C600120F8BD03880A889342E1
:106E600001D0981A704740884988401A70470378C3
:106E70000A78934201D0981A704740784978401AAE
:106E800070470000F8B542680968920092088A428B
:106E900023D10446FFF774FD114905468A68131B88
:106EA000501B5E1B8860002E15D0274661193246A4
:106EB000384605F0EFF806E0A068401BA0602046C9
:106EC000FFF75EFD0419064880688442F4D1B819C2
:106ED000294605F098F90120F8BD0020F8BD000012
:106EE000C4000020FFB5064683B01446D8072AD058
:106EF0002046314608300125002214310746FAF7B2
:106F0000D2F800280CD00021684601706A46122190
:106F10003046019703F0FEF968460078002812D049
:106F20006089218A4018401EE0810E210620615EA2
:106F3000205E814200DDE0812A462146049801F06E
:106F4000C5F907B0F0BD0025EFE7FFB5064689B0EB
:106F500015460F460846FAF720FD044602A93846B2
:106F600005F0B3FF2246114602A800F04CFB022DAB
:106F700004D0012D27D000200DB0F0BD0399029858
:106F80000023059104901A4604A9384606F0F5FD41
:106F900004AA6846B168FAF75EF80028ECD00199B7
:106FA0000098079106900123002206A9384606F0B2
:106FB000E4FD06A902AA0846FAF74DF80028DBD03E
:106FC000082206A908E002AA6846B168FAF743F861
:106FD0000028D1D0082269460C98F9F743F901201E
:106FE000CAE7000070B5044605F00AFF0646002512
:106FF00006E0A068A90000684058FFF7F3FF6D1C89
:10700000B542F6D3608CC1071DD0400840006084B3
:10701000204607F05BFB204607F066FA002E12D0F0
:107020000021204606F079FC00280CD00B49496865
:10703000884208D8C1000A48006808188038826F62
:10704000C16F20469047608C810706D50221884396
:1070500060840021204607F057F970BD2000002011
:1070600098000020FFB581B00A9DE8692E460346CE
:107070004B439B122036002805DD934205DD307A14
:1070800080070DD485E09342F9DB049BCB18434382
:107090009B12002807DD934232DA307A800778D4D9
:1070A000012005B0F0BD9342F7DCA869521C5043A3
:1070B0000002801203120206120E23D0FF206F6A14
:1070C000841A7C432412071B5C1A0094002A34D0D3
:1070D000002C13DB0498844210DAFF20811AC21BB3
:1070E00051434912411A327AC9B2920700D5411A66
:1070F0000198005D09F0ACFB01990855641C1CE087
:10710000A869D4E7FF27DFE7002C10DB04998C4245
:107110000DDA4010381AC1B2307A800701D5FF204D
:10712000411A0198005D09F093FB01990855686ABE
:10713000641C3F1A0498844202DA686AB842E3DBAE
:107140000498844217DA002C15DBA8697843801272
:107150007843C003010EE869002801DAFF20411AD4
:10716000307A800701D5FF20411A0198005D09F0AF
:107170006FFB01990855307A800708D5009904986B
:10718000814206DC00290EDB01980AE001E0641C64
:1071900001D5002085E70498844204DC011B019896
:1071A000001905F030F802207BE7FFB583B00646F2
:1071B0000C981D468069014651438C12002800DD61
:1071C000641C0C9B049F203300931B7ABC4202DAA0
:1071D000980706D4CCE08C127F19A74202DA9807F0
:1071E000F8D47AE0521C424312029412221209028D
:1071F000E4B28912A4460F12049CC9B23C1B974208
:1072000006D0002804DA002902D1FF211746641EA7
:10721000974222D1002C0CDBAC420ADA60460818F7
:107220004110980701D5FF20411A305D09F010FB8D
:1072300030550098641C007A80077ED50498391A6E
:10724000A9427BDA8AE0304604E0002C76D003DDE8
:10725000291B301904F0D7FF83E0002843DA0C988B
:10726000C0694042484380120190002C0CDBAC42C4
:107270000ADA4843C003010E980701D5FF20411ADE
:10728000305D09F0E5FA30550C9881690198FF38B6
:1072900041438912641E11D4AC420FDA019AFF20D7
:1072A000821A4A435112009A411A127AC9B29207BD
:1072B00000D5411A305D09F0CBFA30550098A41C76
:1072C000007A800707D50498391A491EA94248DC7C
:1072D0000029B8DC45E0AC4202DD012007B0F0BD7A
:1072E000002CB5DA3DE0FF20411A0C98C0694843F4
:1072F00080120190002C0EDBAC420CDA019AFF20C8
:1073000051434912411AC9B29A0700D5411A305D5A
:1073100009F09EFA30550C9A0199FF209269411AA2
:107320004A439212641C10D4AC420EDA5143009AC4
:10733000C903127A090E920701E014E018E000D5A3
:10734000411A305D09F084FA30550098641C007AC7
:10735000800708D50498391AA94209DC002900DB06
:1073600071E70220BAE7AC4200DC6EE72C466CE71E
:107370000020B3E7F3B5074681B000261448FAF7BA
:1073800042FA04461FE021461148FAF740FA054642
:107390002068B84201D0002F14D161680298814260
:1073A00001D000280ED121460948FAF7C2FA216916
:1073B000002901D020468847204604F02FFEFAF726
:1073C00095FE01262C46002CDDD13046FEBD000086
:1073D0001C11002070B505460C460948FAF713FA4F
:1073E0000BE00168A94204D14168A14207D0002CFA
:1073F00005D001460248FAF70AFA0028F1D170BD1B
:107400001C11002010B50446442104F0FCFEFF20AE
:10741000F530E062002020626420A0622046012155
:1074200040300180024AE26182780A43827010BDD6
:107430006D74000838B50125AD0200950446C26A96
:107440000023006B194604F041FDE122064B920037
:107450000021009500F0FDF8226AA16A891A4143D3
:107460008812101838BD0000B603000038B5044675
:1074700001208002009000231946E26A206B04F08C
:1074800025FD226AA16A891A41438812101838BD65
:10749000034610B5881A002800DC501A7D21C90067
:1074A00048431946F8F790FF002800D1012010BD8D
:1074B00070B541680546002902D02868FFF75AFFD9
:1074C0001C48FAF72AFA1C4E002802D008F060FA8D
:1074D00070601848FAF7B0F9040029D04422294610
:1074E00004F0D8FD2868A84200D12460214640312C
:1074F0008878FB2210407278920010438870C00791
:1075000012D06169002907D020468847216A0918EE
:107510002162A16A0818A0626268002A04D020686B
:10752000002801D0216A9047FAF7E0FD204670BD9F
:10753000FEE700001C110020B80000200A8802802D
:107540004A8842808A888280C988C18070470A88B8
:1075500002804A8842808A888280C988C1807047B8
:107560000A8802804A8842808A888280C988C180CD
:1075700070470A8802804A8842808A888280C98847
:10758000C18070470A8802804A8842808A88828047
:10759000C988C18070470A8802804A8842808A88E8
:1075A0008280C988C18070470A8802804A884280E8
:1075B0008A888280C988C1807047C1884088081A3B
:1075C000401C00B2704704210022415E825E02230B
:1075D000891A0622825EC35ED01A401C491C4843A9
:1075E000704781880088081A401C00B27047818863
:1075F0000088081A401C00B2704781880088081A69
:10760000401C00B2704703885B1A038083885918B6
:1076100081804188891A4180C1888918C18070475A
:1076200003885B18038083885918818041888918F2
:107630004180C1888918C180704710B5029C0180C3
:1076400042808380C48010BD4288491E5118C18089
:107650007047F0B59C4601239B021C1A23466343E6
:107660009D0A2B4663439F0A034643439E0A4543B4
:107670005543334643437443624654436200A21861
:1076800068004F432818059C9B0AB90A000D120D8B
:10769000634308189B0A8018C018F0BDF8B5064669
:1076A0004804800F1F4614460D46012810D10321BF
:1076B0004903284688437D210901884208DC491096
:1076C000884200DD081A78436421F8F78BFE05B282
:1076D0006004800F012810D103212046490388430C
:1076E0007D210901884208DC4910884200DD081A22
:1076F00078436421F8F776FE04B2A64201DA3046F8
:1077000000E02046A84201DA2846F8BDA64201DA88
:107710003046F8BD2046F8BDF8B506464804800F4F
:107720001F4614460D46012810D10321490328465F
:1077300088437D210901884208DC4910884200DD28
:10774000081A78436421F8F74DFE05B26004800FF3
:10775000012810D103212046490388437D210901D6
:10776000884208DC4910884200DD081A7843642109
:10777000F8F738FE04B2A64201DA304600E02046AF
:10778000A84201DA2846F8BDA64201DA3046F8BD23
:107790002046F8BD002208B51146104600F04CF80E
:1077A00000906846008808BD002208B511461046C2
:1077B00000F058F800906846008808BD002208B51F
:1077C0001146104600F064F800906846008808BD35
:1077D00007B56B469B88810702D00380801C521E30
:1077E0001904591809E0016041608160C1600161BC
:1077F00041618161C1612030103A102AF3D802E062
:107800000380801C521E002AFAD10EBD08B56B46BB
:107810001B88D2085B095B0113433F225201890890
:10782000934349010B435905490DC008C002014368
:107830006B46198088B208BD08B56B461B88D20814
:107840005B095B0113433F225201890893434901BD
:107850000B435905490DC008C00201436B4619800E
:1078600088B208BD08B56B461B88D2085B095B016E
:1078700013433F2252018908934349010B435905A1
:10788000490DC008C00201436B46198088B208BD8B
:1078900008B56B461B88D2085B095B0113433F2286
:1078A00052018908934349010B435905490DC0080A
:1078B000C00201436B46198088B208BD08B56B460B
:1078C0001B88D2085B095B0113433F2252018908E0
:1078D000934349010B435905490DC008C0020143B8
:1078E0006B46198088B208BD08B56B461B88D20864
:1078F0005B095B0113433F2252018908934349010D
:107900000B435905490DC008C00201436B4619805D
:1079100088B208BD17B581B069460889121D0104F7
:1079200008436946D3088988084A0C04214310405B
:107930001140091A5943490908181040020C024322
:1079400069460A8090B204B010BD00001FF8E0073D
:1079500017B581B069460889121D010408436946BC
:10796000D3088988084A0C04214310401140091AA1
:107970005943490908181040020C024369460A801D
:1079800090B204B010BD00001FF8E00701B581B04F
:1079900068468188FF22C80A08325043C01D420948
:1079A000684682704805FF22800E04325043C01C96
:1079B000820968464270C806FF21C00E083148435C
:1079C000C01D410968460170FF21C17000980CBDBF
:1079D000FF2208B511461046FFF744FF00906846A5
:1079E000008808BDF8B50D461E46174604461C2102
:1079F00004F009FCA0C460C4F8BD000038B504461A
:107A0000502104F000FCFF2041302080F0206080F5
:107A10000020C043A080E080002020816081206998
:107A200008210843402188430949084041210902AF
:107A300040183F212061490168460180009100887B
:107A400020870448206460645820A06438BD00008A
:107A50007F00FEFFF5970008F8B505464848F9F79E
:107A6000EBFE040003D0E86B002801D00AE0FEE73B
:107A7000A86C04F04BFA060079D001462A6C28461F
:107A80009047EE63FF216931204604F0BCFBFF20E4
:107A900001215530256001512046FF300821593021
:107AA000F9F7C2FE374E2246F7681E213648F460C9
:107AB00007F082FF606000285AD0286981070BD543
:107AC00000210222695EAA5E5143EA68D2689142AF
:107AD00002D9022188432861684600881F21400995
:107AE000400108433F2149018843084341051F20C5
:107AF000490DC00201436846018088B20090684683
:107B000000880090684600886085FF212920015583
:107B1000002004F027FE2061002004F023FEE06135
:107B2000002004F01FFE194D20622A460021E06962
:107B300007F034F82A460021206A07F02FF80221C6
:107B4000E06904F07DFD0221206A04F079FD002146
:107B5000E06907F01EFA0021206A07F01AFA20698E
:107B600006F08BFAF760002F03D003E0FFE7FEE793
:107B7000FEE7F460606807F0F0FF2046F8BD000003
:107B8000F8100020340000207D130008FFFF0F00D4
:107B9000C26800211161C068416170470148C06836
:107BA0007047000034000020002803D10548C06859
:107BB000002804D000680069C003800D704782204F
:107BC00070470000340000200068C0687047000063
:107BD000002803D10848C068002809D00168087C43
:107BE0008006800F012804D0032802D00020085E00
:107BF00070470220085E70473400002010B500284E
:107C000003D1FFF7CBFF002800D0006A10BD10B5EC
:107C1000002803D1FFF7C2FF002800D0C06910BDC3
:107C200010B5002803D1FFF7B9FF002800D0006984
:107C300010BD10B5002803D1FFF7B0FF002800D019
:107C4000406910BD10B5002801D1FFF7A7FF80687B
:107C500010BD0000002803D10848C068002809D0E2
:107C60000168087C8006800F012804D0032802D018
:107C70000220085E70470020085E70473400002034
:107C800010B5002803D1FFF789FF002805D0FF3089
:107C90000130406D002801DD012010BD002010BD25
:107CA000FFB581B01D000E46044619D0F07A0228B7
:107CB00014D9E769002F04D02046039AB847012859
:107CC0000CD02B4631462046039AFBF721FA0128B7
:107CD00004D005A22046039909F0B7FD05B0F0BD18
:107CE00001A20399F8E700004E6F0A646174610015
:107CF00038B58469049D002C01D00095A04738BD9B
:107D000038B50446182104F07EFA002211461046C8
:107D1000FFF77CFD00906846008800906846008868
:107D20002081FF20E072401C60800120207538BD5A
:107D300070470000FFB5B5B0887E3E9F1E460C46DA
:107D400002287DD9206800287AD03598006A00285A
:107D500076D0202217A8F8F705FA20681590002E93
:107D60006ED0307800286BD035983799826832A869
:107D7000F9F771F9002863D0207F20A90870E27E0E
:107D800069460A71002802D1012020A90870607F8D
:107D9000810706D4379881880088081A401C03B2EE
:107DA0000FE01221615EFD4A0091029001921423BE
:107DB000E35E314621A8226808F0B8F820A8042321
:107DC000C35E15990820085E12211F90615E6A4605
:107DD00008182490379800250088908137984188AA
:107DE000D1811620205E31901820205E0918D181A3
:107DF000002F20D000281ED137990220085E0028CD
:107E000019DABA68111A002900DC811A24980122B3
:107E100040009202101A814201DC386802E0002022
:107E2000C0433860002806DB05466946C889B98822
:107E300040186946C881617F00201422019100E04A
:107E4000AFE00090A25E70192D931599FAF700F833
:107E5000401916902EE0617F00200090169D019140
:107E60001422A25E70192D9B1599F9F7F1FF169D4A
:107E7000694640191690C9892498081800B26946C5
:107E8000C881002F13D001218902C8420FDB386856
:107E900000280CDA68460E213D60415E37980222C8
:107EA000825E881A786037980221415EB960705D01
:107EB000002876D069460E20085E1F994118359833
:107EC00082680220105E8142C5DB20A800782A90DB
:107ED000022802D0032818D02BE0607F009016986B
:107EE0001423411BE35E7019159A08F07FF80746CA
:107EF0003798FFF77CFBC01B6946C20F89891018B1
:107F0000401008186946888113E0607F0090169839
:107F10001423411BE35E7019159A08F067F80746B1
:107F20003798FFF764FBC11B6846808909186846CB
:107F3000818161682191A0682090814203D908461F
:107F4000209921912090A07F800718D012A800F0DE
:107F50002AFAA08910A9088115980E2141560029F6
:107F600000D1012110A84181A17E0174407C8108CB
:107F7000A07F8900C006800F014310A84174002033
:107F80002690FFF707FC2990FFF704FC1F9004A838
:107F900000F05AFF208A694688820C20085E2C90E7
:107FA00067E16AE1694689893198002708186946BE
:107FB0008881701925972B901698401B3090BBE054
:107FC000002101917649219A8A4209D0744A209968
:107FD000914205D0734A29181268304690470190A3
:107FE00025AB2FAA27A92B98F9F71AFF607FC007A6
:107FF0000BD02798232802D0012F14D005E0002FA2
:1080000008D0012F0AD0022F0BD0E0681F90022F5A
:108010004CD04DE02598269001200FE00027E06825
:1080200045E000200AE0202809D125992698081A61
:10803000072805D0A08920A98884022007467BE074
:10804000269A2B9869468018062203780B70401CEC
:10805000491C521EF9D10021684681710078FEF753
:10806000C1FE070168464078FEF7BCFE381829902B
:1080700068468078FEF7B6FE07016846C078FEF7CE
:10808000B1FE3818239068460079FEF7ABFE070171
:1080900068464079FEF7A6FE3818C2B22398C1B2EE
:1080A0002998C0B2FFF7C8FB2990C6E729981F900E
:1080B0002F9A2799159802F018FA28903848219994
:1080C000814225D02099814222D001992198814274
:1080D0001ED30846209988421AD26946888920A969
:1080E00008816946CA8920A94A81A18A411828982D
:1080F000401E081820A988812498401E1018C881A5
:1081000022AA04A9359800F08BFEE08910A988877F
:1081100010A8818F018503AA17A9279B359800F025
:1081200030F92898002807DD68468089A18A41181F
:10813000289809186846818130992598814200D98C
:108140003EE7A07F80071FD56A462C9810802168E3
:108150000820085E10AA0A21515EC20F1018CA0F2B
:1081600051184010491040186A46D18901AB401897
:10817000508091899180D08010AA908F10816A469A
:1081800012A9359800F002F9A07FC00721D06946F6
:108190002C9808802068C989028905E0FF1F00002B
:1081A000FFFF00009000002040898918091A1598E7
:1081B0000D22825601AB881A694648808A898A80D6
:1081C000C88010A9888F08816A4612A9359800F0E6
:1081D000DDF8617F00200090169D01911422701936
:1081E000A25E07462D9B1599F9F732FE169D69464A
:1081F000401916903798008888812A98022802D062
:10820000032816D029E0607F009016981423411BA4
:10821000E35E3846159A07F0E9FE07463798FFF700
:10822000E6F9C01B6946C20F89891018401008186A
:1082300011E0607F009016981423411BE35E3846DE
:10824000159A07F0D3FE07463798FFF7D0F969462D
:108250008989C01B401869468881C98924980622EB
:10826000081800B26946C881359989688A5E9042CB
:1082700003DC705D002800D094E639B0F0BD00004A
:1082800038B50446202103F0BEFFFF20A076FFF79B
:1082900081FA009068460088A0810A4820600A4858
:1082A0006060A060FFF776FA009068460088E08181
:1082B000052006F09FFF009068460088208200207D
:1082C000E07638BD68560108FFFF0000036C002B04
:1082D00000D018477047436C002B00D018477047F8
:1082E000F8B50546C06B16460F46002827D0E86C47
:1082F00003F00CFE04001DD0E96C03F084FFF9F7D5
:1083000051FD296821626968E161A968A16100687D
:108310000822007C4006C10F242001553946204622
:10832000F7F7A0FFEB6B3246214628469847050039
:1083300001D003E0FEE7204603F070FE2846F8BDBA
:1083400070B50C46054601F09FFF206A2860E06981
:108350006860A069A860F9F725FD016840220869F6
:1083600090432422125DD207520E10430861AA6C7A
:10837000002A02D0214628469047204603F04EFEB0
:1083800070BD30B4046AA44630BC604730B44C8839
:10839000002C06D00C7A022C03D9446AA44630BCC7
:1083A000604730BC704738B504460A2103F02BFF04
:1083B00001206080FF202072684600883F2140092C
:1083C0004001490188434105490D6846018088B252
:1083D000009068460088009068460088208038BD7C
:1083E00010B504460A4A0020C300D358002B04D01D
:1083F000401CC0B21028F7D301E0102802D300209F
:10840000C04310BDC300D4509A18516010BD000085
:10841000E8150020FFB585B00E9D0821695E06981D
:108420001646471A0A22AA5E0C202946285E1031F9
:1084300003911C462C31B31A0191B4285BDA0E214A
:10844000695EB4297EDA00287CD00029FCD08842FD
:1084500078DDB24259DC6A6DAD6A5A435B1C5D43FC
:10846000AB120546FF3D9212103D582D01D8002B4E
:1084700009DB451E592D01D8002B04DB5B38B328DE
:1084800002D2002B00DD00230846FF3810385828A0
:1084900001D8002B09DB481E592801D8002B04DB2A
:1084A0005B39B32902D2002B00DD0023D01A401023
:1084B00018180125C71BA74200DD2746002F0DDD38
:1084C000039800903BB232460699059800F094F963
:1084D000050003D13946059803F095FEA74200DD5B
:1084E0002746002F00DA002701985CE0B54278D1DA
:1084F000284609B0F0BDB42868DD0E21695EB429B4
:1085000064DD884262DDB24201DA0120F1E76A6D82
:10851000AD6A5A435B1C5D43AB120546FF3D9212A8
:10852000103D582D01D8002B09DB451E592D01D8CF
:10853000002B04DB5B38B32802D2002B00DD0023C4
:10854000084600E042E0FF381038582801D8002BD8
:1085500009DB481E592801D8002B04DB5B39B329FD
:1085600002D2002B00DD0023D01A4010181801257C
:10857000C71BA74200DD2746002F0DDD01980090A4
:108580003BB232460699059800F036F9050003D152
:108590003946059803F037FEA74200DD2746002F35
:1085A00000DA0027039800900698E41BC01901B276
:1085B000059823B2C0190746324600F01DF906009F
:1085C00094D12146384603F01EFE8FE7012702971B
:1085D000B42807D0002808D0B42809DAB24209DC50
:1085E0000AE049E0B24210DC04E0B24202DC0CE0F6
:1085F000B24201DC032708E003980090234632468C
:108600000699059800F0F8F807460E20285EB42871
:1086100008D000280DD0B4281848285E10DAB042DF
:1086200004DC0FE00A20285EB04206DD0320029041
:1086300003E00A20285EB042F8DD002F17D00EE0DC
:10864000B042F3DD01980090234632460699059822
:1086500000F0D2F80290002F09D0002807D0032F95
:1086600002D0012F05D007E00298032804D1002092
:108670003FE702980128FBD002203AE70A000000F9
:10868000FFB5054681B0FF2068300A9C1746002BD5
:1086900001DA002302E0834200DD0346002C01DA08
:1086A000002402E0844200DD04462846FF224030D8
:1086B00069329C4202DAD11A091903E0E11A002951
:1086C00000DC191B0185AB81EC81029828816F8148
:1086D0001648286001202871FF206A30834200D3A9
:1086E000FEE7B42B01D2002000E00120002C01DBCA
:1086F000934200DDFEE7B42C05D32146B439B429FA
:1087000001D2002600E00126009028463A461030AB
:10871000029900F0C5F8284623463A4600963C30B8
:10872000029900F0BDF805B0F0BD00001584000806
:10873000FFB581B01E4600250B4C0BE0009007688A
:1087400001A807C83346B847002809D0022800D13D
:108750000125083420680028F0D1002D02D0022025
:1087600005B0F0BD0120FBE7E815002010B5017948
:10877000022905D0052902D1806803F04FFC10BD05
:10878000044640690028FAD00169002904DA4068EB
:1087900003F044FC6069F0E74169491E416110BD86
:1087A00070B5134D060008D00024E00029580029B8
:1087B00017D00879022805D002E02868002800D0E8
:1087C000012070BD887C0B4AC0078A5E304603D00A
:1087D0000831F8F7D4FC02E00831F8F764FC00280F
:1087E000EED0641CE4B2102CDFD3002070BD00007A
:1087F000E815002010000000F8B5069CA58A266A3E
:10880000521B658A12B2491B28252D5D09B2002E24
:1088100005D0ED07009440D0FEF724FCF8BDED072D
:1088200010D0207C810725D08107890F012921D014
:10883000022901D1511C1DD4C043800725D1002A33
:1088400018DC22E0227C9407A40F022C12D0D5431E
:10885000AD070FD0012C01D100290BDC920707D006
:10886000D94212D449420ED50021002B0DDD0EE075
:10887000D94201D50120F8BD4A4206D49A420ADA0B
:10888000991A801805E0994201DB0020F8BD994251
:1088900001DA03F0B8FC0220F8BDFEF786FCF8BD53
:1088A000FFB583B01C4616460F46B42B01DDB43C21
:1088B00024B220465A3000B207F072FA4011C519AE
:1088C000204607F06DFA4011801900B20C99019111
:1088D00000902BB232463946039800F003F807B0F7
:1088E000F0BD0000FFB583B00E46154604462C21AE
:1088F0000C9F03F088FCBD4206D10D98032803D1DC
:108900006D1E7F1E2DB23FB2BD4205DD0698069654
:10891000064638462F460546268165810698A08181
:10892000E7810D98207401906682A5820698801BCD
:10893000002801DD014601E00699711A7E1B002E18
:1089400001DD324600E0EA1B27462037914203DD75
:108950003D7A01210D4302E0397A4D086D003D72E8
:108960000021E1612E4A2260A16121710090E80797
:1089700017D00098002807D0014601200005F7F71E
:1089800031FD70438012E061002E08D00120314695
:108990000005F7F727FD009948438012A061E069C0
:1089A00016E0002E08D0012031460005F7F71AFD29
:1089B000009948438012A0610098002807D0014622
:1089C00001200005F7F70EFD70438012E061A069F9
:1089D00020620198FD21800700280CD001988207B1
:1089E000920F0220012A08D0022A11D0019AD24304
:1089F000920711D003E00D4000E005433D72216A6B
:108A000088106062002901DA4042606207B0F0BD60
:108A1000226A002AF1DCEEE7226A002AEDDDEAE7AD
:108A2000F9870008FFB58BB014980F46807C10259D
:108A3000C007C00F0A9014981C460146455F1646B1
:108A4000083106A8FEF79EFD0A98694600289A4854
:108A5000085E33D0B04256DC1E20085EB04252DBC6
:108A60001820085E4119B94206DC6B461C229A5E4A
:108A70003919521B91420BDD6A461A21515E4A197F
:108A8000B24244DC6B461E229A5E521BB2423EDB6F
:108A90000A99002919D0C01B00D50020A04234DC5F
:108AA0001C21595EC91B091A491C4218A24200DD4B
:108AB000211A002929DB0B9A1018FAE0B04214DCC5
:108AC0001E20085EB04210DBCAE7C61BA6420CDCC3
:108AD000002E03DB31460B9803F095FB69461C2002
:108AE000085EC51B6D1C002D02DC00200FB0F0BD20
:108AF000A54204DA0B98611B401903F084FB002E99
:108B000003D1A54201D10120F0E70220EEE76A4639
:108B1000928BC31B101A401C00B284466A46D08B4D
:108B2000401A401C02B2701A00B2A84202DA281A97
:108B3000401E01E0511B401A149900B249694000DF
:108B4000CE68821CB25A375AD21B6F46BA828A68E4
:108B5000125A3A84305A49684018099060461818E9
:108B6000401B801806B25819801A401E05B20A9898
:108B7000002801D0002776E0002722E0C11B0998D9
:108B800008182038C07F0490F019089009D4A0423A
:108B900007DA0B99095C049807F05AFE0B9A0899BA
:108BA0005054E81B0890002809D4A04207DA0B991A
:108BB000095C049807F04CFE0B9A089950547F1CEE
:108BC0003FB269461420085E8742D7DBF019A04205
:108BD00001DA014600E02146002901DA002002E026
:108BE000A04200DB204600B20B9A211A101803F0B5
:108BF0000AFB69461420085E281A411CA14201DACA
:108C00000A4600E02246002A01DA002402E0A142DE
:108C100000DA0C4621B20B984BE0C11B09980818EA
:108C20002038C07FFF21081A0390F01908900AD459
:108C3000A04208DA01460B98415C039807F008FE51
:108C40000B9A08995054E81B0890002809D4A042B8
:108C500007DA0B99095C039807F0FAFD0B9A08995B
:108C600050547F1C3FB269461420085E8742D4DB13
:108C7000681CA04201DA691C00E02146002901DAE3
:108C8000002504E0A04201DA6D1C00E025462AB26E
:108C9000B01AA11A884201DA034600E00B46002B05
:108CA00001DA002002E0884200DB084601B20B989E
:108CB000801803F0A8FA28E71A000000F8B5154656
:108CC000064688880A881C46801A401C02B2C8885A
:108CD0004B88C01A401C00B2824200DA1046401095
:108CE000A84200DA0546002D00DA0025304608309B
:108CF000FEF748FC3582B47435483060022000230A
:108D00003071002D13D0334900201C2242435418E7
:108D10001822A25EAA421BD11C225043401841696E
:108D2000491C41610269102D03DA012102E07361DF
:108D3000F8BD291153187D21C9008B4205DA102D89
:108D400001DA012100E02911511801617061F8BDBB
:108D5000401C0428D9D3002422461C20114641433C
:108D60001C4808184169002906D1002C03D001696C
:108D70002769B94200DA0446521C042AEDD3002CBC
:108D800007D060692361401C6061102D0DDA01205D
:108D90000CE01C2003F0BAF8040005D01C2103F0FD
:108DA00032FA0020C0430CE0FEE7281119187D209C
:108DB000C000814205DA102D01DA012000E02811FF
:108DC00018182061204629467461F9F795FEF8BD10
:108DD000258A000878150020F0B50025084E0746C2
:108DE0002C46E00081194968B94203D13558204624
:108DF00000F008F8641CE4B2102CF2D32846F0BD51
:108E0000E81500200021421C06D0C20003480023C0
:108E1000815883501018436008467047E8150020B9
:108E200030B4D38854881B1B5B1C1BB2012B09DB9D
:108E3000938814881B1B5B1C1BB2012B02DB03698C
:108E400030BC184730BC7047F8B50446382103F0F1
:108E5000DAF9FEF7BDFD694600900888A080FEF7AC
:108E6000B7FD694600900888A61CE080FEF79CFCD0
:108E70006946009008883081FF2525730220A07381
:108E8000FEF792FC694600900888B083FEF78CFCE0
:108E9000009069460988A185074961612046E5700F
:108EA0002030A576857285708575C178C122114004
:108EB0001E31C170F8BD000068560108FFB5CFB083
:108EC000087B589F599E14460D4602287ED90220E1
:108ED000285E00287AD0B74278D01B9052990AB207
:108EE0001C92884200DD1B9201A8FFF7ADFF687B52
:108EF00069468007800F8871A868002808D0002183
:108F00006846C171A8680590297B6846817704E0AE
:108F1000297B6846C17129880181218852980A1AE3
:108F200010A8028361885298091A10A84183529BA5
:108F300020888C465B1EC11810A8818360888E46ED
:108F4000C31810A8C3830284604610A948847146E0
:108F500010A88184C3846888121810A802849646D9
:108F60006A886046801802B210A8428468889446D5
:108F7000091A10A8818468887246181A03B210A8CA
:108F8000C3840020C0431A9000201D90881A401C02
:108F900000B2002812DD6046181A401C00B20028FA
:108FA0000CDD01239D4A18A93DA8FFF787FE01208B
:108FB0001D9000213DA8FFF713FA1A900023974A4D
:108FC00016A943A8FFF77AFE002100E029E043A894
:108FD000FFF706FA1E903846FF306930B04206D0DF
:108FE0003146FF31FF20693169308F421ED18B48F5
:108FF0006946888016AA01A94F98FFF711FF1E98AD
:10900000FFF700FF1A98401C02D01A98FFF7FAFEEB
:1090100043A8FFF7ABFB1D98002802D03DA8FFF73F
:10902000A5FB53B0F0BDFF3F693FBFB28742FAD204
:1090300002E0FF3E693EB6B2FF2069308642F8D2B8
:1090400030B22190009002220021A25E615E3BB20C
:1090500022A82093FFF714FB002122A8FFF7C0F9F4
:109060001F90BE4204D9FF20F11B6930401A00E076
:10907000B81B4F993C28896800912DDD52980A2829
:109080002AD90F9410A81C990180478086805A2104
:109090003846F7F799F98107890F10A8C1805A213E
:1090A0003046F7F791F98107890F10A801811B99C4
:1090B000418101A8139016A814904F9815900FA8FD
:1090C000FBF71BFF0FA8FBF7DBFF0FA8FCF7A0F8CF
:1090D0000FA8FCF785F904E016AA01A94F98FFF73D
:1090E0009FFE22A8FFF742FB43A8FFF73FFB1D9816
:1090F000002802D03DA8FFF739FB1F98FFF782FE3A
:109100001E98FFF77FFE1A98401C02D01A98FFF7AE
:1091100079FE687B400784D51B980FABC2B21C99BF
:109120002098FDF7D5FD6846808F21880FAA411849
:109130006846818710A800882188411810A80180FE
:109140006846C08F618841186846C18710A840886A
:109150006188411810A8418012A80099F7F77BFF99
:1091600012AD002817D000232C4A0FA949A8FFF7F9
:10917000A5FD002149A8FFF733F906464F9816AA26
:10918000856001A94F98FFF74BFE3046FFF73AFE86
:1091900049A8FFF7EBFA1B980FABC2B21C992198B4
:1091A000FDF796FD6846808F21880FAA4118684612
:1091B000818710A800882188411810A8018068467E
:1091C000C08F618841186846C18710A840886188AF
:1091D000411810A8418012A80099F7F73CFF002819
:1091E00017D000230D4A0FA949A8FFF767FD0021FA
:1091F00049A8FFF7F5F804464F9816AA856001A91B
:109200004F98FFF70DFE2046FFF7FCFD49A8FFF73A
:10921000ADFA4F990098886003E70000FF7F0000D7
:1092200070B514460D460646FAF771F822462946EF
:109230003046FAF743FA70BD7CB50446087E0D4609
:1092400002280FD9A26868462968F7F704FF0028AA
:1092500008D0616B002901D020468847626D2946FD
:10926000204690477CBDF0B5CD688BB00C460646D5
:10927000002D02D0207C002872D0207C012800D153
:109280000025706881880088081A401C00B2079089
:10929000B26805A82168F7F7DEFE002860D0F8F76D
:1092A00081FD04903068099004980068C169002924
:1092B0002BD1017C490611D471686F461622022316
:1092C000BA5ECB5ED21A079B5A431423FB5E00277B
:1092D000CF5FD91B51184A00099914E06F46162335
:1092E000FB5E72680227D75F0999DB1B079F7B43F0
:1092F0005F00DB1959186F461423FB5E0027D75F08
:10930000DA1B5300D218511809916168089100299D
:1093100019D0216800228B888A5E6F469B1A5B1CDD
:109320001BB20A931623FB5E0227CF5FD91B0A9B51
:109330006F4659431423FB5E9A1A89184A0008990C
:109340005118089101E000210A91002D28D0007CDD
:10935000000710D46069FEF736F90146002008E0E6
:109360003BE02A5C802A01D9FF2200E000222A5437
:10937000401C8842F5DB606900218288415E16232B
:10938000521A521C17B26A46D35E0222825E981AA3
:109390006A461423D35E7843591A4919451800E0E8
:1093A000002770684188008849420AB2404201B2F1
:1093B00005A8FEF735F904980068C069002818D0A0
:1093C000606800280BD00A98217E6A46A3C205A9CE
:1093D000089B079A099807F0B6F90BB0F0BD207EFC
:1093E0006946A1C1A36805A9079A0998FDF7D8F9AC
:1093F000F3E7607E00280FD061680029217E23D02A
:1094000001AA0490A2C20A98009005A9089B079A95
:10941000099806F04BFFE0E760680028207E0AD03C
:109420000A99009101AAA1C205A9089B079A099867
:1094300006F0FEFFD1E76946A1C1A36805A9079A16
:109440000998FDF70BF8C8E76A460390A2C2A36823
:1094500005A9079A0998FCF75BFFBEE7FEB51D4614
:1094600002242C5F0A9F2646564376007118002678
:10947000AE5F0998B446760076180221795E089BA3
:1094800041434900C9180023FB5E5B005F18A988AF
:109490006346C91A491C09B24900029151004000B3
:1094A000019100900AE039463046029A02F0F2FD3E
:1094B000019886190098C719641C24B20620285EFA
:1094C000A042F0DAFEBD0000FFB59FB01F980D4628
:1094D000816814461BA8FEF75EF81BA8FFF760F929
:1094E00017902888002803D16988C81FF93801D04F
:1094F000012100E0002116911C2106A802F083FE44
:10950000E97A08A80174287B00270107090F08A839
:1095100041740DA806901699179802260843002852
:1095200028D12898042804D00E2808D014281ED04A
:1095300020E0A87A00281DD12298079010E01F98FB
:10954000214682686846F7F786FD00280DD02298EC
:10955000099007970B9429896846018408A8067228
:10956000069406A91F98FFF767FE23B0F0BDA87AFE
:10957000002833D01F986B468168088898868A88AF
:1095800084461A871F9880684188D9861F9880680A
:10959000C0885887A3882788401ADB1B5B1C1BB236
:1095A0001293E3886788401C00B204906046DB1B7E
:1095B000101A5B1C401C1BB200B215930F90F8F7F9
:1095C000F1FBFEF705FB07460DA8FDF7FCFF014682
:1095D0000F980290B94216D8049F19E0A0882188FC
:1095E0006288401AE188401C891A491C0AB200B2FC
:1095F0002299400050430818069409900B94079153
:1096000008A80672ADE738460F99F6F7DDFE074663
:10961000029878431390400002F0A6FC1190139832
:1096200002F0A2FC109009900DA80B90022108A84E
:1096300001721198079068463A21415E1491C08EDC
:109640007F1EC1196846189741872898042806D1BB
:109650002888002803D16988C81FF93801D0022062
:1096600000E0012008A90872B1E00DA91DA8FDF7CE
:1096700092FF6088404202B22088404201B21DA899
:10968000FDF7CEFF16980028109810D02899039166
:10969000059012991598119A019104920B46009029
:1096A00002951DA9229A1F9800F0D2FD0DE0119994
:1096B00003910490289A1298029201950090024614
:1096C0001DA8159B2299F9F744FCA87A022848D9CD
:1096D000A9686A4600911188CB0A434313804A0562
:1096E000930EC90643436A46C90E53804143918095
:1096F000FF21081A002131E0119A4B009A18944674
:1097000012886F463A813E88D30A4343F318374E96
:109710007F887343DB0E5605DB02760D3343560517
:10972000B60E4643BE19324FD2067E433F277F0115
:10973000B60EBB4376011E436F46BB88D20E424332
:109740009A182A4B5A437309D20E5B011A433A8185
:1097500092B2029262463B891380491C139A91424D
:10976000CAD31798002821D068463626865F109FF6
:1097700017E008463421415E324638460F9BFEF71B
:10978000D7FF002802D0022804D006E038460F99FF
:1097900002F039FD022008A908720F983F18761CC4
:1097A00036B269463A20085EB042E2DA06A91F984E
:1097B000FFF742FD6946488F401CC886189940183B
:1097C00002B269464A871498824200DD488768469B
:1097D0003621415E1498814200DC46E7109802F081
:1097E0000BFC119802F008FCBFE60000100808000E
:1097F0000804040010B50C465821204602F003FD71
:1098000010486061104820611048206310482062B1
:109810001048A061104860621048A0621048E062E1
:10982000104860631048A0631048E063104820644B
:10983000104860641048A064104860652C20E06403
:1098400010BD0000BD8E0008C19F000821920008D5
:10985000819A0008C99400088D9B00082D9D00087E
:10986000F79F00084FA200085D940008699900085E
:1098700081980008CD980008759A00086792000842
:10988000F8B517460C460646F8F78CFA0546F80771
:1098900040270028A06A0CD041004908606902F006
:1098A000B2FCA06A79060843A062286801693943BE
:1098B00005E041004908A16228680169B9430161D6
:1098C0006069083411C63460F8BD0000FEB5054675
:1098D000006802900C460098E02188430090686878
:1098E0001646818800881F4A081A401C4005C10A94
:1098F00000981040084300906868C1884088081AA2
:109900000099401CC9024005C90A01434809009159
:10991000A16A4001002901DA052100E00421084381
:109920000090206A2860E0696860A069A860F8F784
:1099300039FA0168402208696B4690432422125D7F
:10994000D207520E1043086122460832314628469B
:10995000FEF7A6F9284600F097FC684601F02CF9BE
:10996000FEBD0000FF03E0FFF8B5064615460C46B5
:10997000D00701D00020F8BDEF07A80749D5A06A9D
:109980000321C00FC007490341182046A162FDF71B
:109990001AFEA16A40004A005208824205D9C90F46
:1099A000C907400040080143A162A06A4000400886
:1099B00002F0ACFA2146606100280ED1A06A0321B2
:1099C000C00FC00789024018A0624000400802F0A2
:1099D0009DFA214660610028CDD0084606C8016086
:1099E000E2606188E181A1892089081A401C05B2E2
:1099F00068002918A06A40004008F6F7F3FC2082AE
:109A0000A06A294640004008F6F7ECFC401060824E
:109A10002EE0084606C801600838E260FDF7D3FD75
:109A200080004108A06AC00FC0070843A062400040
:109A3000400802F06BFA6061A16A4900490802F02F
:109A4000E2FBA06A400040083843A0626069002839
:109A500091D03060204608307060B060F8F7A2F90D
:109A60000068402201699143EA07520E11430161E7
:109A70002046F8BD10B5486902F0D0FA10BD0000CC
:109A8000FFB51C4697B015460E46086800232246CF
:109A90000FA900F087FC002841D010A88188002978
:109AA0003BD04788002F38D010AA2888D288801849
:109AB00000B210AA90813268138952899A1A6B8871
:109AC000C519D218531A10AA128900279A1A13B26C
:109AD00010AAD381179A9268D75FBD421DDB042577
:109AE000555FA84219DC58180221515E884214DBE8
:109AF0000620105E834210DC21460F9800F04DFCDA
:109B000000280AD00F99097B890706D100900FAB76
:109B100013AA31461798FAF7F7FB1BB0F0BD202CBB
:109B2000FBD318488442F8D017488442F5D010A8D7
:109B30002988C0886A88081801B210A800891018FE
:109B400002B210A88088801800B2009010A8408847
:109B5000401803B214A8FDF770FD01A8FFF774F9CF
:109B600002216846C17108A88173817668468177B1
:109B7000B189418401218184179814AA036901A93C
:109B80009847CAE7FFF800000C200000FFB50E461A
:109B90000221715E95B01C46154600297ED0307AB0
:109BA00002287BD900220020AA5E205E824205D1D5
:109BB00002230227EB5EE75FBB426FD0824200DAEE
:109BC0001046CA0F51184910401A694608810022F0
:109BD00000200221AA5E205E715E824200DD1046F6
:109BE000CA0F511849104018694688810222022084
:109BF0000221AA5E205E715E824200DA1046CA0F20
:109C000051184910401A6946488102220220022157
:109C1000AA5E205E715E824200DD1046CA0F5118B6
:109C2000491040186946C881159802A982680846FB
:109C3000F7F711FA002874D0159802A980681290DD
:109C40001598816002200221285E615E884206D15B
:109C500023462A4631461598FAF7AAFC0EE0002062
:109C60000021285E615E2346884215982A463146C7
:109C700002D1FAF701FF01E0FAF752FD707A01070D
:109C800001D440074AD504A8FFF7DEF831886846BA
:109C9000818225490182317AC17400E041E00220CD
:109CA000305E4710C007C017401C1390707A400701
:109CB00018D528886A46C11B684601806888C11B80
:109CC000684641802888C1191398091A684681801E
:109CD0006888C1191398091A6846C18004A91598A3
:109CE000FFF79EF8707A000718D520886A46C11BD6
:109CF000684601806088C11B684641802088C11980
:109D00001398091A684681806088C1191398091A46
:109D10006846C18004A91598FFF782F81599129832
:109D2000886019B0F0BD0000FF7F0000FFB595B05E
:109D30001F461646032B7DD3002E7BD0B80005901E
:109D400002F012F9050075D0308828800024708850
:109D5000688020467F1E16E08100725E8919042308
:109D6000CB5E9A4205D1022206238A5ECB5E9A42DE
:109D700007D0A20052190B8813804988641C5180B7
:109D8000A4B2401C80B2B842E6DB059800228119DB
:109D9000084640383C23B25EC35E9A4205D1022297
:109DA0003E23B25EC35E9A4208D0A000091F40194C
:109DB0000A8802804988641C4180A4B2032C41D3E4
:109DC0007E4903C906900791002024E06A461821C5
:109DD000515E8200AB5E994200DB19466B461983E7
:109DE0001A269E5F53190221595E8E4200DA3146CF
:109DF0006E4671831C21715EAA5E914200DC1146A1
:109E0000B1831E210222715E9A5E914200DC1146EE
:109E1000401CF18380B2A042D8D3159806A982686D
:109E200011A8F7F718F900280CD0159811A9806827
:109E30000D9000E009E01598002681600221695E1E
:109E400001200EE0284602F0D7F819B0F0BD8200DC
:109E5000531902229A5E8A4201DA114606B2401C68
:109E600080B2A042F3D320462C21484302F07CF874
:109E70000590039000200C9610960E90711E00D550
:109E80006118621E701C0A92904200DD0020890059
:109E9000B3006F5AEA5A8000BE1A2F5A5B195B88CA
:109EA0004919401949884088C91AC01ABA1A36B2E5
:109EB00012B209B200B20023514370430F938142A2
:109EC00070DA01200F9002E00F9800286AD00C9EF3
:109ED0000A98761C864200DD0026109F7F1E00D562
:109EE000E719B000844641190220085E0C9902224D
:109EF00089004B199A5E904219DB904213D0634659
:109F0000EB5E695E9C468B420DD00123019300906D
:109F100063460398FEF7E6FC05990398FEF760FA9E
:109F200003982C3003900E980C96401C0E900E98BF
:109F3000A04224D0BB0059190220085E10990222C9
:109F400089004E19B25E904216DB904210D0EB5E53
:109F5000695E8B420CD00026009001960398FEF7B4
:109F6000C1FC05990398FEF73BFA03982C30039047
:109F70000E981097401C0E900E98A042A4D306AAEB
:109F800016991598FEF74CFF0598FEF725FF0598E2
:109F900002F032F8284602F02FF815990D988860E3
:109FA00053E7FFE70C9E761E00D5A619109F0A986E
:109FB0007F1C874295DD002793E7000038210108C8
:109FC00070B514460D460646FBF728FB2246294687
:109FD0003046F9F79CF9224629463046F9F76EFBE0
:109FE000224629463046F9F755FC22462946304696
:109FF000FAF722FF70BDFFB5A1B02C9F0020385E9C
:10A000000D4640420F90012079880004F6F7DCF9F4
:10A010000E90786812900A210F98F6F7E3F9064639
:10A02000401C02900A200F9970430C1A30B205F0C0
:10A03000B7FE0590029800B205F0B2FE5A360490C1
:10A0400030B205F0ADFE039002985A3000B205F030
:10A05000A7FE02900A20061B05983146414304984A
:10A06000604308180A21F6F7BDF90C9003980A21FD
:10A070004643029860433018F6F7B4F90D900C98F7
:10A08000082140110C900D9840110D9010A8415ED0
:10A090000802109010A80A21415E08021190A888B9
:10A0A0002988401A401C04B2E8886988401A401C7C
:10A0B00000B20026199052E016A800900220285EF7
:10A0C00000218219695E15AB08A807F0DCFD18A80D
:10A0D00000900220285E04218219695E17AB08A84F
:10A0E00007F0D1FD179915980290091A189A169839
:10A0F0000190101A049000200090012C09DD080244
:10A10000611EF6F76FF900900498611E0002F6F7E1
:10A1100069F9029980318E46019980318C46397DEA
:10A12000C9072D9920D02F9B2E9A05920791009A4E
:10A130000693634671460193009103900292049442
:10A140002B9B2A9A24992398F8F7A7F82E98610058
:10A1500008182E902F980019761C36B22F90199857
:10A160008642A9DB25B0F0BD04295BD0052915D0B6
:10A17000062957D01429E9D12E9A2F9B06930592D0
:10A1800003900494614670466B46009A07C32B9B6C
:10A190002A9A2499239806F07DFFD7E723992091E6
:10A1A000249906912A9905912B991A90009B2E9833
:10A1B00002931F9004912F98714603901D910020E7
:10A1C0002DE002991D9A41430B129B181A9A1912FD
:10A1D0004243121262441212002907DB069B994285
:10A1E00004DA002A02DB059B9A4201DB002312E01D
:10A1F000209B9E46049B5A4352185300D218734624
:10A20000D1184B780A788E461B02D1181F9A43004A
:10A21000D15271468B78039A1354401C00B2A0426D
:10A22000CFDB93E70A462F9B2E9907920591009961
:10A230000693634672460193009202910390049440
:10A240002B9B2A9A2499239806F061FF7EE770479A
:10A25000FFB587B09C469646129F139E149D109B97
:10A26000119A159900280ED0C46A002C09D00093C9
:10A2700003960192059102970495634672460899E8
:10A28000A0470BB0F0BDFEE7416B002900D00847A6
:10A290007047007A4006400E704740687047017A68
:10A2A00015290BD0142909D0162907D0182905D053
:10A2B000172903D0192901D0002070470069704781
:10A2C000017A01291FD002291DD003291BD004299E
:10A2D00019D0052917D0062915D0072913D0082928
:10A2E00011D009290FD00A290DD00B290BD00C2928
:10A2F00009D00D2907D00E2905D00F2903D0102928
:10A3000001D00020704700697047006970470068FD
:10A310007047000010B588B0002817D00090019059
:10A320006B461972002004920390187EF9214008B0
:10A3300040000840064C18766068059068466360E7
:10A34000FBF74CFF0599616008B010BD0120FBE7E9
:10A3500000000020027A132A06D102690020105E54
:10A36000884200DD014611807047704710B5092909
:10A3700000D120210469FCF70BFB002806D061689E
:10A38000C0000818618A890B01D0002010BD006848
:10A3900021680003000B081810BD002801D0426896
:10A3A0001047FEE7FFB581B001980C46002811D098
:10A3B000002C10D00026054626602F68214628462E
:10A3C000049B039AB847002809D0A07BC00603D499
:10A3D000256010E0FEE7FEE7002E00D12E466D69F5
:10A3E000002DEAD1002E09D0356821463046049B65
:10A3F000039AA8472660012005B0F0BD03982028E5
:10A4000005D31149884202D01049884202D1002068
:10A41000E08008E001990820085EC10F0818C00319
:10A42000000CE080801CA080002020600199098938
:10A4300021816081A081A07B102100090001401CC6
:10A440000843A0730020D7E7FFF800000C200000AD
:10A45000FFB581B00C46092A42D00026019811466A
:10A460000569FCF795FA07003DD000200090E868E8
:10A4700000280AD004990198FCF78AFA020004D057
:10A4800039460198FCF72AFB00906868F9004018EB
:10A49000298A009A51430A110168090D002E00D043
:10A4A0004900891808310909A18041792181017980
:10A4B000E18006228256628107228256A281A07B19
:10A4C0006A8A0009D2040001120F1043EF221040E3
:10A4D000A073002E01D04800E080012005B0F0BD3F
:10A4E00001262022BAE70020F8E71FB5002808D08F
:10A4F00013460A466946FFF755FF6846808804B050
:10A5000010BDFEE770B50446406800281AD0C26846
:10A51000002A19D0216890470546606840880028C5
:10A520000AD0A068002807D0C068002801D001F038
:10A5300075FDA06801F072FD002020606060A060E1
:10A54000284670BD0B2070BD092070BD10B50446B3
:10A550000748F7F758F908E008680078A04201D1E9
:10A56000086810BD0248F7F752F90100F4D110BD98
:10A570001011002010B50446F5F752FE002808D04F
:10A58000215C2E2907D02F2903D05C2901D0401E41
:10A59000F6D102A010BD2018401C10BD0000000024
:10A5A0004178401C3A2900D1401C7047F8B5174645
:10A5B0000E00054630D03078FFF7C8FF04002DD0DC
:10A5C0006168002902D08847002829D0A0680028A7
:10A5D00028D03046FFF7E4FF0146A3683A462046FC
:10A5E0009847002820D0411C1ED011C56088083D26
:10A5F00000280FD0102001F089FCA860002815D099
:10A60000102101F000FE0020A968C0430860A9687D
:10A61000400048600020F8BD0B20F8BD0320F8BDC5
:10A620000120F8BD0920F8BD0C20F8BDFEE77CB57F
:10A630001C4600230546002C00D0236068680028D3
:10A640000BD00669002E0AD001934388002B01AB82
:10A6500007D0284600F010F809E00B207CBD092047
:10A660007CBD00932D6813460A462946B047002C4E
:10A67000F6D0019921607CBDFFB50546806814467F
:10A6800086680268416885B0C068019068680027E4
:10A6900043880293B24249D88E4247D2B01A82B25E
:10A6A000981A891B884200D3084606460198B4428E
:10A6B00007D881182246069801F0ECFC089804603F
:10A6C00069E081183246069801F0E4FC002003900E
:10A6D000029903A88C42009008D90698A31B8219FE
:10A6E000686829680769B847074617E068682968F5
:10A6F0000769029B019AB8470746A868426802604A
:10A700000398A96812184A60A11B814200D208462A
:10A7100082B206980199801901F0BCFC03983018A8
:10A72000A04200D204460898046030E019469C42DA
:10A7300008D908990091066929682346069AB04706
:10A74000074624E00198002807D1084601F0DEFB07
:10A75000A9680028C8601DD001900020039003A8BC
:10A760000090686829680769029B019AB847074604
:10A77000A8680660039AA868B1184160944200D2A4
:10A780002246089802600199069801F083FC002F88
:10A7900001D006E0FEE7A8680899826809685118A8
:10A7A0008160384609B0F0BDF8B546680446002E11
:10A7B0001FD0B569002D1ED073880020002B36D025
:10A7C000002A1AD0012A21D0022A11D1134620686A
:10A7D0000A4601463046A847002809D1606821682A
:10A7E000C3696A469847002802D1A268009991601F
:10A7F000F8BD0B20F8BD0920F8BDA2689160A368E0
:10A800000A461D68A9420CD3596808E0A3689A68F3
:10A8100052189A60A1680B689A4202D349688A422A
:10A82000EAD96068216884690023A047F8BD13460F
:10A8300020680A4601463046A847F8BD70B50C4668
:10A84000817886B06143091215468A4201DC01888D
:10A850000BE0027A910009180B46203B9B7F634373
:10A860001B129D4204DB091F09886846018057E0DE
:10A8700001235AE0990009188978614309128D4231
:10A8800051DC99000E18301F01886846018000983D
:10A89000FDF77CF800903188684681800198FDF7CB
:10A8A00075F8019030462038807FB178604361436D
:10A8B00000120912091A3AD0281A00B20202101A1C
:10A8C000F5F790FDC1B2FF20421A6846037900787F
:10A8D0004B4350431818164B5843C40E6846008A21
:10A8E0004009400104436846437940784B43504354
:10A8F00018180F4B5843800E43013F2040018443FA
:10A9000023436846847980784C4350430849201893
:10A910004843C00EC1025805400D014368460182FC
:10A9200088B206B070BD5B1CDBB29A42A2D8FEE7CB
:10A930000201010010B54168002901DA01F06EFB47
:10A9400010BD0000FEB50546407A17460E4640078A
:10A950002FD0224C2078002803D100F043F80120AA
:10A960002070687A4007400F022818D039463246D6
:10A970002846F8F7EAFA0190002000906A4601A9FB
:10A980001748FCF750FA01280BD03A4631462846C2
:10A99000F7F73AFB009000280BD0002418E031466E
:10A9A000E5E700981E224168D1410222091DD141EC
:10A9B0004160FEBD22462846FFF740FF0290009806
:10A9C00061008068401869460989641C018024B2CE
:10A9D00000980E21415EA142ECDCFEBDC4000020C7
:10A9E0006568000870B5094D0446286801F016FB3B
:10A9F000204601F08BFA2860054D0028A86004D09D
:10AA0000214601F000FC6C6070BDFEE7A80000204C
:10AA1000C400002070B506000C4633D0084600F094
:10AA20007EF83046F6F7EFFE05E00868A04229D030
:10AA30003046F6F7ECFE0100F7D1204602F07DFA31
:10AA4000002809D0A1688968002905D0C96809686B
:10AA5000A14201D100F04CF8A068002802D12046A4
:10AA600001F030FCA06886603046F6F736FF05003E
:10AA700009D030462C60F6F7C6FEA84202D1304617
:10AA800000F036F870BDFEE710B50446064A0749E7
:10AA9000FBF7F9FE6269002A04D0002802D10121E7
:10AAA0002046904710BD00000F1800080718000846
:10AAB00010B50446064A0749FBF7E5FE6269002A1D
:10AAC00004D0002802D100212046904710BD00008C
:10AAD0001918000821180008014800687047000094
:10AAE00008000020002802D0007F8007C00F7047B8
:10AAF00070B50446007F0107CD0F08210843207779
:10AB00004007204602D4FFF7BFFF01E0FFF7D0FF68
:10AB1000207FF7210840E9000843207770BDF8B591
:10AB2000064602F00AFA040040D0E0680027002838
:10AB30002AD00068B04222D1207FC10702D040084D
:10AB4000400020772046F6F75EFEE168884210D18B
:10AB50002046F6F765FEE16888420AD12046FBF7F9
:10AB600097FFE16802460B680F211846FFF7D2FBFA
:10AB700002E02046FFF7BCFFE068002804D0E06850
:10AB80000068B04200D1E7602046F6F73CFE10E0D6
:10AB900028682946B042204609D1F6F7CAFE284661
:10ABA00001F03CFAB068002800D08760F8BDF6F7E5
:10ABB0002EFE0500ECD1F8BD7047014600B500201F
:10ABC0000B00F6F769F90F0A0A0A0A090B090D0FBB
:10ABD00011130D0F11130A00102000BD182000BD25
:10ABE000012000BD022000BD042000BD082000BDE2
:10ABF000014600B5891E00200B00F6F74DF90D083F
:10AC000009090809080808080808080809000120B7
:10AC100000BD01460020032901D0062900D10120F2
:10AC2000704770B54C6A0D46002C14D0287C012862
:10AC300002D12046FFF766FCE068002801D001F051
:10AC4000EDF92069002801D001F0E8F9204601F073
:10AC5000E5F90020686270BD7FB514460D460846D0
:10AC600000F0C9FB2C49002804D001281DD002287F
:10AC700042D03EE02A68D006C00E001F112838D20C
:10AC800020680840D102490D8902084320602968E4
:10AC9000C002490DC00A49050843206029784009CF
:10ACA0004001C906C90E084332E02846FFF762FC9E
:10ACB0001AA1F5F739FB00281BD102222946684664
:10ACC000FFF774FC00280ED103AB0422214668462E
:10ACD000FFF7ADFC05466846FFF714FC002D08D1D0
:10ACE0000398042805D12078C006C00E001F112843
:10ACF0000FD3002004B070BD2068084001218902F4
:10AD00004018C002C00AC9024018400940010B3077
:10AD100020600120EEE70000FF03E0FF62696E00A3
:10AD2000FFB58FB059A000680A9059A000680B9039
:10AD30000E4658A00FC806AC0FC40F98694680682D
:10AD400001908A880020D1B2130A08E04200189CC2
:10AD50008218A154189C1219401C537000B2129A08
:10AD60009042F3DB002003900F98007DC006C00ED8
:10AD7000FFF723FF01218140491E059088B20C9006
:10AD80000F98002440692746C106C90E25460B29A5
:10AD900006D00C2912D00D291FD00E2930D12AE05F
:10ADA000C002400DC01DC4081198F110604347183F
:10ADB0007007400F07210D1A0AA80CE0C002400DD1
:10ADC000C01C84081198B11060434718B007400FA9
:10ADD00006210D1A0BA8039012E0C002400D401C82
:10ADE00044081198711060434718F007400F042180
:10ADF0000D1A06A8EFE7C002440D119860438719A9
:10AE00000F98466A204601F0AFF8029000283BD028
:10AE10000F98007C002811D00022391D3046FFF722
:10AE2000C3FC0023224630460299FFF700FC02993A
:10AE3000059A002008239A1A53B21EE00F98406822
:10AE40008068C119F4E70A780C9CEA4022400F9C04
:10AE5000247DE406E40E0E2C01D0039CA25C440089
:10AE60000619189C3419A270059AAA1A55B2002D19
:10AE700001DA1D46491C401C00B2129A9042E2DBE6
:10AE8000029801F0B9F8012013B0F0BD00FF0000F6
:10AE90000055AAFF00112233445566778899AABB52
:10AEA000CCDDEEFFFFB585B005980C46007DC006F1
:10AEB000C00EFFF782FE01218140491E019088B239
:10AEC00002900598002740693D46C106C90E3E46DE
:10AED000072906D0082912D009291ED00A2932D103
:10AEE00029E0C002400DC01DC7080798E110784353
:10AEF00046186007400F07210D1A083623E0C002EC
:10AF0000400DC01C87080798A11078434618A00779
:10AF1000400F06210D1A103615E0C002400D401CEE
:10AF200047080798611078434618E007400F04214E
:10AF30000D1A403607E0C002470D079801217843FB
:10AF40000019890246180598406A0090384601F0B9
:10AF50000BF8040011D00598007C002810D00022C6
:10AF6000311D0098FFF720FC00233A462146009847
:10AF7000FFF75DFB214600202AE0002009B0F0BD6C
:10AF80000598406880688119F5E70A78029BEA40D5
:10AF90001A40009B5600DB689B191B886E46B381E4
:10AFA00046000E9F8619BB550E9F1B0AF61973703B
:10AFB000009B1B699A5CB270019AAA1A55B2002DC7
:10AFC00004DA019A08239A1A55B2491C401C00B2AF
:10AFD000089A9042D9DB204601F00EF80120CDE717
:10AFE000FEB50646087C0C46012802D0002826D073
:10AFF00029E06068FFF7BEFA6DA1F5F795F9002822
:10B000005ED1022268466168FFF7D0FA0028F7D1C6
:10B01000606A002808D1142000F078FF60620028E0
:10B020000CD0142101F0EFF8606A69460C220B780D
:10B030000370401C491C521EF9D104E0FEE7606811
:10B040008068002871D06169C806C00E0E2816D02D
:10B05000142814D004283CD005283AD0062838D02B
:10B0600007283AD0082838D0092836D00A2834D002
:10B070000B2829D00C2827D00D2825D092E0227C3F
:10B08000002A1ED0CA02520D490D4A4314281CD072
:10B0900001265643304600F039FF050010D0676A9C
:10B0A000002204213846FFF77FFB00233246294661
:10B0B0003846FFF7BCFA002809D0284600F0AEFF5A
:10B0C00074E060688068A0616AE00326E1E7A5613A
:10B0D00066E0207C0028F4D062E0FFF76EFD0127D7
:10B0E0008740606A002808D1142000F00FFF6062DA
:10B0F00000281BD0142101F086F87800656A00F062
:10B1000005FFE860002812D0384600F0FFFE2861F5
:10B1100000280DD0E868002844D0207C012808D001
:10B12000606800248068009038E03AE0FEE7FEE7BF
:10B13000FEE7002204212846FFF736FB002417E033
:10B140000023042269462846FFF771FA6846027810
:10B1500041788078FCF7B2FB0190E8686100411803
:10B1600068468088088068462969C0780855641C4C
:10B17000BC42E5D314E00099A0000A5C461871783F
:10B18000B078FCF79BFB0190E868610040186946C5
:10B19000898801802969F0780855641CBC42EAD38B
:10B1A0000120FEBD21463046FFF73BFD0020FEBDDD
:10B1B00062696E00F0B50C46207D87B01D46C00662
:10B1C0000027C00E0C9B0D991646042816D00528A2
:10B1D00014D0062812D00B283BD00C2839D00D28CB
:10B1E00037D00E2835D007283AD0082838D009287B
:10B1F00036D00A2834D0002007B0F0BD227C012AC6
:10B2000035D105930391616A0191FFF7D6FC07469A
:10B2100060690022C002400D684380197843C11064
:10B22000091D0198FFF7C0FA002500280FD10598E5
:10B23000FC08444302AB2246029503990198FFF7AC
:10B24000F6F9002803D10298844200D101252F4647
:10B250000DE000912A4631462046FFF761FD05E0EA
:10B2600000912A4631462046FFF71CFE0746384625
:10B27000C2E710B50446006800280CD0C268002A56
:10B2800001D021469047207C012804D1606800F05D
:10B29000C5FE0020606010BD10B50548F6F7CCFA79
:10B2A000040004D0142100F0AEFF204610BDFEE7DC
:10B2B00034110020F8B50F4605460421384600F049
:10B2C000A2FF002D05D0284600F095F8002802D0F6
:10B2D00004E00020F8BDA8680028FBD000260A483A
:10B2E000F6F791FA0CE02368002B05D03A46294680
:10B2F00098470646012805D021460348F6F787FA05
:10B300000400F0D13046F8BD34110020FFB50E46E0
:10B3100081B01D460446282100F075FF002E18D08C
:10B32000304600F068F8002802D1B168002910D03A
:10B330006946898921812074E56001280CD0666006
:10B3400000272348F6F75FFA0546204614300090A0
:10B3500033E0002005B0F0BD3046F4F761FF401C3B
:10B3600000F0D4FD6060002803D03146F4F732FFCE
:10B37000E6E7FEE72B68002B1AD06868002817D094
:10B3800031462846009A98470746012810D1256083
:10B390006A6821462846904707460128DAD00421EA
:10B3A000009800F030FF00202062A0616062E06140
:10B3B00029460748F6F72BFA0546002DDAD1207CFE
:10B3C000012802D1606800F029FE3846C2E700007B
:10B3D00034110020FEB505680026AC68089F002CDB
:10B3E00007D0009313460A46014601972846A04716
:10B3F00006463046FEBD0321002806D000780146EF
:10B4000020395F2903D801207047084670478028FB
:10B4100001D3022070470020704700000148806877
:10B42000704700000C00002010B5002804D0014631
:10B430000348F6F7ECF910BD0148F6F7E4F910BD42
:10B4400004110020002806D001680978012903D0E2
:10B45000032901D000207047403000790007000F19
:10B460007047002806D001680978012903D0032914
:10B4700001D000207047006B7047002801D00068A1
:10B480000078704738B5154C2078002824D100F09A
:10B49000DBFDF6F7B7FCF6F721F8F5F72DFDF6F72B
:10B4A00025F8FCF745FCF6F769FBFF2169310C48EC
:10B4B000F6F7BAF95C210B48F6F7B6F9F6F778FC1F
:10B4C000F6F702F90848009068460078112804D081
:10B4D000FEF74BFF0120207038BDFEE7180000206A
:10B4E000F8100020041100204433221170B5002010
:10B4F0000C460D4640344862217AE7221140217201
:10B50000411EE962227AD208D2002272A080E08035
:10B51000A86329636863090CE9632964A862207A37
:10B52000BF21084020720221284601F089F800213D
:10B53000284600F05BFC02A1284600F08FFC70BD9D
:10B54000546578740000000010B50146034800F00F
:10B55000CCFF044601F03AF8204610BD701F0108E8
:10B5600010B508460C4600F00AF84820005D0007B8
:10B5700002D4606A00F052FD0020606210BD70B518
:10B58000054604464035287A400604D5A06A0028BE
:10B5900001D000F043FD287ABF2108402872002026
:10B5A000A06270BDF0B587B00E463C4801F010FCBB
:10B5B000012814D13046FEF76CFE05463046FEF7F2
:10B5C000A6FE04462A2D0CD0132D10D0292D08D00C
:10B5D0002C2D1AD0152D02D13046F9F7F9FA07B003
:10B5E000F0BD00F0D3FB204600F060F9F7E7002142
:10B5F00002F08EFA01460820085EC117890F08186C
:10B6000081103046FEF7A6FEE9E7002102F080FA3D
:10B6100004900021204602F080FA03900021204689
:10B6200002F081FA07464820005D0025C10600D5DA
:10B630000125800601D502200543204601F02CFC9F
:10B640000021204602F087FA1549884204D1608C17
:10B65000000501D4134802E0204601F01DFC0190D2
:10B6600000970295616A05A8039B049A04F05EFCAA
:10B670003046FEF74AFE00216B461422415E9A5E78
:10B68000914200DC1146018002221621825E595E41
:10B690008A4200DD11464180A1E70000701F0108C9
:10B6A000D1270000FF1F0000F3B593B00C005AD063
:10B6B000139800211222019002F0A9F9218810228A
:10B6C000091A684681840021139802F0A0F9618864
:10B6D000091A6846C18405A9139801F096FB1398CE
:10B6E0000025476A6846018B808A2C46081A401C50
:10B6F00000B20C902946139802F00AFA0490002137
:10B70000139802F010FA00900021139802F005FA45
:10B71000079004980821415E002006460D9001988C
:10B720000E914030007AC10600D50126800601D571
:10B73000022006430021139802F00DFA584988426E
:10B7400005D11398408C000501D4042006430198CC
:10B750000021426A139800F0B2FE12900E990098F0
:10B760000818119025E0FEE7002000900196781956
:10B770000C9B079A0499F6F76BFB0419684626227E
:10B78000825E0E990D98401882420CDC454A009466
:10B7900012686946384690470A280DD0385D00285F
:10B7A0000AD1641C08E011990D982546081800B2CA
:10B7B0000D90785D0028D7D1781901900020009075
:10B7C0001298022802D0032814D022E0611B0096B0
:10B7D000079B049A019804F009FC69460A8B898A40
:10B7E000511A491C09B2CA0F5118C20F491010183A
:10B7F00040100BE0611B0096079B049A019804F02F
:10B80000F5FB69460A8B898A511A491C081A00B24D
:10B8100000900020694608730A900C90002C2BD1F0
:10B820002EE00AAB0FAA0EA90198F6F7F9FAF00775
:10B8300007D00A990198415C03A8F6F78BFB002812
:10B840001AD10F9A0E990498FEF74FFE6A462421EA
:10B85000515E009A00B2101881421EDB0A994A1903
:10B86000A2421AD00C9A5219BA5C002A15D0079A33
:10B870000C91801800B200900A984019A042D0D3D1
:10B88000094C0A9922680198904706462268294681
:10B8900038469047801915B0F0BD0C980A90EFE734
:10B8A000D12700008C00002090000020F0B5044655
:10B8B000406A9BB000287DD00020C043206304A9CB
:10B8C000204601F0A2FA6846818A008A081A401CC4
:10B8D00000B201900021204602F01AF9074600212B
:10B8E000204602F020F907900021204602F015F9C9
:10B8F000254640350690287A0026C10600D5012647
:10B90000800601D5022006430021204602F023F9DB
:10B91000FE49884204D1608C000501D4042006430E
:10B92000079902960091616A3A4618A8069B04F0AE
:10B93000FDFA204603F05EF8287A4007400F0228FF
:10B9400004D003287ED001287DD019E200212046B2
:10B9500001F092FF0604360C08D1204601F0BEFA31
:10B96000FCF722F90321F4F73DFD86B206A8FBF7A8
:10B9700049FDE74910A806940183FF202D3013905C
:10B980001590002001906846818A008A2022081ABA
:10B99000401C01B210A8825E914235DA00200E9060
:10B9A0000F90891ADB481091014607902046FBF75B
:10B9B00011FD00E0E7E100210A46002804D0016BF8
:10B9C000403080788007C20F119888420FDD1291B5
:10B9D00010A9887E400840008876002A07D00221FE
:10B9E000084310A9887610990E980E911090304651
:10B9F000109A0E99FBF74CFD1190149006A8FBF7D6
:10BA000057FD0120019005E0C2492046FBF7B2FC3A
:10BA10000020A8806946C88A498A2222401A10A9B3
:10BA2000401C8A5E00B290427EDA019900297BD1E7
:10BA3000821A0820385E0E91101A1090B6480F91A5
:10BA4000014601E028E0D3E007902046FBF7C2FC66
:10BA500000210A46002804D0016B4030807880071E
:10BA6000C20F119888420FDD129110A9887E4008FC
:10BA700040008876002A07D00221084310A9887662
:10BA800010990E980E9110903046109A0E99FBF76F
:10BA9000FFFC11901490A7E020460021642201F0E1
:10BAA000B6FF06460021204601F0E6FE0004000C29
:10BAB000019009D1204601F011FAFCF775F8032135
:10BAC000F4F790FC80B2019006A8FBF79BFC90492C
:10BAD00010A806940183002002906846818A008A9B
:10BAE0002022081A401C01B210A8825E914238DA66
:10BAF00000212022199111463846FEF7F6FC41003C
:10BB0000401810AA2021515E401840421090199907
:10BB1000804807900E910F91109A0198FBF7B8FC9E
:10BB200011907C49204600E02FE0FBF753FC0028F1
:10BB300000D0006B002E04D0306B1290F06B15908B
:10BB400009E01199814206DD129010A8807E41081B
:10BB5000490010A8817606A8FBF7AAFC01200290F4
:10BB600005E06C492046FBF705FC0020A8806846EC
:10BB7000C18A408A081A401C02B210A82221415EE4
:10BB80008A4202DA0298002806D063492046FBF771
:10BB9000F1FB0020E880F3E00822BA5E0020511893
:10BBA00049420E900F9010915B480A4607900E99FB
:10BBB0000198FBF76DFC119057492046FBF70AFCF2
:10BBC000002800D0006B002E04D0306B1290F06B78
:10BBD000159009E01199814206DD129010A8807E2F
:10BBE0004108490010A8817606A8FBF761FCC7E070
:10BBF0006846C18A408A081A401C02B210A8222155
:10BC0000415E8A4209DA0820385E814205DD4349F7
:10BC1000606A09688847032802D80020C043AEE064
:10BC20006946888A098A2E22461A11463846761CA9
:10BC3000FEF75BFC06990822401841004018301AB4
:10BC400069468880C88A498A401A401C00B2694601
:10BC5000C880BA5E079906460A925118F4F7C2FBEB
:10BC60000A9A8A4205DC701A6946C8803989081820
:10BC700002E0701A0799401A6946C88001A9204657
:10BC8000FFF712FD0A90606AF4F7CAFA244A02909C
:10BC90001268606A0A999047224E089006E032685E
:10BCA00008A9606A90470A98401E0A90089802996D
:10BCB000C01C8842F3D80026089F0096606A089945
:10BCC0004018194909688847184A8019C6B212688D
:10BCD00008A9606A9047032E08D808990298814203
:10BCE00004D80098401C00900328E7D9616A2046D8
:10BCF000C919009603910646FFF741FC00990429F3
:10BD000025D9481C00F002F9B06211E0D1270000EB
:10BD1000FFFF00005D15010869150108940000206F
:10BD2000880000208C00002080000020840000207B
:10BD3000002825D0009A039900F0ACF9B26A009966
:10BD400000205054287A40210843287209E0287ABC
:10BD5000BF210840287230462830009A039900F02D
:10BD600099F900202E213B18626A401CD154032807
:10BD7000F9D3616A0020FF1CC8550A98C01CE06214
:10BD8000204602F07AF91BB0F0BD000070B50646FF
:10BD900004464036307A4007400F012823D1E16A3B
:10BDA000481C20D0104A606A1268C91E904701469C
:10BDB000327A0020520601D5A56A06E025462835CC
:10BDC00003E02E5C401C9E54C0B2636A0A189E5C5D
:10BDD000002EF6D12B5C626A081813542046FFF738
:10BDE000CEFB701EE06270BD8800002070B50E466C
:10BDF00005461849FBF7BEFA17492846FBF7BAFA79
:10BE00002C4600204034A080E080022E0CD0032E6F
:10BE10000AD0042E08D0207ADF2108402072400783
:10BE2000400F012804D009E0207A20210843F5E7DB
:10BE3000E86A401C02D02846FFF7A8FF207A710765
:10BE4000C008C000490F084320722846FFF72EFDA6
:10BE500070BD00005D1501086915010870B50E463A
:10BE6000054602F00AF9002E00D16E6A2C46686A77
:10BE70004034B0420CD1217A090709D4F4F7D0F943
:10BE8000411C686A00F0EEF86862002819D1FEE7EC
:10BE9000002806D0217A090703D400F0BFF800215A
:10BEA00069623046F4F7BCF9401C00F02FF8686274
:10BEB00000280AD03146F4F78DF9207AF72108409E
:10BEC00020722846FFF7F2FC70BDFEE710B51C4655
:10BED000029B8A4201DB904207DA8A4201DB8842F8
:10BEE00009DD8A4203DC904201DC184610BD8A421B
:10BEF00003DC884201DB204610BD401A521A1B1B8E
:10BF000058431146F4F76EFA001910BD70B50400DD
:10BF100010D0094D0146686803F0B9FE010007D052
:10BF2000A8680019A860EA68904200D81046E86046
:10BF3000084670BD004870BD5C000020F8B50024C4
:10BF4000084D2646E700E859002805D000F066F8BD
:10BF5000EE51781986718680641CE4B2802CF1D38E
:10BF6000F8BD000078110020F8B505000AD00020C7
:10BF7000C04300221F4C0127D30019198E79F60700
:10BF800002D013E00020F8BD8988A9420ED3A9424F
:10BF900004D1D00000198771E058F8BD002804DBF7
:10BFA000C3001B199B88994200D250B2521CD2B2D6
:10BFB000802AE1D3002804DBC00001198F712058CA
:10BFC000F8BD0020C10009198979C90704D0401CB7
:10BFD000C0B28028F6D3FEE7C600A059294600F07B
:10BFE00041F8002804D031198F718D80A051F8BD1F
:10BFF000FEE7000078110020074A0021CB00D3584B
:10C00000834204D10020C900891888717047491CF7
:10C01000C9B28029F2D3704778110020094910B5C0
:10C0200088420DD000280BD0064C0146606803F012
:10C0300002FEA168814201D9081A00E00020A06038
:10C0400010BD00005C00002010B501210903034869
:10C0500003F0E2FD0249486010BD0000EC00002042
:10C060005C00002010B5002906D0094A904207D193
:10C070000846FFF74BFF10BDFFF7D0FF044810BD87
:10C080000A4601460248406803F013FE10BD000056
:10C090005C00002030B584078D07A40FAD0F034668
:10C0A000A54243D14DE00C781C704C785C708C78C4
:10C0B0009C70CC78DC700C791C714C795C718C793B
:10C0C0009C71CC79DC710C7A1C724C7A5C728C7A23
:10C0D0009C72CC7ADC720C7B1C734C7B5C738C7B0B
:10C0E0009C73CC7BDC730C7C1C744C7C5C748C7CF3
:10C0F0009C74CC7CDC740C7D1C754C7D5C758C7DDB
:10C100009C75CC7DDC750C7E1C764C7E5C768C7EC2
:10C110009C76CC7EDC760C7F1C774C7F5C778C7FAA
:10C120009C77CC7FDC772031203A2033202ABAD884
:10C1300004E00C781C70491C521E5B1C002AF8D1CC
:10C1400030BD002C20D004252C1B05E00D781D707F
:10C15000491C521E5B1C641E002C15D0002AF5D110
:10C1600012E00C681C604C685C608C689C60CC6859
:10C17000DC600C691C614C695C618C699C61CC69F8
:10C180002031203ADC612033202AEAD802E010C9AD
:10C19000121F10C3042AFAD804E00C781C70491C42
:10C1A000521E5B1C002AF8D130BD10B583079B0FCF
:10C1B0000AD00424E31A03E00170401C521E5B1EE7
:10C1C000002B01D0002AF7D10B025B180C041B19BD
:10C1D0000C061B1909E0036043608360C3600361C0
:10C1E00043618361C3612030203A202AF3D801E003
:10C1F00008C0121F042AFBD802E00170401C521E26
:10C20000002AFAD110BD830710B59B0F0022002B26
:10C2100015D00424E31A03E00270401C491E5B1E83
:10C22000002B0CD00029F7D110BD02604260826063
:10C23000C260026142618261C261203020392029DE
:10C24000F3D801E004C0091F0429FBD802E0027002
:10C25000401C491E0029FAD110BD820710B5920F6B
:10C26000FF23002A0BD00424A21A03E00370401C11
:10C27000491E521E002A02D00029F7D110BD00220B
:10C28000D24309E0026042608260C26002614261A2
:10C290008261C261203020392029F3D801E004C036
:10C2A000091F0429FBD802E00370401C491E002925
:10C2B000FAD110BD10B5028C11438A4201D002F0B0
:10C2C0007DFE10BD10B504468068002814D10B48CF
:10C2D0004168491C41601C20FFF718FEA06000283F
:10C2E0000BD01C21FFF78FFFA1680F204876A068B4
:10C2F0000322017E1143017610BDFEE718000020E5
:10C30000FEB50E460546012101F0F0FC00284ED195
:10C31000284600F021FE044600F0E0FD0746FBF74A
:10C320007FFCA0420ED03846FBF783FCA04209D028
:10C330003846FBF76CFCA04204D03846FBF75EFCA5
:10C34000A04234D10124E4042146284601F0D5FC62
:10C35000002820D12846F5F720FB0746294614314E
:10C360006846FBF7F4F8684600886A46C11B6846D1
:10C3700001804088C11B684641808088C119684699
:10C380008180C088C1196846C18031460846F4F7EB
:10C3900062FE00280CD0002301223146284601F01D
:10C3A000ECFB1DE0012101F0A1FC002801D00020E0
:10C3B000FEBD2146284601F0A0FC002810D1A96945
:10C3C000686901910090002301226946284601F026
:10C3D000D4FB31466A460846F4F73DFE0028E7D014
:10C3E000284600F0B5FD0500DCD10120FEBDF8B502
:10C3F0000E460746002501F074FB040035D0314697
:10C40000384601F062FB02282FD9E00F00194410D2
:10C4100031463846641C01F05EFB001900B2009002
:10C420003146384601F045FB04463146384601F0B6
:10C4300046FB002C01DD214600E06142002801DDC1
:10C44000024600E04242914205DD002C01DD20461B
:10C4500004E0604202E0002800DC404200994018FD
:10C4600000B2002800DA284605463146384601F079
:10C4700098FA04000ED03146384601F086FA0228B8
:10C4800008D93146384601F086FA0019A84200DB87
:10C4900005462DB238463146692201F0B8FA04B299
:10C4A000384631466A2201F0B2FA00B2844200DC1A
:10C4B0000446002C01DD281905B22846F8BD7CB5DC
:10C4C0000C4605465B2201F0A2FAC6B269460E7020
:10C4D00028462146162201F09AFA69460871002E74
:10C4E00001D10120087008787CBDF8B50D460746DB
:10C4F000002600E00068002817D081690903090CB4
:10C50000F8D080690003000C0090FFF7FFFC0400E6
:10C510000DD00099FFF777FE276001276560002D99
:10C5200007D0A86800282FD031E03046ECE7002083
:10C53000F8BDFBF733FB05001BD0EA68002A1CD0CE
:10C54000686A401C810068621046FFF78BFDE86056
:10C55000696A8900091F4450A682E6820020FBF721
:10C5600037FB401E20830020FBF774FB401E6083D6
:10C5700020E02046FFF752FDD9E70420FFF7C6FC74
:10C58000E86004606F62E7E72846FFF79BFEA86853
:10C590000168002910D04168491C4160A8688900E1
:10C5A0000068FFF75FFDA9680860A968496889000D
:10C5B000091F44502046F8BD0420FFF7A7FCA968D6
:10C5C00008600460A8684760F4E7000070B505469D
:10C5D00001F0C0FD002000F063FA284603F0B4F932
:10C5E000284600F06FF8012000F05AFA0F21134A94
:10C5F0000904284602F016FA284602F0FBF9FEF775
:10C600006BFA030008D0284601F07EFD002803D015
:10C6100029461846FEF7FEF9284600F099FC04006A
:10C620000BD02A462221FDF775FE2A4623212046FB
:10C63000FDF770FE284601F020FD70BDFFFF0000F1
:10C640007FB50C46064601F06DFD0546E0060CD5AB
:10C6500002AA6946304600F0C0FD6946304601F046
:10C660002CFD02A9304601F028FDF069A043F061DD
:10C67000E0070FD0304601F000FD304601F052FDDA
:10C68000002807D0304600F063FC01F063FD30461F
:10C6900001F060FD304601F045FDA84202D1E00105
:10C6A000800F04D0304600F053FC01F053FD7FBDF5
:10C6B00010B5028C13468A4311468B4201D002F01A
:10C6C0007DFC10BD70B5046805462068002803D0C5
:10C6D00028602846FFF7F6FF2C6062682046002A93
:10C6E00001D02946904770BDF8B54D680C46002D25
:10C6F0001DD0284600F090FC0646284600F058FD64
:10C70000074628460021102201F081F9E98A122209
:10C710004018C01BE082401E60832846002101F0C3
:10C7200076F9A98A4018801BA082401E2083094800
:10C73000E061002D02D008480848E0610246084840
:10C740000243E261002D03D00120C0030243E261F5
:10C75000F8BD0000021000000230000002330000AB
:10C760007408000010B501460348FFF7BEFE0446FA
:10C77000FFF72CFF204610BD181D010870B50C46B0
:10C780000846F4F795FE002000F08AF92046154A85
:10C79000002102F003FA012000F082F90021204676
:10C7A000FAF7E8FD204600F0C8FB002802D020463A
:10C7B000FEF7B5F9A068002813D00068002500280E
:10C7C00003D0FFF72BFCA0680560A068C0680028B4
:10C7D00003D0FFF723FCA068C560A068FFF71EFC2C
:10C7E000A56070BDFFFF0F00F1B5A4B02498FDF760
:10C7F00050FD06462498FDF78AFD012700240546D2
:10C80000122E6AD0152E79D0182E75D12498FDF7E6
:10C8100046FD014611902846F8F7AAFE0021284659
:10C8200001F067F800280BD02846FF302130FCF7D4
:10C83000D3FA060004D0FBF799FF3046FFF7DCFB84
:10C840000021284601F041F8002855D002A8FCF745
:10C85000FBFA6846C47208A884708474847702AABC
:10C860000021284601F0A4FA0021284601F067F9CA
:10C8700010900021284601F05CF906462946143143
:10C880006846FAF75BFE684601881098091A684600
:10C890000180818810980918684681804088811B32
:10C8A00068464180C08881196846C18012A81199E4
:10C8B00000F0EEF87548139002A8169068461F9491
:10C8C0001590149712AA1A212846FDF723FD6A46EF
:10C8D00002A91198FCF7A4FAD1E02498FDF715FD00
:10C8E00006460078022807D00021284601F001F80A
:10C8F000002804D00220307025B0F0BD41E00021B6
:10C90000284601F0D0F804900021284601F017F9DC
:10C9100003900021284601F00CF9294602901431B9
:10C920006846FAF70BFE684601880398091A6846BC
:10C93000018081880398091868468180418802989F
:10C94000091A68464180C188029809186846C18062
:10C9500070686946049AF4F7A6FB00280DD0002100
:10C96000284600F0A6FFFD2807D3284600216022B4
:10C9700001F04DF8C0B2FD2801D23770BCE7347029
:10C98000BAE72498FDF78BFC109002A8FCF75CFA3C
:10C990000021284600F099FF002803D008A9C87A92
:10C9A0003843C87202AA0021284601F001FA00218A
:10C9B000284601F0C4F807460021284601F0B9F8DE
:10C9C00029460646143168461191FAF7B7FD6846C4
:10C9D0000088C11B684601808088C1196846818033
:10C9E0004088811B68464180C08881196846C180A3
:10C9F00012A8109900F04CF82448139002A8169041
:10CA000068461F941590149412AA1A212846FDF71F
:10CA100081FC0021284600F06CFF002807D0684602
:10CA20000089002803D0069E0127069401E0069E97
:10CA300000276A4602A91098FCF7F2F9002F1ED0D1
:10CA40001820FFF791FA074668460822825E002305
:10CA500038461199FCF732F92946FF312131384621
:10CA6000FBF7BEFC002E0AD06846C47208A8847288
:10CA70008474847706966A4602A910982AE712AA57
:10CA80001B212846FDF746FC36E70000181D01086B
:10CA900070B50D4604464821FFF7B5FB256070BD13
:10CAA000014908707047000028000020F3B585B0E8
:10CAB0000698FDF7EEFB04460698FDF7EEFB0546EB
:10CAC000012C22D0082C22D0032C42D02A2C42D078
:10CAD0000D2C4FD00E2C7DD0092C7CD00A2C7BD075
:10CAE0000F2C7AD0292C79D0222C78D0242C77D0F6
:10CAF000132C76D0152C03D0182C01D0122C02D177
:10CB00000698FFF771FE07B0F0BD2021F8E0202164
:10CB1000FFF7CEFD0698FDF7D3FBFEF7A2FC002839
:10CB2000F1D10821284601F0E1F80028EBD0288C4B
:10CB3000C00709D001212846FFF7BAFD00221C21B9
:10CB40002846FDF7E7FBDEE701212846FFF7B2FBA9
:10CB5000F4E72021EEE000F053F90646002406E059
:10CB6000A868A1000068405801F0F4FA641CB442BF
:10CB7000F6D3C8E7082101F0B9F8002818D00698C4
:10CB8000FDF7C3FB0478132C06D0112C04D0142C11
:10CB900007D0122C05D008E001212846FFF78AFBB8
:10CBA00003E001212846FFF783FD0A2CC6D1AAE73E
:10CBB00081210901284601F099F80028A3D02846D0
:10CBC00001F095FA00289ED10027284600F024FAAB
:10CBD000064607E066E092E095E0AAE0ADE0C9E035
:10CBE000E7E0EBE0284600F079FA04460698FDF706
:10CBF0008CFB007812281BD011280CD0132829D0C8
:10CC0000142880D1284600F0FDF9800703D0002EBB
:10CC100036DC002C34DC284600F094F90446284623
:10CC200000F0D4FAE117890F09198910401A0BE0B6
:10CC3000284600F087F90446284600F0C7FAE117B5
:10CC4000890F09198910401801B23A46284602F0A6
:10CC500069F958E7284600F0D5F98007E8D0002E9A
:10CC600001DC002CE4DD284601F03AF804462846B1
:10CC700000F0A5FAE117890F0919891040180BE097
:10CC8000284601F02DF80446284600F098FAE117EE
:10CC9000890F09198910401A01B23A46284602F054
:10CCA0002DF930E70121890201F020F8002803D096
:10CCB0000121284602F005F9284600F03EF9FDF76B
:10CCC00011FF06460224FEF7A9FB002802D10698B0
:10CCD000FDF7F6FAFEF7D1FB022801D0042800D1B7
:10CCE0000624002E04D0082004432146284607E0ED
:10CCF00021462846FFF7DEFA082128461AE040219F
:10CD0000FFF7D8FAFFE64021FFF7D2FC284600F0F3
:10CD100080FD02289DD102AA6946284600F05DFAEE
:10CD20006946284601F0C9F902A9284601F0C5F96B
:10CD3000E9E60E21FFF7BCFCE5E6002100F090FDDE
:10CD400004460021284600F0E2FD204302D0284698
:10CD500001F000FA284600F053F80646002406E0E9
:10CD6000A868A1000068405801F0F4F9641CB442BE
:10CD7000F6D3C8E60021012200F049FE06B228469B
:10CD80000021042200F043FE04B20021284600F0F6
:10CD900067FD07460021284600F0B9FD384304D15D
:10CDA0000A48864201D08442ACD1284601F0D2F92B
:10CDB000A9E6688C022108436884F6E70021FFF7A2
:10CDC00016FB01460698FDF7C5FA9CE6D127000040
:10CDD00010B50C46002800D16068006800280DD00E
:10CDE00001690029F9D00021E160026921469047DC
:10CDF000217E0120C90700D0002010BD012010BDF8
:10CE00008068002800D04068704770B50C46054621
:10CE1000002100F062FD06462146284600F055F844
:10CE2000704202B211462046FAF7EDFB0021284677
:10CE300000F0C9FD2188401820800021284600F01C
:10CE4000CEFDA188081AA0800021284600F0D3FD5D
:10CE50006188401860800021284600F0A8FDE18824
:10CE6000081AE08070BD70B50446002100F0C3FDD3
:10CE700005460021204600F09AFD06460021204686
:10CE800000F02BFD0246204600F05CF8401B801BA2
:10CE90005100401A00B270BD70B50446002100F088
:10CEA00092FD05460021204600F099FD064600212E
:10CEB000204600F012FD0246204600F011FF401B04
:10CEC000801B5100401A00B270BD0A46014610B5E1
:10CED00014311046FAF73BFB10BD000070B54168F5
:10CEE000002901D000F038F804460B48F4F78BFC19
:10CEF0000EE00021426A05E0C3688D005B59A34241
:10CF000008D0491C8A42F7D801460348F4F77FFC51
:10CF10000028EED170BD0000F810002080680028C5
:10CF200005D0827E9206920E8A4201D80020704778
:10CF3000C0680C225143401870478068002800D018
:10CF400080687047418BC08A081A401C00B2704745
:10CF5000002800D04068704700B50146FFF7F8FF91
:10CF60000028FAD1084600BDFEB50646234CFFF75F
:10CF700047FF0746002510E0B068A9000068405848
:10CF80001F49009000F0B9FE002805D100991A2031
:10CF9000085EA04200DB04466D1CBD42ECD30021BC
:10CFA000304600F02EFD00900021304600F005FDD7
:10CFB00007460021304600F096FC05460F488442A3
:10CFC00004D0708BC01B401B201A04B2304600F006
:10CFD00029FC01903046FFF7B5FF0099401AC01BAD
:10CFE0006900411A0198411A304600F0EFF8081A1A
:10CFF00000B2844200DD2046FEBD000001E0FFFFDC
:10D00000010004008068002803D0407E0007000F64
:10D0100070470F2070470000F0B585B0064600212C
:10D0200000F035FC012807D0B068002802D0008A43
:10D03000404200B205B0F0BD0021304600F0D5FC02
:10D0400003900021304600F0C4FC019000213046DE
:10D0500000F049FC00901F4C3046FFF7D1FE074618
:10D06000002510E0B068A900006840581A490290F5
:10D0700000F043FE002805D102991420085EA0426A
:10D0800000DC04466D1CBD42ECD31248844207D03C
:10D0900000990198B28A40181018001B04B201E0F0
:10D0A0000C4C6442304600F0CBFB0546304600F0A5
:10D0B00017FE0399411A0198091A00984000081AAE
:10D0C000291A304600F07BF8401800B28442B1DDE6
:10D0D0002046AFE7FF1F000001000400FEB5064632
:10D0E000002100F0D4FB012806D0284C3046FFF781
:10D0F00087FE0746002518E0B168002902D01020FD
:10D10000085EFEBD0020FEBDB068A9000068405862
:10D110001F49009000F0F1FD002805D1009918206A
:10D12000085EA04200DB04466D1CBD42ECD300212A
:10D13000304600F05AFC07460021304600F049FC1A
:10D1400000900021304600F0CEFB05460F48844297
:10D1500004D0308BC01B401B201A04B2304600F0B4
:10D160006FFB0190304600F0BBFDC11B0098081A10
:10D170006900411A0198411A304600F020F8081A57
:10D1800000B28442BFDD2046FEBD000001E0FFFF8B
:10D19000010004008068002802D0007E0007800F94
:10D1A00070478068002802D0007E8006800F70479C
:10D1B0008068002802D0408A404200B270478068F0
:10D1C000002802D0008A404200B2704780680028E0
:10D1D00002D0408A404200B27047F0B500271646A0
:10D1E0000C46FF4393B0054600223B4611462046BD
:10D1F0000097FAF722FA00223B4611463046009784
:10D20000FAF71BFA1021284600F070FD002815D00F
:10D21000284600F0FEFA070010D00020FEF704F9BF
:10D220000290022F08D00DE0FEF71BF9A8420298E9
:10D2300006D0FEF7F9F802900028F5D113B0F0BD42
:10D240000028FBD02846FFF7B3FF05902846FFF7DC
:10D250008BFE0C902846FFF7DFFE0B902846FFF769
:10D260003DFF09902846FFF7CDFE03900020009077
:10D2700003980007800F14D0012F10D0032F02D085
:10D28000022F07D00DE00598002808DC0C98002834
:10D2900005DC06E00298FEF7D5F80C2801D1012044
:10D2A000009000200A900398800714D0012F10D01E
:10D2B000032F02D0022F07D00DE00B98002808DCC6
:10D2C0000998002805DC06E00298FEF7BBF8032861
:10D2D00001D101200A9000990A980843AED001219B
:10D2E0000904284600F0D3FA012800D000200121CB
:10D2F0000E900904284600F084FB012106900904E1
:10D30000284600F05AFB01210F900904284600F03E
:10D3100060FB074601210904284600F066FB0D90DA
:10D3200001222846110400F072FB00B20290284648
:10D33000FFF708FE0490284600F0D2FC0390009806
:10D34000002800D0029808900A98002800D002987F
:10D350001090012128460904212200F058FBC0B298
:10D36000022809D2012128460904312200F04FFB8E
:10D37000C0B2022800D261E70599049841180C98C0
:10D38000081800B20790009800286ED0079800286F
:10D39000FBD0E88A7080688BF0800E98002807D058
:10D3A000A88AC01930800299491E4018B08007E051
:10D3B000298B0D98081AB0800299401A401C3080C1
:10D3C00006990498411A0F98091A1098081A049996
:10D3D000009048430799F3F705F800B20590002044
:10D3E000FAF7E2FB0A214843FF21403150308842DE
:10D3F00009DD0020FAF7D8FB0A214843A02150306C
:10D40000F2F7F0FF00E001200599884201DA0846B2
:10D4100014E00020FAF7C8FB0A214843FF214031FD
:10D420005030884209DD0020FAF7BEFB0A2148434C
:10D43000A0215030F2F7D6FF00E0012000B20590A5
:10D440000099081A00B2009004990798401A01B296
:10D4500000290BDCE98A069808187080698B0F9800
:10D46000091A1098081A401EF0808AE00C9A009859
:10D470005043F2F7B7FF0099EA8A081A0699401854
:10D48000101801B2718005981622401E0818F0800D
:10D49000AA5E06981018814234DA70800020FAF7EC
:10D4A00083FB0A214843FF2140315030884209DD87
:10D4B0000020FAF779FB0A214843A0215030F2F707
:10D4C00091FF00E001200221715E40180621715E8B
:10D4D000884217DD0020FAF767FB0A214843FF2145
:10D4E00040315030884209DD0020FAF75DFB0A2107
:10D4F0004843A0215030F2F775FF00E00120718809
:10D500004018F0801A22AA5E10980621121A0F986D
:10D51000715E101A814234DDF0800020FAF744FB7E
:10D520000A214843FF2140315030884209DD002064
:10D53000FAF73AFB0A214843A0215030F2F752FF94
:10D5400000E001200621715E081A0221715E884206
:10D5500017DA0020FAF728FB0A214843FF2140315F
:10D560005030884209DD0020FAF71EFB0A214843AB
:10D57000A0215030F2F736FF00E00120F188081AB0
:10D5800070800B99039841180998081800B204900C
:10D590000A98002800D151E604980028FBD0698B36
:10D5A0000F98081AE0800299401A401C6080A88AEF
:10D5B0002080288BA0800398C11B0D98091A089819
:10D5C000081A0399009048430499F2F70BFF06B23A
:10D5D0000020FAF7E9FA0A214843FF214031503090
:10D5E000884209DD0020FAF7DFFA0A214843A0212A
:10D5F0005030F2F7F7FE00E00120B04215DB0020CA
:10D60000FAF7D2FA0A214843FF21403150308842CC
:10D610000ADD0020FAF7C8FA0A214843A021503059
:10D62000F2F7E0FE064600E00126009836B2801BC5
:10D6300000B2009003990498401A01B2002916DC48
:10D640000E980028A88A08D0C1190898401E08180A
:10D650002080298B0D98081A07E0C0192080298B9B
:10D660000D98091A0898081A401EA080E6E5099A44
:10D6700000985043F2F7B6FE0099081A0E9900B2CE
:10D680000029A98A76D008180899761E79184018BA
:10D6900000B220808219A2801422AA5E5118814211
:10D6A00032DD21800020FAF77FFA0A214843FF2665
:10D6B00040365030B04209DD0020FAF775FA0A21F1
:10D6C0004843A0215030F2F78DFE00E001200021F8
:10D6D000615E40180421615E884215DD0020FAF782
:10D6E00063FA0A2148435030B04209DD0020FAF7BE
:10D6F0005BFA0A214843A0215030F2F773FE00E0A4
:10D70000012021884018A08004211822615EAA5EB1
:10D7100075E0A0800020FAF747FA0A214843FF2568
:10D7200040355030A84270DD0020FAF73DFA0A215A
:10D730004843A0215030F2F755FE0421615E081ADB
:10D740000021615E884291DA0020FAF72DFA0A2161
:10D7500048435030A8425ADD0020FAF725FA0A2142
:10D760004843A0215030F2F73DFEA188081A2080DE
:10D7700064E5FFE7C019081800B2761E2080811901
:10D78000A1801421695EC919884232DA2180002003
:10D79000FAF70AFA0A214843FF2640365030B042D1
:10D7A00009DD0020FAF700FA0A214843A021503091
:10D7B000F2F718FE00E001200021615E401804210C
:10D7C000615E884215DD0020FAF7EEF90A21484330
:10D7D0005030B04209DD0020FAF7E6F90A2148434B
:10D7E000A0215030F2F7FEFD00E001202188401812
:10D7F000A08018220421AA5E0898615E121A0D9872
:10D80000101A814285DC19E5FFE7012095E7012028
:10D81000ABE78068002803D0007E8007800F704748
:10D820000320704708B505496A46496800912C21D4
:10D83000FCF770FD69460220085E08BD341D010832
:10D8400008B505496A46096800912C21FCF762FD7C
:10D8500069460020085E08BD341D0108008C704731
:10D8600010B5092200F0D3F8C0B210BD10B50922DE
:10D8700000F0CDF8C0B210BD10B5662200F0C7F8B8
:10D8800010BD10B5162200F0C2F8C0B210BD10B520
:10D89000162200F0BCF8C0B210BD70B50C460546AB
:10D8A000202200F0B4F8024621462846F4F7A7F8F3
:10D8B00070BD10B5212200F0AAF8C0B210BD10B59D
:10D8C000682200F0A4F8C0B210BD10B5342200F0F8
:10D8D0009EF8002800D0012010BD10B5322200F0C3
:10D8E00096F800B210BD10B5322200F090F800B2E8
:10D8F00010BD10B5172200F08AF8002800D00120D2
:10D9000010BD10B5042200F082F800B210BD10B5B1
:10D910000A2200F07CF880B210BD10B50A2200F097
:10D9200076F880B210BD10B5602200F070F8C0B279
:10D9300010BD70B50E460546FFF7F5FF02281CD94D
:10D94000FF24FD2802D20102081A040A002E01D089
:10D95000002603E02846FFF7FBFA0546002D0AD013
:10D9600031462846FFF7DFFF022806D9FD28F1D20D
:10D970004443240AEEE7022C01D8002070BDFD2CA0
:10D9800001D3FF2070BD204670BD10B5372200F0D6
:10D990003EF8C0B210BD10B5382200F038F800B221
:10D9A00010BD10B5352200F032F800B210BD10B530
:10D9B000112200F02CF800B210BD10B5112200F0B9
:10D9C00026F800B210BD10B5122200F020F800B207
:10D9D00010BD10B5122200F01AF800B210BD10B53B
:10D9E000132200F014F800B210BD10B5132200F09D
:10D9F0000EF800B210BD10B5102200F008F800B209
:10DA000010BD10B5102200F002F800B210BDF7B53D
:10DA1000064682B014460121104601F091FE0746E9
:10DA2000002516E06B46224630460399F9F7D8F8F0
:10DA3000054601282AD0002F0FD0022D05D00398CB
:10DA4000002802D00020039003E03046FFF780FA60
:10DA50000646002EE6D1012D18D00398002803D1E8
:10DA6000012C05D0042C03D0204601F001FE0CE06F
:10DA7000316811E0012C0CD0C88A00280BD0002995
:10DA80000CD0012C0CD01620085E0090009805B038
:10DA9000F0BD888AF1E709680029EBD10020F4E79E
:10DAA0001420085EF1E710B50B22FFF7B0FF00B2BB
:10DAB00010BD10B54122FFF7AAFF00B210BD10B58E
:10DAC0004222FFF7A4FF00B210BD10B54522FFF7B8
:10DAD0009EFFC0B210BD10B54322FFF798FF00B201
:10DAE00010BD10B54022FFF792FF00B210BD70B517
:10DAF0000C4605465522FFF78AFF02462146284676
:10DB0000F3F77DFF70BD10B55722FFF780FF10BD02
:10DB100010B55722FFF77BFF10BD10B55822FFF755
:10DB200076FF00B210BD10B55922FFF770FF00B2AA
:10DB300010BD10B56A22FFF76AFF00B210BD10B524
:10DB40006922FFF764FF00B210BD10B50122FFF794
:10DB50005EFF00B210BD10B50122FFF758FF00B202
:10DB600010BD10B50722FFF752FF00B210BD10B56F
:10DB70000822FFF74CFF00B210BDF0B5074685B094
:10DB80000C4608886946088060884880208888801C
:10DB9000E088C880A088088160884881A088888142
:10DBA000E088C8811D461646384601F0D5FA2B4656
:10DBB0003246384601A901F0CFFA2B4632463846A4
:10DBC00002A901F0C9FA2B463246384603A901F0F2
:10DBD000C3FA694600200423085ECB5E984201DA4E
:10DBE000054600E01D4608220E468A5E0C21715E45
:10DBF0008A4201DA164600E00E46B54203DA984240
:10DC000006DB184604E08A4201DA104600E00846C6
:10DC10002080684600230421C35E415E8B4201DD03
:10DC20001D4600E00D4608220646825E0C20305E4E
:10DC3000824201DD164600E00646B54205DD8B4214
:10DC400001DD184604E0084602E0824200DD10468D
:10DC5000A080694602230620CB5E085E834201DA7B
:10DC60001D4600E005460A220E468A5E0E21715EC0
:10DC70008A4201DA164600E00E46B54203DA8342D4
:10DC800006DA184604E08A4201DA104600E0084647
:10DC90006080684602220623825EC35E9A4201DDEE
:10DCA000154600E01D460A210646415E0E20305E04
:10DCB000814201DD0E4600E00646B54205DD9A428E
:10DCC00001DD104604E0184602E0814200DD08460E
:10DCD000E080052211462046F9F795FC05B0F0BD1D
:10DCE000018B808A081A401C00B27047C0698143CA
:10DCF00001D00020704701207047C069084000D063
:10DD000001207047F8B514460D4606465622FFF727
:10DD10007EFEC0B2A076022807D929463046FFF71A
:10DD200008FE022802D80020A076F8BDFD2803D204
:10DD3000A17E4143080AA076A07E0228F5D9294693
:10DD40003046FFF7D4FE009068460088A081304638
:10DD500029465822FFF75BFEA08230462946592209
:10DD6000FFF755FE6082304629465A22FFF74FFEE4
:10DD7000A17F4007C908400FC9000143A177002DCA
:10DD80000AD029463046FFF79AFD4007810EA07F52
:10DD9000C72210400843A07729463046FFF7B3FE5C
:10DDA0002060304629465B22FFF731FE2077F8BD20
:10DDB000FEB514460D460646FFF7BBFD2746203745
:10DDC0000290002D0CD0022805D80020E070A0762B
:10DDD000B870B87241E129463046FFF770FDA07077
:10DDE000304629460B22FFF712FE2080E178A01C66
:10DDF000019000295CD0304629462122FFF707FE1A
:10DE0000C0B2E070022853D929463046FFF745FDDD
:10DE1000009068460088A080304629462622FFF7F9
:10DE2000F6FD010007D0487A400704D00A22A01D61
:10DE3000FEF730F93CE0304629462322FFF7E7FDA4
:10DE40004107E07B490FC008C0000843E07340076A
:10DE500022D029463046FFF720FD69460090088809
:10DE6000E080222229463046FFF7D1FD02462946AE
:10DE70003046F3F7C4FD0090694601980988018196
:10DE8000304629462422FFF7C2FD2072304629463B
:10DE90002522FFF7BCFD2073304629462722FFF7D5
:10DEA000B6FDE17B4007C722800E11400143E173BC
:10DEB000304629463222FFF7AAFD00B2208400280E
:10DEC00025D0B878002822D0304629463122FFF7E5
:10DED0009EFDC0B2B870022819D9304629463322B7
:10DEE000FFF795FDC006810EF878C1221040084367
:10DEF000F870302229463046FFF789FD0246294650
:10DF00003046F3F77CFD009068460088E0832946A0
:10DF10003046FFF746FDE08400281CD0B87A002880
:10DF200019D029463046FFF730FDB872022812D9C1
:10DF300029463046FFF72FFD2085362229463046F8
:10DF4000FFF765FD024629463046F3F758FD00907D
:10DF500068460088A084A07E002832D0304629463A
:10DF60002822FFF754FD206100282AD03046294698
:10DF70002922FFF74CFDC0B2A076022821D92069E2
:10DF8000FDF739FA02286AD02A2229463046FFF7DF
:10DF90003EFD024629463046F3F731FD00906846C3
:10DFA00000882083304629462B22FFF730FDE0769B
:10DFB000304629462C22FFF72AFD002800D00120F8
:10DFC0002077B87D00282DD029463046FFF789FDFF
:10DFD000E085002826D0B87D022823D9294630467E
:10DFE000FFF773FDB87502281CD929463046FFF7A4
:10DFF00060FD208629463046FFF761FD6086294690
:10E000003046FFF768FDA086442229463046FFF7D8
:10E01000FEFC024629463046F3F7F1FC00906846C4
:10E020000088A0850298FD2818D2E078029948431C
:10E03000000AE070A07E02994843000AA076B878F2
:10E0400002994843000AB870B87A02994843000A16
:10E05000B872B87D02994843000AB875FEBD2946DA
:10E060003046FFF750FD606129463046FFF73FFD1F
:10E070000090684600882083A3E77CB50446F3F748
:10E080008CFC0546214614316846F9F760FA68466B
:10E090000088411B684601804088411B68464180DA
:10E0A0008088411968468180C08841196846C180CE
:10E0B0006946204600F001F87CBD7CB50C4605465B
:10E0C000FEF70CFFF9F7DCFD00280FD0214668466B
:10E0D000F9F73DFA69462846FEF712F9002805D0FF
:10E0E0002846FEF7FBFE6946F3F70CFB7CBD006893
:10E0F000002808D0017E8907F9D0007E8007800FB4
:10E10000012800D0002070470068002809D0017E57
:10E110000907890FF8D0007E0007800F012800D082
:10E120000020704710B504460949FFF7E6FD0028B6
:10E1300001D0002010BD2046FEF70AFF0028F9D0CC
:10E140000021FFF7EAFB0028F4D0012010BD0000F9
:10E150000100060010B5418C012211434184FEF7F5
:10E16000FBFE418C042211434184FEF7B7FE406858
:10E17000002801D001F0FAFC10BDFFB581B01746B0
:10E180000198FEF73DFE0646002523E00198A90010
:10E190008068006844580498002806D0012189044A
:10E1A0002046FFF7A3FD002813D1A18A029800237F
:10E1B0000818A082E08A3A46C019E082218B0298B2
:10E1C00008182083608BC019608320460299FFF7EE
:10E1D000D4FF6D1CB542D9D305B0F0BDF0B545688C
:10E1E0008BB016460F460446002D34D00021284639
:10E1F000FFF7E9FB019000212846FFF7FCFB012116
:10E20000009089042046FFF771FD002809D001988D
:10E21000A98A3818081807B20098E98A301808182F
:10E2200010E02846FEF7CBFFAA8A01995118081A78
:10E23000C01907B22846FEF7C9FFEA8A00995118AB
:10E24000081A801906B200212846FFF746FB391844
:10E2500030180FB206B2A08A381A07B26846078093
:10E26000E08A301A06B268464680002F01D1002E9F
:10E2700042D02046FFF701FF08A92046FEF725FE01
:10E2800000200090002D0ED006A92846FEF7BDFD07
:10E29000002206A908A8F2F706FF0090002802D184
:10E2A000284600F053FEA08A3246C019A082E08AB8
:10E2B00039468019E082208B0023C0192083608BAF
:10E2C000801960832046FFF758FF002D11D02246A9
:10E2D00022212846FCF71EF82046FFF7CEFE2046F6
:10E2E000002206A91430F2F7DEFE0099002907D1BA
:10E2F00004E02046FFF7C1FE0BB0F0BD0028FBD0C4
:10E30000284600F023FEF7E7F8B50D460646FEF76F
:10E3100048FF002814D13046FEF74AFF0446304635
:10E32000FEF722FE00280BDA002C09DD4042844271
:10E3300000DB044622B22B460021304600F0BAFC36
:10E340003046FEF727FF002823D13046FEF764FE53
:10E3500004463046FEF7C2FE074600213046FFF76E
:10E3600096FA01280BD0002F13DA002C11DD784229
:10E37000844200DB044621B22B46002206E0002C3A
:10E3800007DA002F05DD2B4600222146304600F03B
:10E3900091FCF8BDF3B59BB004468068029014A9C7
:10E3A0001C98FEF792FD1C98F3F7F7FA0146024617
:10E3B00014A8F9F728F914AA12A80299F2F74BFE4B
:10E3C000002806D10121C9041C98FFF78FFC002802
:10E3D0004AD012A8A0600126224614211C98FBF7FF
:10E3E00099FF224615211C98FBF794FF224616211F
:10E3F0001C98FBF78FFFFF21002000F0CFFF07469E
:10E40000FF21002000F0CAFF0546FF21002000F098
:10E41000C5FF010668460088C90E4009400108434F
:10E420003F2149018843A908490108434105F808EB
:10E43000490DC00201436846018088B2009003A8DC
:10E44000FAF702FD6846018801823322C273012275
:10E4500082854C2208A882736846418514AA03A9C4
:10E460002046FAF7DDFC00E000260121C9041C98D3
:10E47000FFF73CFC002805D0082216A80299F1F706
:10E48000F1FE07E01C9A16A814320299F2F7E3FD98
:10E49000002812D016A8A0601C98FEF7B1FC074611
:10E4A000002508E01C98A9008068006841582046B3
:10E4B00002F0D2FB6D1CBD42F4D3002E10D012A886
:10E4C000A060224617211C98FBF724FF2246182142
:10E4D0001C98FBF71FFF224619211C98FBF71AFF17
:10E4E0000298A0601DB0F0BDF1B58AB00A98FFF7A0
:10E4F00019FE00287ED10A98FEF72AFD0890002117
:10E500000A98FFF72EFB019000210A98FFF72FFBD6
:10E510000646089800280CD0FEF7BEFC0590089827
:10E52000FEF7A1FC074601984004800F012803D0A4
:10E5300015E0324601998AE0032101984903884396
:10E540007D21090188420ADC4910884200DD081A51
:10E55000059948436421F1F745FF00B2019070042A
:10E56000800F012810D103213046490388437D21C3
:10E570000901884208DC4910884200DD081A784306
:10E580006421F1F72FFF06B200216B220A98FFF7F2
:10E590003EFA05B200216C220A98FFF738FA00B261
:10E5A00006900A98FFF79CFB03900A98FEF7CAFCB6
:10E5B00004466804800F012811D10321284649032D
:10E5C00088437D210901884209DC4910884200DD29
:10E5D000081A039948436421F1F704FF05B206982D
:10E5E0004004800F012813D1032106984903884372
:10E5F0007D2100E02EE00901884209DC49108842B3
:10E6000000DD081A60436421F1F7ECFE00B20690C9
:10E6100001980021401905B20698301806B20A98F0
:10E62000FFF724F900280AD001280ED0801E03002D
:10E63000F2F732FC08121C2A2E37223D400B002133
:10E640000898FFF71EF9012810D0324629460A988B
:10E65000FFF7C4FD0BB0F0BD05990398CA0F511820
:10E66000C20F101849104010081A02E003990598CB
:10E67000401A401905B2E8E7F80FE10FC01909196F
:10E6800040104910401A00E0381B801906B2DCE740
:10E6900005980399C20F1018CA0F4010511849105D
:10E6A00001E003990598401A401905B2ECE7039977
:10E6B000059807E005980399C20F1018CA0F40107B
:10E6C00051184910401A401905B2D5E7F0B5044673
:10E6D000408C8FB0010501D540057CD42046FEF763
:10E6E00037FC0A90002877D02046FEF795FC06906C
:10E6F000608C0026000503D52046FFF7F1FA67E09D
:10E7000000212046FFF721FA0546A148854201D1A4
:10E71000012600E000266804800F012809D10320AB
:10E720004003294681437D200001814201DC012014
:10E7300000E0002002900A98FEF7AEFB0746002E8C
:10E7400004D02046F4F7F6F805462FE0029800289A
:10E750002CD00A98408C00051AD400210A98FFF7A3
:10E76000F4F901468A48814212D100212046FFF780
:10E77000B4F8054600212046FFF725F9401900901E
:10E7800000212046FFF72BF94119009808180CE0EA
:10E7900003212846490388437D21C900884200DDC2
:10E7A000081A78436421F1F71DFE05B220460021C6
:10E7B0000222FFF72CF900B2039020460021032229
:10E7C000FFF725F902B23B4628460399F8F7A4FF64
:10E7D0000746204601E08BE08BE0FEF7E9FC08905D
:10E7E00000200790608C400503D52046FEF7AAFB69
:10E7F0006AE000212046FFF784F865490546884213
:10E8000001D1012000E0002007906804800F01285A
:10E8100009D103204003294681437D200001814224
:10E8200001DC012000E0002002900A98FEF71BFBAB
:10E8300001900798002804D02046F4F705F8054613
:10E8400030E0029800282DD00A98408C40051AD458
:10E8500000210A98FFF755F801464D48814212D130
:10E8600000212046FFF739F8054600212046FFF732
:10E87000C2F84019049000212046FFF798F841198A
:10E88000049808180DE003212846490388437D2198
:10E89000C900884200DD081A019948436421F1F754
:10E8A000A1FD05B2204600210522FFF7B0F800B215
:10E8B0000390204600210622FFF7A9F802B228465D
:10E8C000019B0399F8F7EAFE05460798064305D031
:10E8D00000232046089A069900F0E6FA2046FFF742
:10E8E000FFF9B84207D12046FEF72CFBA84202D11F
:10E8F00000200FB0F0BD2046FFF7BFFB0BA920465C
:10E90000FEF7E3FA0DA90A98FEF77FFA00220DA997
:10E910000BA8F2F7C8FB060002D10A9800F016FB1C
:10E92000E08A6D1E4019608300212046FEF7A9FF92
:10E9300001281DD0A08A7F1EC01920830BAA29217F
:10E940002046FBF7E7FC224622210A98FBF7E2FC6F
:10E950002046FFF792FB608C02210843608420462A
:10E9600000220DA91430F2F79EFB002E07D104E01F
:10E97000208BC01B401CA082E0E7002802D00A9830
:10E9800000F0E4FA204600F005F80120B1E70000AD
:10E99000D127000038B50446F2F7FFFF05460021F5
:10E9A000684601806A4613212046FBF7B3FC68469F
:10E9B0000021415EA94202D02046FFF75EFBA0681D
:10E9C000002803D069460988C1820AE068460088A9
:10E9D000002806D02046FDF775FC6846A16800882F
:10E9E000C88269460020085EA84202D02046FFF790
:10E9F00044FB38BD70B505460021FFF7A6F8044674
:10EA000000212846FEF77DFF05498C4203D088424D
:10EA100001D0002070BD2846FFF79CFB012070BD8F
:10EA2000D1270000F7B50546594882B000780C465A
:10EA300000287BD02846FFF720FBFF20000404407D
:10EA40000421049800F07CFE06460221049800F0A0
:10EA500077FE00900121049800F072FE01901021D1
:10EA6000049800F06DFE0746002E1FD00F20000412
:10EA7000844213D0002C11D0284600210422FEF736
:10EA8000C6FF444900B2884208D02846002101222E
:10EA9000FEF7BDFF3F4900B2884207D100222A217C
:10EAA0002846FBF737FC2846FFF754FB0F200004ED
:10EAB000844201D0002C0CD137490498884201D0FF
:10EAC000002E06D02846FEF743FA002801D0FFF7B3
:10EAD00041FB0F200004844201D0002C39D1002FCB
:10EAE00037D0284600216E22FEF791FF00B20028A1
:10EAF00008D1284600216D22FEF789FF00B2C11F10
:10EB0000F93901D0022713E0284600216122FEF7DF
:10EB10007EFFC0B2FF2807D1284600216822FEF7F9
:10EB200076FF0006000E02D0012701E02DE000274D
:10EB3000A868002806D0817E8906890EBA01114393
:10EB4000817606E0002F04D02846FDF7BBFBA868BD
:10EB5000F1E7114F0498B84202D00098002802D083
:10EB60002846FFF717FF2846FFF787FA0498B842B0
:10EB700004D0009801993043084206D001200004D7
:10EB8000844202D0284602F045FA05B0F0BD0000EC
:10EB900028000020D1270000FFFF0000F0B5044648
:10EBA0008BB090B20390FF2000040240404E0F460D
:10EBB0000192002903D0F879002800D10026002511
:10EBC000284664E0E268E9000091091D0692099177
:10EBD0005258374B964691B21202120E12049446C6
:10EBE000039A9A4201D091420ED10F220199120448
:10EBF000914202D0019A944506D1002F06D0009A86
:10EC000006998958B94201D06D1C40E070468001D8
:10EC100005D50023264A2046019902F063FFE168EA
:10EC200009980858C20101D480010CD500980858F1
:10EC300000F0F2FDE16800980858FDF7EFF9E1688F
:10EC4000009800220A50284607E0E268C1005318E5
:10EC50000831521806CA06C3401C618C8905890E0A
:10EC6000491E8142F1D8618C3F228805800E000147
:10EC7000103880051201800D91430843608480059F
:10EC8000800EC100E068FDF7EDF9E0600120618CC5
:10EC90008905890EA94295D8002806D0002E04D0F7
:10ECA000324620460199FFF7BDFE0BB0F0BD0000D3
:10ECB000FFFF0000F0B507461646084693B00D4624
:10ECC00030431CD0012B1CD03D493846F8F752FB8D
:10ECD0003C493846F8F74EFB002209213846FBF73D
:10ECE00019FB01280BD1324629463846F2F763FE5C
:10ECF000012804D100220A213846FBF70BFB13B090
:10ED0000F0BD3846FEF7EAF811906846F8F77AFB4E
:10ED1000FF242D48913400970390002D26D01198A0
:10ED2000F8F756FF400080102A460021F8F7B0FBA4
:10ED3000C82801D2C82002E0A04200D920460B908A
:10ED40003846FEF73CFA4142281A0A901D480190C5
:10ED50001E480891099107906A4609213846FBF739
:10ED6000D9FA0128CBD16846F8F7A2FB002EC6D00D
:10ED70001198F8F76FFF4000801032460021F8F735
:10ED800087FBC82801D2C82002E0A04200D9204653
:10ED90000B903846FEF71AFA4142301A0A9008489A
:10EDA00001900A480891099107906A46092138465E
:10EDB000FBF7B0FA0128A2D16846F8F779FB9EE785
:10EDC000531401083D1401089B1101083574000813
:10EDD000FFB51546084681B00C46284362D001981D
:10EDE00000F0EEF90198FEF7EAF9404200B2009017
:10EDF000001904B200210198FEF749FD012813D043
:10EE0000002C13DC25DA0198FEF706F90646019876
:10EE1000FEF764F9301800B2002800DA0020404202
:10EE2000844216DA04B214E0002C01DA002410E067
:10EE3000002C0EDD0198FEF7EFF806460198FEF76C
:10EE40004DF9301800B2002800DA0020844200DDBD
:10EE500004460198FEF7BAF9404206B2701905B2AD
:10EE6000002D01DD002511E0002D0FDA0198FEF7DD
:10EE70009FF907460198FEF777F8381800B2002886
:10EE800000DA00204042854200DA05B20098201ADC
:10EE900001B2A81B02B20846104303D0049B01989C
:10EEA000FFF708FF05B0F0BD70B516461D460446D5
:10EEB0001A4600F023F82A463146204600F032F880
:10EEC00070BDF8B50E46044600F07AF900200090B7
:10EED0002046FEF73DF82746054614370AE033463C
:10EEE0006A462146384602F05FF92C462046FEF776
:10EEF0002FF80546002DF2D1F8BD000070B50D4683
:10EF0000144606460649F8F735FA3046FEF757F933
:10EF1000401B01B2234600223046FFF759FF70BD67
:10EF20003D14010870B50D46144606460649F8F72B
:10EF300021FA3046FEF74AF9401B02B2234600216F
:10EF40003046FFF745FF70BD531401081FB5044656
:10EF500002AA6946FEF741F96846F8F734FB002833
:10EF600004D102A8F8F72FFB002811D06846F8F763
:10EF70002AFB002803D069462046FFF79EF802A826
:10EF8000F8F721FB002803D002A92046FFF795F8E7
:10EF90001FBD70B50C460546FDF794F9A868017EC3
:10EFA0008A07920FA24208D08908A2078900920F0F
:10EFB000114301762846FFF760F870BDF3B591B0B4
:10EFC00011981299008C88427ED004901198018487
:10EFD000129A04991198F2F7D9FD0990002873D07C
:10EFE0000524E4012046FCF7BFFF21460390FDF70E
:10EFF0000AF9002420466DE011980299C068CD00FE
:10F0000041192D1D0A9140590002000A00F0A2F892
:10F0100005901198C06840590002000A00F096F867
:10F02000069012990598884352D10A984068800149
:10F030004ED40A980BAA0068672100F069FA0128EB
:10F0400046D100200B9D39E000261AE014200399D8
:10F05000704341180F914868079000F07BF80890C2
:10F06000079800F073F82968CA5B0F9909898A42EA
:10F0700006D10699884203D105990898884202D2A0
:10F08000761CA642E2D3A64216D120461422504353
:10F09000039AA9891152039A298A80184180A96884
:10F0A000C1602968C95B0181696801610A99496881
:10F0B0000902090A641C41600D98401C0D902968E2
:10F0C0004700C85B002800E031E001D0202CBBD312
:10F0D0000298401C02901198408C8005810E029885
:10F0E000814201D9202C87D300250EE014200399FA
:10F0F00068434618706800F029F801460096129B94
:10F10000049A1198F2F79CFC6D1CA542EED303986B
:10F11000FCF772FF099801280BD003280DD00228B4
:10F1200005D11198FEF7A9FF1198FFF733FC13B032
:10F13000F0BD1198FEF7A1FFF9E70F21024A09047B
:10F140001198FFF76FFCF2E7FFFF0000FF210904B1
:10F150000840704780B27047FFB581B01E46154623
:10F16000070017D0F2F721FC022815D00024002E4A
:10F1700014D0002D07D03846FDF7EAFE33462A4664
:10F180000299FFF7E9FF002C04D032463846029975
:10F1900002F0FCFC05B0F0BD0124E8E7002C04D02F
:10F1A00032463846029902F0F1FC002DF2D0384682
:10F1B000FDF7CEFE33462A460299FFF7CDFFE9E779
:10F1C00070B50B4D2978002910D101212970FDF768
:10F1D000C3FE0446042604E0B04360842046F7F7EB
:10F1E00001FF608C4107F7D40020287070BD00003B
:10F1F0002000002008B5132805D3F8F7DFFA0090A7
:10F200006846008808BD04494000401801886846E7
:10F21000018088B208BD00003C1D0108FFB587B021
:10F22000044608981D461646002802D1F01FF938FA
:10F2300077D020882988401A00B2208061886A88A7
:10F24000891A09B26180089A002A7ED04348016871
:10F250001046914248D00746E1200001874200DD78
:10F260003F1A002F00DA3F180A213846F1F7BAF8A2
:10F270000290401C019002980A2148433F1A0298CC
:10F2800000B200F08DFD0590019800B200F088FDFD
:10F29000049002985A3000B200F082FD0390019869
:10F2A0005A3000B200F07CFD02900A20C11B059884
:10F2B000019141430498784308180A21F1F792F824
:10F2C00004900199039841430298784308180A2151
:10F2D000F1F788F80146049842112048491142602C
:10F2E00081601E490898086000210220615E205E4E
:10F2F000F21FF93A17D0194B9A685B6894461F467B
:10F300004A434743D21B724397142A884B43BA1887
:10F3100022806246424398187043801469884018DE
:10F3200060800BB0F0BD0D4A936852681E461746C8
:10F330004E434743F61B2F88B612F6194A43434300
:10F34000D01826808012E9E7FFE770432A88001270
:10F3500080182080714308125988E0E74C00002093
:10F3600010B504220023825EC35E4088D21AD40FF7
:10F37000A218521012B20C889B1880184988E31A00
:10F38000081A1BB200B25B43404352431818904224
:10F3900001D8012010BD002010BD000010B5084BA1
:10F3A00004461A68091B50035040420C4240500169
:10F3B0005040491C1860F1F707F8081910BD00000B
:10F3C00058000020FEB50E46002507462A46143197
:10F3D000F1F769FE002828D001213046FEF786FCAF
:10F3E000002821D13046F2F7E0FA00281CD1002194
:10F3F000684601706A46122130460197FAF78AFF83
:10F400006846007802280FD03046FDF7F9FC401E10
:10F4100004000DD4B068A100006841583846FFF7D9
:10F42000D1FF050009D101E00020FEBD641EF1D529
:10F4300068460078002800D135462846FEBD000009
:10F44000F0B585B0002553E04919FF312131097C21
:10F4500000294CD1002443E00119FF312131097CFE
:10F4600000293CD1A5423AD0E10003910918EA00F5
:10F470001018303030310292F1F765FE00282ED09E
:10F480002048039940680A180299303209186846E2
:10F490003031F1F751FF6846F8F795F819490646FB
:10F4A0000298496840183030F8F78DF8154907463A
:10F4B0000398496840183030F8F785F838188642C4
:10F4C0000DD2104E02987168401869463030F8F736
:10F4D00047F8706801210019FF3021300174641C65
:10F4E000084EFF2170685131095AA142B4D86D1CF1
:10F4F0000448FF2241685132525AAA42A4D805B0AA
:10F50000F0BD00002C00002010B500F053F810BD35
:10F5100070B514468288264DC379AA4218D10022BC
:10F5200013E00568D600AD192E88B604B60C8E42DD
:10F530000AD12888010430D4400401D530461CE0AB
:10F5400068682060012070BD521C9342E9D82CE00D
:10F55000002B2AD0012B1AD90668980035180022F2
:10F5600012E05000285A8004800C88420BD15100D0
:10F57000695A0B0411D4490402D500F079F8E0E788
:10F58000900080190FE0521C9342EAD80DE09304DA
:10F590009B0C8B4209D1110401D5022070BD51048E
:10F5A00001D51846E9E70068CBE7002070BD0000F0
:10F5B000FFFF000070B514468288264DC379AA4229
:10F5C00018D1002213E00568D600AD192E88B604C4
:10F5D000B60C8E420AD12888010430D4400401D5EB
:10F5E00030461CE068682060012070BD521C9342C8
:10F5F000E9D82CE0002B2AD0012B1AD906689800F4
:10F600003518002212E05000285A8004800C8842ED
:10F610000BD15100695A0B0411D4490402D500F0F2
:10F6200027F8E0E7900080190FE0521C9342EAD8D7
:10F630000DE093049B0C8B4209D1110401D50220EB
:10F6400070BD510401D51846E9E70068CBE70020FA
:10F6500070BD0000FFFF000010B50821FCF7D3FDCE
:10F6600010BDC079002801D00020704701207047EC
:10F670001CB50022FF21452854D01EDC302844D080
:10F680000EDC222841D006DC032852D0062850D0B8
:10F69000202830D135E0252844D029282BD141E03D
:10F6A000362832D004DC31283CD0332823D13BE04B
:10F6B000372837D044281ED127E0552825D00EDC26
:10F6C0004E282FD006DC46282CD047281DD04D28A8
:10F6D00011D11AE0522818D053280CD122E060280A
:10F6E00020D004DC56281DD0572804D11FE0612803
:10F6F00018D06D2802D0009200981CBDFF20013068
:10F7000013E0FF221146104602E000221146104687
:10F71000F8F7EAF801906846808801906846818889
:10F720000180E9E70091E7E70F200090E4E7024855
:10F73000FBE70248F9E7000068560108FF1F0000D8
:10F7400010B50C46F2F73CFB204000D0012010BD64
:10F75000F3B5044681882F4881B0814258D0E079C2
:10F76000002851D0012804D0266881007518002196
:10F770004CE089040298890C814249D10020A08084
:10F78000E07140E04A00AA5A9304029A9B0C93420B
:10F790003BD1022811D00621401E4843FCF7B6FB9E
:10F7A000002831D02060E1798446491EC9B2E17158
:10F7B00089000A18002001461FE00120E07100299D
:10F7C00004D02888A0803068206019E06888A08074
:10F7D0007068F9E743009E46EF5A029B9F420BD0A8
:10F7E0008F006346FB188700BF193F681F60734690
:10F7F0004F00EB5AD353491C401CE3798342E9D2B2
:10F800003046FCF70BFC0120FEBD491C8842B9D8EC
:10F810000020FEBDFFFF000010B5044680880749A8
:10F82000884209D0E079012802D92068FCF7F6FB6C
:10F8300008212046FCF7E7FC10BD0000FFFF000098
:10F8400010B5024B00F008F810BD000051F8000898
:10F850001080196070470000FFB504468088394960
:10F8600081B01D4688424CD002998E04E179B60CD5
:10F870000092012933D9226888001318481E0DD43C
:10F880004700DF5BBF04BF0CB74205D18100891878
:10F890004000C2180B4631E0401EF1D50620491C3D
:10F8A00041431046FCF7DEFB01002AD02160E079DD
:10F8B0008200521803E04300D75A9B189F80401ED5
:10F8C000F9D5E079401CC0B28200E07153184000C5
:10F8D000C218191F0B46921E0099029827E00129B1
:10F8E00006D00120E0712346221D009902981EE0F7
:10F8F0008004800CB04206D12346221D0099029854
:10F90000A84705B0F0BD0C20FCF700FB0028F8D09C
:10F9100021682060E279521CD2B2E2719200121882
:10F92000A3881380031D0160921C00990298A847C8
:10F930003046F2F73EFAA179012282401143A171CB
:10F94000DFE70000FFFF000070B5044600F00EF88E
:10F95000050008D02046044A0021FFF71FF9214680
:10F960002846F2F78BFC70BDFFFF0F0010B5002892
:10F9700002D0FDF7B3FA01E0F8F710F9F8F762F9F1
:10F9800010BD10B5044600F003F8001B10BD0000C8
:10F990000349012248680A700B78002BFBD070479E
:10F9A00044000020034900220A704A681018486089
:10F9B0007047000044000020F8B5074615460E4683
:10F9C0000A48F1F739FF04000FD00020A760C043B8
:10F9D0002660206100206061FFF7DAFFE56060606B
:10F9E0000349012008712046F8BDFEE7EC10002015
:10F9F0006C00002010B5044601460548F1F799FF58
:10FA000004490120C8702046FCF708FB10BD000027
:10FA1000EC1000206C000020FEB54B4CA0780028B4
:10FA200001D00120FEBD0120A07020780026002812
:10FA300005D0FFF7ADFF0090002802D007E0A670C8
:10FA4000EFE72069401C2061642800D926613F4D02
:10FA50000020E07020713E48F1F7D5FE28603AE0C2
:10FA60003B48F1F7D4FE2E680746307DC00731D100
:10FA70000190304600F07DF8002812D130690190E5
:10FA8000002801DD401E3061FFF782FF7060B16821
:10FA9000002904D00198002801D030468847012071
:10FAA0000190E078002805D13069002802D1304665
:10FAB000FFF7A0FF019800280CD02079E1780843D7
:10FAC00008D028680028C3D10025ED432048F1F76D
:10FAD0009AFE11E02F6029680029C1D1F4E7307D3A
:10FAE000C00705D1304600F044F8A84200D20546D0
:10FAF00031461748F1F78BFE0600F0D10098FFF76A
:10FB000040FFE1684018E060A068FFF73AFFFF227D
:10FB1000F5320146904213D3E06864225043F0F777
:10FB200053FCC0B26070642801D9002001E0642158
:10FB3000081A607000202646E060FFF729FFB060D9
:10FB40000020A0702846FEBD6C0000209C00002014
:10FB5000EC10002001214161704710B50446FFF709
:10FB600017FF2168401A401E606010BD00214161EE
:10FB7000704710B504464068FFF703FF21688142D3
:10FB800001D8002010BD081A10BD000070B5034652
:10FB9000083A9007800F121A0C46880704D11046C5
:10FBA0000F490C38884201D3002070BD207802250F
:10FBB0008107890F114301200143A943261F2160BA
:10FBC00031461846F2F7FFFC3046F2F734FD017972
:10FBD0008907890F4908490029434160204670BDC3
:10FBE000F50F000070B5810701D0002070BD806066
:10FBF0000023C0601A460361940021184B61002164
:10FC0000D40124188E00A619491CF0622029F9DBC2
:10FC1000521C062AF0DB70BD70B50D460646FFF794
:10FC2000E1FF0446CB2080002A1A81192046FFF705
:10FC3000ADFF204670BDF8B50026002923D0083955
:10FC40004E6805460C46F00700D0FEE70846F2F77E
:10FC50004BFD2179284689070DD52768002F14D040
:10FC60003979C90712D03946F2F7A8FD214638463E
:10FC7000F2F78EFC044621462846F2F74FFD014676
:10FC80002846F2F7A0FC3046F8BDFEE7FEE770B567
:10FC90000A46054604211046F2F798F90446014643
:10FCA0002846F2F7CEFC014622462846F2F75CFDD4
:10FCB00070BDF7B584B0049800250C46019000296A
:10FCC00024D0069800281DD02546083D2846F2F786
:10FCD00040FD00906868042187080098BF004068D4
:10FCE00080088000C019001D02900698F2F76EF996
:10FCF00006460698B84201D9002E0DD02879C007D3
:10FD00000DD0FEE70498FFF796FF47E006990498A8
:10FD1000FFF7BDFF054641E0002007B0F0BDBE4241
:10FD200017D900980079C00702D00298864210D9EE
:10FD300006990498FFF7ABFF05002FD0069887427D
:10FD400000D307463A4621462846FCF7A3F9214648
:10FD5000D8E7BE4206D929460198F2F7DFFC2846CB
:10FD6000F2F7CFFC2879019FC00700D0FEE73146AB
:10FD70002846F2F71EFC00280FD031462846F2F73D
:10FD80002EFD416802229143416001463846F2F758
:10FD9000C5FC01463846F2F716FC25462846BCE766
:10FDA00010B5FF2469342146F0F71CFB002901DA65
:10FDB000091909B20C4A5A2901DA480007E0084635
:10FDC0005A385A2805D2B420401A00B24000105EBA
:10FDD00010BD0846B4385A2800D3601A00B240005B
:10FDE000105A404200B210BDB81E0108FFB585B0E0
:10FDF00005980F9F00287CD00078002879D00698BD
:10FE0000002874D00E98800701D54348089000243C
:10FE1000601E424A0194039402940490526825465D
:10FE2000264601A90598904700900198039053E059
:10FE30003A4A03A952680598904702900E98761C9A
:10FE4000C00705D000991098F2F784F800283ED139
:10FE5000029A00990698FAF748FB00B229180DB2E9
:10FE6000002802DD0798281805B20498401C05D127
:10FE70000798291A0898814200DD049400980A28FE
:10FE80001AD00D2818D0014627204002244A081A0B
:10FE9000904211D9002005E022A2125C8A420BD0C8
:10FEA000401CC0B21FA2125C002AF5D1002F0ED058
:10FEB0000498401C0AD00AE0002C05D10498401C8C
:10FEC00002D1002F00D03D60761E09E03D60019C0C
:10FED00003980190029800900598005D0028A7D132
:10FEE0000498401C06D0119800280ED0049809B040
:10FEF000F0BD0EE0002E05D000980D2803D1029829
:10FF00000A2800D1019C2046F1E7002F01D00020F3
:10FF100038600020EBE70000FF1F00008000002099
:10FF2000A5510000202C2E3B3A2D5F00FFB5044662
:10FF3000002085B020800F46608000294ED00798B1
:10FF400000284BD01098800701D526480F90002537
:10FF500002950798068929E00020009010997819E9
:10FF6000019103900F9B089A0799F1F771FF02998D
:10FF70001D4A4018029002200E99205E7118411807
:10FF800091422BD80E9980194018608010980090EB
:10FF90000298089B411B079A039800F027F800215C
:10FFA000615E814200DB08462080029D785D00286A
:10FFB000D2D1002D0BD078192038C07F0A2801D06B
:10FFC0000D2804D10E98618830180818608002202E
:10FFD000205E002804D00E99401A608009B0F0BD60
:10FFE0006680FBE7FF1F0000FF7F0000FFB585B0C4
:10FFF0001E460D4607000DD0079800280BD0387814
:020000040801F1
:10000000002808D000206946029004460873002D9D
:100010001DD123E0002009B0F0BD02AB01AA694662
:100020003846F1F7FDFE0E98C00705D003A80099E9
:10003000F1F790FF00280AD1019A00990798FAF782
:1000400054FA00B2002802DD2018801904B2029888
:10005000A842E2D3002C01DDA01B04B22046DAE75F
:10006000F8B500240F460646254608E00749301932
:1000700009688847002800D1012004196D1CBD4281
:1000800002D2305D0028F1D12046F8BD800000206A
:10009000F8B5074600200D460446064E009004E0E1
:1000A0007268694638469047641C0098A842F7D3A6
:1000B0002046F8BD80000020F8B500240546074E14
:1000C000009404E07268694628469047641C0098D2
:1000D000285C0028F6D12046F8BD000080000020F2
:1000E00038B5002403460094002900D169460A6807
:1000F000985C050601D404460FE04509062D06D09C
:1001000005090E2D0DD0C5081E2D0DD005E0C00629
:10011000400D1DE09B069B0E1C18521C20460A60D9
:1001200038BD0007000C0AE0521C0A609C5C4007C6
:10013000C00AA509022D11D1A406A40B2018521C37
:100140000A609C5CA509022D08D1A406240D201884
:10015000521C0A609B5C9C09022CDBD0002038BD3D
:10016000F8B5074608680025401E0C460E4E08608C
:1001700001E0042D15D220683168C0198847002895
:1001800004D1216800290CD0491E21606D1CEDB2FC
:100190000028EED020680090726869463846904783
:1001A000F8BD0020F8BD00008000002000780106A6
:1001B00001D4012070474109062907D001090E2901
:1001C00006D0C0081E2805D00020704702207047C6
:1001D00003207047042070472B4896B082690121A4
:1001E0000A4382618069084014900807F0F72EFBEB
:1001F0000321081FF0F75EFEF0F7FEFDF0F724FC88
:100200000120F0F717FB00210B20F0F753FE01202F
:100210001E49C0020860F0F7D9FC6420F0F7E6FB45
:10022000FBF730F9F0F782FA7D20C000F0F7DEFB33
:100230001923DB01002216491648F7F7D3FB68465D
:10024000F7F7DCFB134803901348FF210590413179
:1002500068460180F0214180F7F7FEFB6420F0F74B
:10026000C5FBF7F79BFCF7F7DBFCFBF76DF90BA180
:10027000FBF7F4FD0520F0F7B9FBFFF7CDFB0A20F3
:10028000FFF790FBF6E700000010024000E100E0FD
:100290006817002068300020E106000873696E6767
:1002A0006C6520667265713A00000000F0B58E88BA
:1002B0000F888DB0F61B761C37B2CE88498804466D
:1002C000711A491C1D46169809B2129B0891012803
:1002D00005D0022805D0032850D1524802E05248E8
:1002E00000E05248069051000B91149859000A9171
:1002F00000282188684601802988818005D01498CB
:100300000078FD283CD313983DE0069B139A009992
:1003100001989847079000202CE0002622E06846CC
:10032000818870000390285A814205D1684601886F
:100330000398205A81420FD003980019018868461B
:10034000018003984019018868468180069B139AB2
:100350000099019898470790039869460019898B7E
:100360000180761CBE42DADB0B9804190A98451905
:100370000498401C089904908842CEDB0DB0F0BD73
:1003800013994843000A02460390069B009901987E
:1003900098470C9000203FE0002631E01498805DE3
:1003A00000282CD0FD2801D3139802E0139948436C
:1003B000000A69468A8871000791695A8A4208D101
:1003C00069460A880799615A8A4202D10399814293
:1003D00010D0079909190A8869460A8007994919AE
:1003E0000A8869468A8002460390069B0099019814
:1003F00098470C90079869460019098E0180761C71
:10040000BE42CBDB0B98159904190A98451914982C
:10041000401814900498401C0146049008988142AA
:10042000BADBABE75D2E0008D92D0008C72E000807
:10043000F0B51C468B880E888FB09B1B5B1C1FB2CF
:10044000CB8849880546591A491C09B21498049169
:1004500051004000169B0B910A901598002B05D077
:10046000FD287DD9381F039000202DE1FD2811D3F0
:1004700000267F0009E03A4621462846FBF70AFE9F
:100480000B9845190A980419761C04988642F2DBE9
:100490000FB0F0BD00201DE0002613E070004219EF
:1004A0000392128869460A83001900888882159A87
:1004B00006990598F7F72EFA05906946039A888AF7
:1004C0001080761CBE42E9DB0B9845190A98041986
:1004D0000198401C049901908842DDDBD8E716980A
:1004E000002605901BE005980278002A13D0FF2A09
:1004F0001CD071004819099000886B4618840819AF
:100500000088988308990798F7F704FA06906B46D5
:100510000998198B01800598401C761C0590BE42F5
:1005200001DA8007DFD105980C9077E0700041195F
:10053000001900880880EEE7006800286AD0401C97
:1005400074D00C9805900278002A15D0FF2A7DD02F
:10055000730058190990008869460884181900E04A
:10056000BEE00088888308990798F7F7D3F90690CA
:1005700069460998098B01800598401C059002780E
:10058000002A14D0FF2A67D071004B19981C0890DC
:1005900058886B4698840819408898830999079869
:1005A000F7F7B8F906906B460898198B0180059803
:1005B000401C05900278002A13D0FF2A52D0700008
:1005C0004119099189886B4619840019808898839C
:1005D00008990798F7F79EF906906B46188B0999CA
:1005E000888005984278002A14D0FF2A3FD07000F6
:1005F0004319991C0591D9886B4619840019C08844
:10060000988308990798F7F785F906906B4605993E
:10061000188B88800C98001D361D0C90039886421C
:100620000C9889DB059043E000E00FE07100481969
:1006300009190A88831C02809C464B8843808A1CC7
:1006400089888180634690889880E3E7700041192B
:100650000019008808808FE7700041190019408850
:100660004880A4E77000411900198088B8E770003D
:1006700041190019C088C880CCE70278002A13D03D
:10068000FF2A27D071004819099000886B4618840A
:1006900008190088988308990798F7F73BF906909E
:1006A0006B460998198B01800598401C761C0590B3
:1006B000BE42E2DB0B98179945190A98041916985F
:1006C000401816900198401C04990190884200DA65
:1006D00005E7DDE670004119001900880880E3E7AE
:1006E00000202BE000261DE01698805D002818D021
:1006F000FD2801D3159A02E015994843020A7000BB
:100700004119039109886B469982001900889883E2
:1007100005990798F7F7FEF805906B460399988AB4
:100720000880761CBE42DFDB0B98179945190A98A2
:1007300004191698401816900198401C04990190CD
:100740008842CFDBA4E6FFB58DB00C46169DF1F7CD
:1007500029FB0A90A0882188401A401C06B2E08834
:100760006188401A401C00B20690690018980991EF
:10077000002822D0002050E0002516E017980290B3
:100780001098690008180088694688806188039875
:10079000081800B2009020880F9A401903B20A98F6
:1007A0000D990068C769B8476D1CB542E6DB109922
:1007B0000998401810900398401C069903908842AD
:1007C000DADB11B0F0BD00251BE0405D002817D03A
:1007D00017994843000A0290109869000818008889
:1007E0006946888061880398081800B200902088C4
:1007F0000F9A401903B20A980D990068C769B84763
:100800006D1C1898B542E0DB1999401818901099A2
:100810000998401810900398401C0699039088424C
:10082000D1DBCEE770B515460E460446802805D2CA
:10083000E117890F002009198C1006E001F035F846
:10084000411FCC4020214C40801F30602C6070BD87
:10085000FD2902D2022901D80020704748430249ED
:1008600048434000000E70478180000070B5094D7C
:1008700004466868002809D0002C08D02046F6F706
:100880007FF8A9682018884200D3002070BD024874
:10089000006870BDC4000020A8000020002903D01B
:1008A0000068091D401802607047002902D00068E6
:1008B0004018026070470000F0B5504E0546706861
:1008C00089B00168CC6BC9688968216001680969D1
:1008D0008A0701D4C90726D0F7F7BCF9401E07B232
:1008E0007068F7F775F9401E03B20022114601A89F
:1008F0000097F6F7A2FE01A9616070680068027CAB
:10090000C068920705D5826902231A438261A160FB
:100910006EE08169C9078A0F8169022399431143F7
:100920008161A56064E0A9882A88891A491C09B2F6
:100930000391E9886A88891A491C09B20291F7F77C
:1009400089F901460620285E814203DC7068F7F7CA
:1009500081F9401E07B22948029A03994068F6F7C8
:1009600007F9002603900220285E23E02B886A46C0
:100970001382AB8893825082D18204A86060A06009
:100980001E4840680168C968896821601621515E67
:10099000B94200DDD7821626965FB74205D10068BE
:1009A000C0688169022211438161204600F028F865
:1009B000079800B2039941180791491EB942D5DD45
:1009C000B74218D02A8869460A82AA888A82488251
:1009D000CF8204A86060A060084840680168C968C8
:1009E000896821600068C0688169022211438161C1
:1009F000204600F005F809B0F0BD00002C000020F2
:100A0000F0B5644C074691B06068F7F7DDF8F96817
:100A10000546002901D038468847606800210068F3
:100A20000222415E825EE8685143814201D1012089
:100A300000E00020296800290ED06968002908D04C
:100A4000002806D108E060680068816A002900D0AB
:100A5000884728690028F6D100256068F7F7E0F894
:100A60007A6801461046FEF7ADFC064660684169AB
:100A7000002903D07868FEF7A5FC054630462843D8
:100A80004DD16068F7F7E6F8401E00B2009060684C
:100A9000F7F79EF8401E03B2002211460EA8F6F7A3
:100AA000CCFD386B002814D06846F8F7CDF96168A2
:100AB0006A46C86A049008462030437A9376498D86
:100AC0009180407AD0703B6B0EAA694638469847B1
:100AD00025E06068C06A002813D006A9FAF7EAFB8F
:100AE00001281CD16846F7F70BF960682921095CD9
:100AF0006A46D172C36A0EAA69463846F7F7D0F83B
:100B00000DE06846F8F7A0F960686946428D8A8072
:100B10002030407AC87038467A68F8F781F9606802
:100B20002821095CC9070FD0002E00D1066938467C
:100B3000314600F0A1F960684069002816D0002D08
:100B400000D1054629460EE04069002806D0002D58
:100B500000D105462946384600F08EF9002E01D115
:100B6000606806693146384600F086F96068F7F734
:100B70004EF80146384600F07FF96068F7F73EF816
:100B80000146384600F078F96068F3F7B1F911B022
:100B9000F0BD00002C000020F8B52E4C0020206095
:100BA000FF2061685130405A002852D0002505E0EE
:100BB0000A18FF322132127C002A1AD0401EF7D5C3
:100BC0000868416B002900D0884760680168C968DF
:100BD0008A69520852008A610168C9688A690227D5
:100BE000BA438A612030017A04221143017200263F
:100BF00024E00546E4E78119FF312131097C002911
:100C00001BD1AE4205D10168C9688A6901231A4324
:100C10008A610168CA689169B9439161F100081855
:100C200030300091FFF748FE0099606808183030B6
:100C3000F6F7C9FC216840182060761CFF21606827
:100C40005131095AB142D6DC2030017AFB221140E1
:100C50000172F8BD2C000020F3B50C468DB00121C7
:100C60002046FDF743F8002831D12046F0F79DFEDD
:100C7000050028D0204600216122FCF7C8FEC0B242
:100C80000B90022823D302AB2A4621460D98F6F793
:100C90005CF901281BD1214601270022143102A84A
:100CA000F0F701FA002815D000216846017002A86B
:100CB00001906A4612212046F9F72CFB684600781D
:100CC000002806D006E021460D98FDF763FB0FB023
:100CD000F0BD0027012D01D1022007433A4602A9A9
:100CE0000D98F7F7FDFA0500F1D0204600216F229C
:100CF000FCF78DFE00B26946088001900A902046FC
:100D000000217022FCF783FE06B269464E800A98E5
:100D10004004800F012817D103210198490388431B
:100D20007D21090188420FDC218BA28A891A491C86
:100D30000AB27D21C900884200DD081A50436421AF
:100D4000EFF750FB694608807004800F012816D128
:100D50000320400386437D20000186420FDC608B28
:100D6000E18A401A401C7D21C90000B28E4200DD9C
:100D70008E1B70436421EFF735FB6946488004A859
:100D8000F6F7BEFF69460B98C876204600216E2212
:100D9000FCF73DFE00B269460882E1210901884264
:100DA00001DD401A02E0002802DA40186946088294
:100DB000204600216D22FCF72AFE69464882204623
:100DC00000216822FCF723FE69460877294808A914
:100DD00040680068007C0007C00F0871B8073CD568
:100DE00003CD69602860688869894018401E00B298
:100DF000E880083D0621695E88422EDDE9812CE00D
:100E0000B80705D53B462A4620460D99F6F76AF8FD
:100E100021460D98FDF7BEFA6846A18A008804AA0B
:100E200009180D9840680088091A68468182E18A8D
:100E3000408809180D9840684088091A6846C182A0
:100E400029460D98F7F747FAB8070DD5E889401CF1
:100E50006881698A4018401EE8810A206A460E218E
:100E6000285E515E8842CBDD29460D98F7F768FA77
:100E70002DE700002C000020F3B581B00C0005D157
:100E80001B484068F6F7CCFE04002BD021460198A1
:100E9000FFF7E2FE20E00027FBF7B2FF0646002541
:100EA00009E0A068A9000068002F41581BD00198F4
:100EB000FFF7D2FE6D1CB542F3D317212046019AED
:100EC000F9F728FA18212046019AF9F723FA19218F
:100ED0002046019AF9F71EFA20460094FCF738F8EC
:100EE0000400D8D1FEBD00988142E3D10127E1E79B
:100EF0002C000020F0B5464C8FB0606801680A7C79
:100F0000D2077DD0C968496800297ED0FF305930AA
:100F1000F0F703FD002878D160680168CA6893681B
:100F20000D9311688B4200D151680C91F6F750FE79
:100F30000B90202103A8EFF7F4F900253CE04119BC
:100F4000FF312131097C002935D1FF305930F0F7CC
:100F50005AFC06462DE02E4C31466068FF30593071
:100F6000F0F755FC00906168E8004218314603A88C
:100F70003032EFF7D9FF0746401C19D000240BE0B0
:100F8000FF305930F0F778FCE20003A9511808222D
:100F9000EFF768F9641C64B21D48BC4240683146F2
:100FA000EEDBFF305930F0F7C4FC3046FBF736F883
:100FB000009E002ECFD16D1C154CFF216068513171
:100FC000095AA942BBD825466868FF305930F0F766
:100FD0001AFC11E00C980B996A4613C268680A461D
:100FE00000682346C06B0D99866BB0476868214640
:100FF000FF305930F0F70BFC0400EBD1686800E0DB
:1010000003E0FF305930F0F7E8FB0FB0F0BD00000F
:101010002C000020F8B50746FBF7F2FE0546002439
:1010200012E0B868A100006846583046FDF725F880
:1010300000222A213046F9F76DF93046FDF71DF8F8
:101040003046FFF7E7FF641CAC42EAD3F8BD70B549
:10105000CD688C68002D1BD0002C1AD0E560AC60E8
:10106000D5012D189E00AD19EE6A8E420FD1EC62AB
:1010700084420CD191000D180124264669699E40D6
:10108000B143696103D101699440A143016170BD1D
:10109000FEE7FEE7FFB582B086468C460022119F30
:1010A0000B9E0C9D0F982EE00D990E9B51435343C0
:1010B00009121B128C195B1924121B12002C06DB5F
:1010C000644504DA002B02DB04998B4201DB002328
:1010D00016E005994B4300931B195B007344019381
:1010E000109B5100C918019B1B880B80059B04991C
:1010F0004B435B0071465918009B0C1919190B786A
:10110000BB54521C12B28242CEDB06B0F0BDFFB51A
:1011100081B00E9E0A9D0B9CF0F744FE006831469C
:10112000806B00901098FBF798F80020024630E0A2
:101130000C990D9B4143434309121B1249191B197A
:1011400009121B12002907DB029FB94204DA002BA7
:1011500002DB039FBB4202DB10990A540BE0019FA4
:10116000BC46049F7B43591849000F9B61444700CC
:10117000FB18098819801199062908D10F99430095
:10118000C95A6B461B88994201D110990A54401CD8
:1011900000B2B042CCDB05B0F0BD10B50068002253
:1011A0000A21F9F7B7F810BDFFB58DB00C46084617
:1011B000FBF7CEFE06461021FCF798FD002874D000
:1011C0003046FBF71FFF079000253046FBF7E9FF8D
:1011D000143408940990002800D10D9C0021304659
:1011E000FCF781FB059000213046FCF70AFC014624
:1011F0000598081807B200213046FCF7DEFB0146CF
:101200000598081800B20490F08A6188C019421A43
:101210000F984188501A00B20090728B0498101AEF
:10122000E288801A081A00B20B903046FBF78AFE5B
:10123000C11B0498081A00B20A90009800280CDB21
:101240000B98002814DA0098002806DD0546304681
:10125000FBF7AEFF401B0AD40AE00B98002807DD1D
:10126000404205B23046FBF77FFEE84200D500253C
:101270000998012804D0022806D003280CD115E0D3
:10128000F08A6188C01903E0718B0498081AE1881C
:101290004919401A401905B200243046FBF77AFF7D
:1012A0000990002815D0089F14E0C0E00A98F18A40
:1012B000C20F10184010C0190918E0886288801AFF
:1012C000401C00B2C30F1818401040191018081A1B
:1012D000E0E70D9F00213046FCF77BFB05994018A5
:1012E00000B2049000213046FCF77FFB05994018BE
:1012F00002B20592B18A0498338B08183988421AD1
:101300000F980188501A059A00B29A1ABB88D21A0F
:10131000891A09B200280ADB002912DA002806DD42
:1013200004463046FBF778FE001B09D409E000298B
:1013300007DD484204B23046FBF7D0FEE04200D55C
:1013400000243046FCF7CCFC0499411A0598081A91
:10135000099900B2012904D0022907D003290DD12F
:1013600024E0B18A04980818398803E0318B059885
:10137000081AB9880919401A001904B22D493046D3
:10138000F5F7F8FF07462C493046F5F7F3FF01461D
:101390003846084306D000220A213046F8F7BAFF43
:1013A000012844D10798C00712D014E0C20F1018CA
:1013B00042100498B18A10180818B9883A88891A16
:1013C000491C09B2CB0F5918491009195118D2E715
:1013D000002C00DA00240798800702D4002C00DDDE
:1013E00000240798400702D4002D00DA0025079852
:1013F000000702D4002D00DD00250F980021415E7A
:101400001098002800D0204608180F9908800F98DF
:101410000221415E1098002800D0284608180F9934
:101420002A46488021463046109BFDF743FC11B008
:10143000F0BD0000531401083D14010810B5034627
:10144000FBF7BDFE401801B200221846F0F7B3FAD0
:1014500010BD10B50346FBF7B9FE401802B20021DB
:101460001846F0F7A8FA10BDF8B505460C46084630
:10147000F7F7EAFC0126360431462846FCF719FA4C
:10148000E070022808D9284631462022FCF7BFFA2E
:10149000009068460088A080284631463122FCF73B
:1014A000B6FA2746C0B22037B870022814D92846A9
:1014B00031463222FCF7ABFA00B22084002809DD65
:1014C000284631463022FCF7A2FA00906846008890
:1014D000E08301E00020B870284631464522FCF741
:1014E00096FAC0B2B87502281AD928463146402269
:1014F000FCF78DFA00B2E08500280FDD2846432274
:101500003146FCF784FAA086284644223146FCF78F
:101510007EFA009068460088A08501E00020B8753A
:1015200031462846FCF705FAFD2807D2E178414309
:10153000090AE1704143080AB870B875E0780028DC
:1015400005D1B878002802D1B87D002805D03146F1
:101550002846FCF7A8FA20800120F8BD10B54422E7
:101560001152FCF78AFD10BD10B546221152FCF74E
:1015700084FD10BDF7B58CB004460D9846104010A0
:1015800005900D98C00700D1761E60000890FAF70C
:10159000EBFC054600200E9B26E00898C018099039
:1015A0004038C18F0D984143601E15D44200A952A6
:1015B000059F0022C719A74201DA7A009A5A8A1AAF
:1015C000811B012901D5198803E04900C918403958
:1015D000C98F5118401EE9D529461846089AFAF7CE
:1015E00059FD0298099B401C0290A042D5DBFF20C8
:1015F000800101900D99EEF7E7FE80B20990002777
:1016000020466043069012E0780004900E99085A34
:1016100000280AD00199884201D1099802E00D9969
:10162000EEF7E0FE0E9A0499505206987F1CB842DD
:10163000EAD8002039E00E99420051188E460A88F7
:101640000D99F4464A43002121E0002A01DA0023E3
:1016500000E093114F00EB53059BCB1A002B02DCEB
:1016600063461B8804E063431B185F000E9BDB5B33
:10167000D71A8A19521CA24200DB621E624312185A
:1016800053000E9AD25A089BBA189C44491CA14296
:10169000DBDB7246002105E04B00EB5A1380089B10
:1016A0009A18491CA142F7DB401CA042C3DB284624
:1016B000FAF7A2FC0FB0F0BDFFB58FB01F460D4684
:1016C0001646D4190E9201A80F99F5F76DFFF00F89
:1016D00080194110C819F207D217821A6846921E63
:1016E0000281491CC1800F98F5F787FF01466846C3
:1016F0000089411A684681800F98F5F75EFF014620
:101700006846C08800230918684641813A4601A905
:1017100008A8F7F7D3FA0E9E012E00D076102046C7
:10172000FAF722FC0490059500203DE0214604983C
:10173000FAF793FD08A800900698089F02B223B21A
:1017400000210498B847002809D004983146007851
:101750008001EEF747FE0599012708801CE0610033
:101760000598FAF750FD19E004990498C919203931
:10177000C05DC97F884207D105997800411840397A
:10178000CA8F05990A5206E080013146EEF72AFE1B
:1017900005997A0088527F1CA742E5DB0598610015
:1017A000081805900698401C0690A042BEDB0498DD
:1017B000FAF722FC08A8F6F7D9FF012E18D020B2BC
:1017C0002A4631460790FFF7D5FE0E98C007C00F96
:1017D000801900B2119001282BDD0146FF20800105
:1017E000EEF700FE002680B227466743009019E01E
:1017F0000020644304E04200A95A89092954401C8E
:101800008442F8DC13B0F0BD70000590285A00281F
:1018100007D0FF2810D080011199EEF7E3FD05995C
:101820006852761CB742EFD82A4611990798FFF7FD
:10183000A1FE0020644305E00098F0E74200A95CA7
:101840002954401C8442F9DCDCE7F0B597B0074628
:1018500014460D4601A8F7F7F7FAFF221146104685
:10186000F5F7D4FF0090684600880090684601882C
:10187000018100262A4601A93846F7F7D1FA0FA8B8
:10188000F6F7FEFC23462A460FA938460096F6F7DF
:1018900051FA17B0F0BDC14310B5491C0840EFF72D
:1018A000E4FA2021081A401E10BD10B5002803D00C
:1018B000EFF7DBFA2021081A401E10BDF0B50568CD
:1018C0000446688C0023800585B0800E0CE0DA00A9
:1018D000EE680392121DB258960104D51202A66852
:1018E000120AB24204D05B1C9842F0D805B0F0BD99
:1018F000A088844644285CD00EDC33284CD006DC1B
:10190000202856D0222854D0302813D151E0342832
:1019100042D036280ED14CE0622840D006DC472861
:1019200047D0552845D0572804D135E0672833D013
:10193000682831D000292BD0FF292BD02269E068FC
:10194000121A4A43111208180090E868D90040584A
:10195000012601AA6146FDF7D7FD002809D00199AB
:101960000098884205D1684601888088814200D16C
:101970000026E9680398009A0858A188FDF760FFDF
:10198000002EB3D0A288A1682068FDF74BF8ADE720
:10199000E068D9E72069D7E7FF29FBDAF8E7E068D4
:1019A0000028F7D02269002ACED08029CCDB009213
:1019B000CBE7002901DCA08902E0FF2902DB208AB5
:1019C00069461DE020690290E0680490C8B2001DDD
:1019D000C7086946088A0B4E0104084369460A890C
:1019E000304011040A433240111A7943490908185A
:1019F0003040020C024369460A8190B20290088985
:101A00000880A2E71FF8E007F8B50468A0882568F9
:101A100000902348EFF7F7FE10E0A1420BD00868D2
:101A20002268904207D18868A268904203D18888D2
:101A3000A28890422FD01A48EFF7E9FE0100ECD1BE
:101A4000688C00268005800E27E0F700EA68391DC3
:101A500051588A0120D50902A268090A91421BD176
:101A600021460F48EFF765FF2046FAF7D7FAE868F6
:101A7000F100441820680099FDF76AFEE868C05933
:101A8000FDF7EFFD002806D0606821680202120A07
:101A90002846FDF783F8F8BD761CB042D5D8F8BDCE
:101AA0004011002070B50468FF20A66800040640BD
:101AB000A28831462068FBF7AAFFE060A5880020D5
:101AC000A08023462A463146206800F00BF8A58006
:101AD000A1682068F5F736F9A1880068E268FDF78B
:101AE000AFFE70BDFFB5074681B00E460025254804
:101AF000EFF796FE04463FE0049884423ED021462C
:101B00002048EFF789FE00902068B84233D1A068E2
:101B1000B04203D00F20000486422CD1A188039844
:101B2000814202D01849884225D1002512E0E80000
:101B3000F968021D8A5893010BD50F231B049E429E
:101B400003D01202120AB24203D10858A188FDF74D
:101B5000FFFD6D1C788C8005800EA842E7D800211F
:101B60002046F5F707FC21460648EFF7E2FE20463F
:101B7000FAF754FA0125009C002CBDD1284605B087
:101B8000F0BD000040110020FFFF0000F7B582B05B
:101B9000044600216E22FBF73AFF05B220460021E1
:101BA0006D22FBF734FF06B2002D02D1F01FF93889
:101BB00067D0204600216F22FBF729FF6946088085
:101BC000204600217022FBF722FF69464880002052
:101BD000085E7D274104890FFF00012919D10321E7
:101BE000490388437900884213DC20461430F5F716
:101BF000F8FC024669460020085E03214903884339
